:020000040800F2
:100000000020001071ED0208A1B3020849A5000804
:100010009DB3020899B3020895B3020800000000DE
:1000200000000000000000000000000091B3020882
:100030008DB302080000000085B3020805BB00086C
:10004000D9ED0208D9ED0208D9ED0208D9ED020870
:10005000D9ED0208D9ED02080958020835590208FD
:10006000F9580208BD5802088158020811330008E7
:1000700001330008F1320008E1320008D1320008F3
:10008000BD320008A9320008D9ED0208D9ED0208F6
:100090006D990208D9ED0208D9ED02084558020809
:1000A0005DB20008ADB20008D9ED0208BDB200088B
:1000B0009DB200088DB20008D9ED0208D9ED020802
:1000C000D9ED0208D9ED0208D9ED0208D9ED0208F0
:1000D000D9ED0208014F02080DBC000891BB0008D1
:1000E000CD570208D9ED02085D990208D9ED020842
:1000F0006DB20008D9ED02087DB20008D9ED020802
:10010000000000000000000000000000D9ED02081F
:10011000D9ED0208D9ED02080D1B0108F11A0108FA
:1001200095320008813200086D320008593200080B
:1001300045320008D9ED0208000000000000000070
:10014000D9ED0208D9ED0208D9ED0208000000003F
:10015000000000000000000000000000000000009F
:100160000000000000000000D9ED0208D9ED0208EF
:10017000D9ED0208000000000000000000000000AF
:0801800000000000D9ED0208A7
:10018800002870B51EDB0928044620DD012303EB97
:1001980083035B00B0FBF3F2092AF8D87BB10E4E5B
:1001A800B4FBF3F00928CCBF57223022A6FB03E5A5
:1001B800024403FB1044EB0801F8012BF0D10023A3
:1001C8000B7070BD2D230B7040420131DBE73030DE
:1001D80001F8010BF3E700BFCDCCCCCC884230B49A
:1001E8004FF001042ED301FB04F4B0FBF4F58D426B
:1001F800F9D284B1AAB901E0B0FBF4F5092DCCBF5E
:10020800572230222A4404FB150003F8012BB4FBC3
:10021800F1F4002CF0D100221A7030BC7047B0FB0A
:10022800F4F5092DCCBF372230222A4404FB1500EF
:1002380003F8012BB4FBF1F4002CF0D100221A7062
:1002480030BC70470546002AEBD1D7E703685A1C33
:1002580002601970704700BF2DE9F047089C2578A7
:10026800002B804689460CBF4FF0200A4FF0300A19
:10027800661C35B3002A29DD334601E0024698B1F1
:1002880013F8011B501E0029F8D1971E60B13D4696
:10029800013D51464046C8476B1C002BF8DC2578C9
:1002A80027EAE770013055B1041B29464046C84784
:1002B800301916F8015B002DF7D1BDE8F087BDE8CD
:1002C800F087002A04DC2846BDE8F0870020EBE729
:1002D800571EDCE783684268D0ED037A00EB8301A0
:1002E8000133934281ED040A836004BF00238360D5
:1002F80000EB830393ED047A036870EE277A9A4241
:10030800C0ED037A77EEC77AC0ED037A0CDA0133D1
:1003180007EE103AF8EEC76AB7EE007A87EEA60A3B
:10032800036030EE070A704707EE102AB8EEC77A66
:1003380087EE870A704700BF90ED057A90ED004A76
:10034800D0ED066AD0ED014AD0ED047A90ED035A5B
:10035800D0ED025AA4EE007AB0EE406AB0EE470A39
:10036800B0EE667AA6EE247A67EEC07AA0EE457AF9
:10037800E6EE257A80ED057AC0ED067A704700BF73
:10038800D0ED057A90ED013AD0ED003AD0ED064A6D
:1003980090ED024A90ED077A90ED035A90ED086AC5
:1003A800D0ED045AC0ED067AF0EE406A27EE830AD3
:1003B800C0ED056AA3EEA60A80ED087AA4EE240A29
:1003C800A5EE470AA5EEC60A80ED070A704700BFEA
:1003D800D0ED007A90ED017A30EE670AE7EE007A08
:1003E800B0EE670AC0ED007A704700BF704700BFE3
:1003F8000A44914214D030B40139551E41F2210209
:1004080011F8014F082380EA042004044CBF82EA53
:1004180040004000013B80B2F7D18D42F0D130BCA2
:10042800704700BF4FF40063838270474FF4006346
:1004380083827047012380F84530704770B40468A0
:10044800037B2268022101FA03F31A4213D042699E
:100458000A495C2000FB02124FF6FE76506852896A
:10046800C5680068296831402960C168D24392B2E2
:100478000A40C260636070BC704700BFF44B002044
:1004880030B40A4B1D7875B1094B002003EBC50544
:100498001A6899885062D4682143D160083323F8D8
:1004A800040CAB42F4D130BC704700BFD44E0020DE
:1004B800D84E002010B40268047B11680223A340C0
:1004C800194209D00649406800240C7001684FF6AB
:1004D800FE742140016053605DF8044B704700BF13
:1004E8001A3C0020014B186824F0B4BD10200020ED
:1004F800F0B5836983B0054613B11A689B881385E4
:100508006869264F8389C3244FF47A734FF0060E27
:100518006E464FF6FF71013703E0013B9BB28B42F9
:100528001DD002899207F8D504734FF47A7302E05C
:10053800A3B28B4213D00289D20703F1FF34F7D557
:10054800027BD2B20EB132700136BEF1000F08D074
:100558000EF1FF3EFF24002FE3D03C78DBE725F0C7
:100568003DFAAB6913B11A689B8893619DF8050041
:100578009DF801609DF802109DF803409DF8042045
:100588009DF8063041EA062143EA002342EA0422A4
:10059800012029876A87AB8703B0F0BD28020308CA
:1005A800037C022B01D000207047F0B5836983B02B
:1005B80013B11A689B881385044640F2E9334069F1
:1005C80001E0002B59D00289013B12F0020F9BB2C7
:1005D800F7D0C323037340F2E93301E0002B4CD07A
:1005E8000289013B12F0010F9BB2F7D0037B6069CF
:1005F8004FF0060E83896E464FF47A734FF6FF71FB
:10060800FF2703E0013B9BB28B4233D00289950759
:10061800F8D507734FF47A7302E0ABB28B4229D056
:100628000289D20703F1FF35F7D5027BD2B20EB1AA
:1006380032700136BEF1010EE8D1A36913B11A6810
:100648009B8893619DF804009DF800609DF8011057
:100658009DF802509DF803209DF8053041EA0621D7
:1006680043EA002342EA0522012021876287A38703
:1006780003B0F0BD25F0B2F9DFE725F0AFF9B6E732
:10068800037A022B01D000207047F0B5036983B0CC
:1006980013B11A689B881385044640F2E933C06891
:1006A80001E0002B59D00289013B12F0020F9BB2E6
:1006B800F7D0BB23037340F2E93301E0002B4CD0A1
:1006C8000289013B12F0010F9BB2F7D0037BE0686F
:1006D8004FF0060E83896E464FF47A734FF6FF711A
:1006E800FF2703E0013B9BB28B4233D00289950779
:1006F800F8D507734FF47A7302E0ABB28B4229D076
:100708000289D20703F1FF35F7D5027BD2B20EB1C9
:1007180032700136BEF1010EE8D1236913B11A68AF
:100728009B8893619DF804009DF800609DF8011076
:100738009DF802509DF803209DF8053041EA0621F6
:1007480043EA002342EA05220120E18222836383EF
:1007580003B0F0BD25F042F9DFE725F03FF9B6E731
:100768002DE9F04F87B0019090F85500002840F02F
:100778007185019B1B7C022B00F0E085BB4CBC4DB6
:10078800DFF8F492BB48DFF8F4E24FF0640A4FF068
:10079800100C4FF47A76D9F80430C3F30803002B11
:1007A80040F05684EFF31183002B40F05184216808
:1007B800826800BF23689942F9D12F6806FB07F3C6
:1007C8009B1AB3FBF7F306FB013101270091D9F817
:1007D8000430C3F30803002B40F00084EFF31183C7
:1007E800002B40F0FB832368816800BF2268934296
:1007F800F9D1D5F800B006FB0BF2521AB2FBFBF2A6
:1008080006FB0323009A9B1AB3F57A7FDFD3BAF16C
:10081800010AC0D1019B1B7C022B01F03380DFF859
:1008280058929448DFF854E24FF0640A4FF0100CE5
:100838004FF47A76D9F80430C3F30803002B40F05C
:10084800EB83EFF31183002B40F0E6832168826885
:1008580000BF23689942F9D12F6806FB07F39B1A5A
:10086800B3FBF7F306FB013101270091D9F80430F7
:10087800C3F30803002B40F09483EFF31183002B9C
:1008880040F08F832368816800BF22689342F9D1C2
:10089800D5F800B006FB0BF2521AB2FBFBF206FBCE
:1008A8000323009A9B1AB3F57A7FDFD3BAF1010AC2
:1008B800C0D1019B1B7C022B00F09D87DFF8B8910B
:1008C8006C48DFF8B8E14FF0640A4FF0100C4FF4B1
:1008D8007A76D9F80430C3F30803002B40F0648417
:1008E800EFF31183002B40F05F842168826800BF1A
:1008F80023689942F9D12F6806FB07F39B1AB3FBCB
:10090800F7F306FB013101270091D9F80430C3F34E
:100918000803002B40F02883EFF31183002B40F0ED
:1009280023832368816800BF22689342F9D1D5F8F0
:1009380000B006FB0BF2521AB2FBFBF206FB0323D4
:10094800009A9B1AB3F57A7FDFD3BAF1010AC0D1B6
:10095800019B1B7C022B00F00487DFF81C914548A3
:10096800DFF818E14FF00F0A4FF0100C4FF47A76C9
:10097800D9F80430C3F30803002B40F0F883EFF3F1
:100988001183002B40F0F3832168826800BF23683D
:100998009942F9D12F6806FB07F39B1AB3FBF7F3CB
:1009A80006FB013101270091D9F80430C3F308038D
:1009B800002B40F0BC82EFF31183002B40F0B7828C
:1009C8002368816800BF22689342F9D1D5F800B046
:1009D80006FB0BF2521AB2FBFBF206FB0323009A4A
:1009E8009B1AB3F57A7FDFD3BAF1010AC0D1019916
:1009F80091F84F200B7C042A34BF18261A26022BA4
:100A080000F06786DFF870901A48DFF870E04FF062
:100A18000F0A4FF0100C4FF47A76D9F80430C3F36C
:100A28000803002B40F0F983EFF31183002B40F00B
:100A3800F4832168826800BF23689942F9D12F683E
:100A480006FB07F39B1AB3FBF7F306FB01310127FB
:100A58000091D9F80430C3F30803002B40F04A8210
:100A6800EFF31183002B40F0458209E0BC710020B0
:100A7800C071002010E000E000ED00E0B871002037
:100A88002368816800BF22689342F9D1D5F800B085
:100A980006FB0BF2521AB2FBFBF206FB0323009A89
:100AA8009B1AB3F57A7FD4D3BAF1010AB5D1019B69
:100AB8001B7C022B00F0C385DFF8DC92B448DFF81A
:100AC800D4E24FF00F0A4FF0100C4FF47A76D9F8B1
:100AD8000430C3F30803002B40F08383EFF3118342
:100AE800002B40F07E832168826800BF236899420A
:100AF800F9D12F6806FB07F39B1AB3FBF7F306FB44
:100B0800013101270091D9F80430C3F30803002B01
:100B180040F0D381EFF31183002B40F0CE8123689E
:100B2800816800BF22689342F9D1D5F800B006FB6E
:100B38000BF2521AB2FBFBF206FB0323009A9B1A34
:100B4800B3F57A7FDFD3BAF1010AC0D1019B1B7CD0
:100B5800022B00F02985DFF840928D48DFF834E257
:100B68004FF00F0A4FF0100C4FF47A76D9F8043092
:100B7800C3F30803002B40F0A482EFF31183002B8A
:100B880040F09F822168826800BF23689942F9D1AA
:100B98002F6806FB07F39B1AB3FBF7F306FB01313B
:100BA80001270091D9F80430C3F30803002B40F063
:100BB8006781EFF31183002B40F06281236881681D
:100BC80000BF22689342F9D1D5F800B006FB0BF2BA
:100BD800521AB2FBFBF206FB0323009A9B1AB3F5E9
:100BE8007A7FDFD3BAF1010AC0D1019B1B7C022BAB
:100BF80000F08184DFF8A0916548DFF898E14FF0B4
:100C0800640A4FF0100C4FF47A76D9F80430C3F325
:100C18000803002B40F03982EFF31183002B40F0DA
:100C280034822168826800BF23689942F9D12F680D
:100C380006FB07F39B1AB3FBF7F306FB0131012709
:100C48000091D9F80430C3F30803002B40F0FB806F
:100C5800EFF31183002B40F0F6802368816800BF12
:100C680022689342F9D1D5F800B006FB0BF2521A6C
:100C7800B2FBFBF206FB0323009A9B1AB3F57A7FBB
:100C8800DFD3BAF1010AC0D1019B1B7C022B00F013
:100C9800E883DFF804913E48DFF8F8E04FF00F0AE8
:100CA8004FF0100C4FF47A76D9F80430C3F30803E8
:100CB800002B40F04082EFF31183002B40F03B8281
:100CC8002168826800BF23689942F9D12F6806FB22
:100CD80007F39B1AB3FBF7F306FB013101270091D9
:100CE800D9F80430C3F30803002B40F08F80EFF3EA
:100CF8001183002B40F08A802368816800BF226836
:100D08009342F9D1D5F800B006FB0BF2521AB2FBA8
:100D1800FBF206FB0323009A9B1AB3F57A7FDFD315
:100D2800BAF1010AC0D1019B1B7C022B00F0508351
:100D3800DFF864801649174F4FF00F094FF0100E77
:100D48004FF47A70D8F80430C3F30803002B40F04E
:100D5800D481EFF31183002B40F0CF8122688E6895
:100D680000BF23689A42F9D1D5F800C000FB0CF304
:100D78009B1BB3FBFCF300FB023300930126D8F85E
:100D88000430C3F308032BBBEFF3118313BB05E057
:100D980010E000E0B871002000ED00E02368D1F811
:100DA80008A000BF22689342F8D1D5F800B000FB34
:100DB8000BFCACEB0A0CBCFBFBFC00FB03C3009A6E
:100DC8009B1AB3F57A7FDAD3B9F10109BAD107B022
:100DD800BDE8F08FEFF3118A8EF312888A680B68EA
:100DE800DB0344BF3E608A682368D7F800C05FFA17
:100DF8008AFA8AF31188D5F800A09C4400FB0AF30C
:100E08009B1AB3FBFAF300FB0C33D8E7EFF3118816
:100E18008CF3128881680368DB0344BFCEF8007046
:100E280081682368DEF800205FFA88F888F3118863
:100E3800D5F800801A4406FB08F35B1AB3FBF8F3F5
:100E480006FB023367E7EFF311888CF31288816899
:100E58000368DB0344BFCEF8007081682368DEF8BE
:100E680000205FFA88F888F31188D5F800801A44C2
:100E780006FB08F35B1AB3FBF8F306FB0233FBE649
:100E8800EFF311888CF3128881680368DB0344BF91
:100E9800CEF8007081682368DEF800205FFA88F8D1
:100EA80088F31188D5F800801A4406FB08F35B1A0A
:100EB800B3FBF8F306FB02338FE6EFF311888CF3EC
:100EC800128881680368DB0344BFCEF8007081682C
:100ED8002368DEF800205FFA88F888F31188D5F8CF
:100EE80000801A4406FB08F35B1AB3FBF8F306FB11
:100EF800023323E6EFF311888CF3128881680368C4
:100F0800DB0344BFCEF8007081682368DEF8002058
:100F18005FFA88F888F31188D5F800801A4406FB30
:100F280008F35B1AB3FBF8F306FB0233B7E5EFF3FC
:100F380011888CF3128881680368DB0344BFCEF8FC
:100F4800007081682368DEF800205FFA88F888F36B
:100F58001188D5F800801A4406FB08F35B1AB3FB26
:100F6800F8F306FB02333AE5EFF311888CF31288A5
:100F780081680368DB0344BFCEF80070816823688A
:100F8800DEF800205FFA88F888F31188D5F8008029
:100F98001A4406FB08F35B1AB3FBF8F306FB0233AB
:100FA800CEE4EFF311888CF3128881680368DB03C1
:100FB80044BFCEF8007081682368DEF800205FFA2D
:100FC80088F888F31188D5F800801A4406FB08F3DE
:100FD8005B1AB3FBF8F306FB023362E4EFF3118804
:100FE8008CF3128881680368DB0344BFCEF8007075
:100FF80081682368DEF800205FFA88F888F3118892
:10100800D5F800801A4406FB08F35B1AB3FBF8F323
:1010180006FB0233FFF7F6BBEFF311828CF312885D
:1010280087680368D90303D50123CEF800308768A1
:101038002368DEF80010D2B282F311882A681944B6
:1010480006FB02F3DB1BB3FBF2F306FB01310BE4F7
:10105800EFF311828CF3128887680368D90303D5EC
:101068000123CEF8003087682368DEF80010D2B27A
:1010780082F311882A68194406FB02F3DB1BB3FBD1
:10108800F2F306FB0131FFF7A0BBEFF311828CF3FB
:10109800128887680368D90303D50123CEF8003086
:1010A80087682368DEF80010D2B282F311882A68B4
:1010B800194406FB02F3DB1BB3FBF2F306FB013119
:1010C800BDE5EFF311828CF3128887680368D903B2
:1010D80003D50123CEF8003087682368DEF80010B6
:1010E800D2B282F311882A68194406FB02F3DB1B8B
:1010F800B3FBF2F306FB013152E5EFF311868EF3F1
:101108001288D1F808C00B68DA0303D501233B60C5
:10111800D1F808C023683A68F6B286F311882E68B9
:101128001A4400FB06F3A3EB0C03B3FBF6F300FB36
:101138000233009322E6EFF311828CF3128887685A
:101148000368D90303D50123CEF8003087682368E4
:10115800DEF80010D2B282F311882A68194406FB1F
:1011680002F3DB1BB3FBF2F306FB0131B6E5EFF349
:1011780011828CF3128887680368D90303D5012389
:10118800CEF8003087682368DEF80010D2B282F308
:1011980011882A68194406FB02F3DB1BB3FBF2F340
:1011A80006FB0131FFF7FEBBEFF311828CF31288C7
:1011B80087680368D90303D50123CEF80030876810
:1011C8002368DEF80010D2B282F311882A68194425
:1011D80006FB02F3DB1BB3FBF2F306FB0131FFF75F
:1011E80092BBEFF311828CF3128887680368D903E6
:1011F80003D50123CEF8003087682368DEF8001095
:10120800D2B282F311882A68194406FB02F3DB1B69
:10121800B3FBF2F306FB013173E4EFF311828CF3B5
:10122800128887680368D90303D50123CEF80030F4
:1012380087682368DEF80010D2B282F311882A6822
:10124800194406FB02F3DB1BB3FBF2F306FB013187
:10125800FFF7FDBB24F01EF90446002800F0928336
:10126800036885881A8A15407FF483AA03F13843F6
:101278009B0AA749C5712022C85CA27128F0AAFF61
:10128800A38805952068049304A92AF07DFBA38808
:101298000199A04ACA60B3FA83F2C2F11F02561C30
:1012A80039D0D1B201F0FC0303F1804303F5803358
:1012B80001F003019E68DFF870E288000F2787407D
:1012C80026EA0706019F21680C374EF822709E60B7
:1012D800D3F808E0904E914FC1F38721814041EA4D
:1012E8000E014FF00108996008FA02FEB118C7F81C
:1012F80000E0082304A804920F7A8DF815308DF8C1
:1013080016808DF8145029F0D3FA854AD35DF02B56
:1013180000F33D83A388B3FA83F3C3F11F03581C7A
:101328003FF427AA012202FA03F37E490A6813430D
:101338000B60019B1B7C022B7FF420AA019B9B69FD
:1013480013B11A689B881385019B586940F2E933E9
:1013580002E0002B00F0DD820289013B12F0020F4F
:101368009BB2F6D06B23037340F2E93302E0002B03
:1013780000F0CF820289013B12F0010F9BB2F6D038
:10138800037B019B586940F2E93302E0002B00F02F
:10139800BD820289013B12F0020F9BB2F6D0802376
:1013A800037340F2E93302E0002B00F0AF820289B8
:1013B800013B12F0010F9BB2F6D0037B019B9B69A6
:1013C800002B3FF4DBA91A689B889361FFF7D6B915
:1013D800019B9B6913B11A689B881385019B586907
:1013E80040F2E93302E0002B00F0C9820289013B98
:1013F80012F0020F9BB2F6D03823037340F2E933A0
:1014080002E0002B00F0BB820289013B12F0010FC1
:101418009BB2F6D0037B019B586940F2E93302E0A6
:10142800002B00F0A9820289013B12F0020F9BB247
:10143800F6D00123037340F2E93302E0002B00F0F9
:101448009B820289013B12F0010F9BB2F6D0037B0D
:10145800019B9B69002B3FF46BAC1A689B889361D6
:1014680066E4019B9B6913B11A689B881385019BED
:10147800586940F2E93302E0002B00F07A820289D1
:10148800013B12F0020F9BB2F6D03723037340F2F0
:10149800E93302E0002B00F06C820289013B12F074
:1014A800010F9BB2F6D0037B019B586940F2E933E8
:1014B80002E0002B00F05A820289013B12F0020F71
:1014C8009BB2F6D01023037340F2E93302E0002BFD
:1014D80000F04C820289013B12F0010F9BB2F6D05A
:1014E800037B019B9B69002B3FF4D3AB1A689B8855
:1014F8009361FFF7CEBB019A936992F8506013B1DC
:101508001A689B881385019B586940F2E93310E0FB
:10151800302703083D04000828020308140401408A
:10152800506300200004014010630020002B00F0ED
:101538001A820289013B12F0020F9BB2F6D01923DE
:10154800037340F2E93302E0002B00F00C820289B9
:10155800013B12F0010F9BB2F6D0037B019B586947
:1015680040F2E93302E0002B00F0FA810289013BE6
:1015780012F0020F9BB2F6D0067340F2E93302E094
:10158800002B00F0ED810289013B12F0010F9BB2A4
:10159800F6D0037B019B9B69002B3FF42BAB1A68A9
:1015A8009B889361FFF726BB019A936992F84E6076
:1015B80013B11A689B881385019B586940F2E93377
:1015C80002E0002B00F0C9810289013B12F0020FF2
:1015D8009BB2F6D01A23037340F2E93302E0002BE2
:1015E80000F0BB810289013B12F0010F9BB2F6D0DB
:1015F800037B019B586940F2E93302E0002B00F0BD
:10160800A9810289013B12F0020F9BB2F6D0067342
:1016180040F2E93302E0002B00F09C810289013B93
:1016280012F0010F9BB2F6D0037B019B9B69002B44
:101638003FF491AA1A689B889361FFF78CBA019BC3
:101648009B6913B11A689B881385019B586940F2FE
:10165800E93302E0002B00F07A810289013B12F0A5
:10166800020F9BB2F6D01C23037340F2E93302E069
:10167800002B00F06C810289013B12F0010F9BB234
:10168800F6D0037B019B586940F2E93302E0002B56
:1016980000F05A810289013B12F0020F9BB2F6D08A
:1016A8001823037340F2E93302E0002B00F04C8169
:1016B8000289013B12F0010F9BB2F6D0037B019B1C
:1016C8009B69002B3FF4F8A91A689B889361FFF780
:1016D800F3B98B6913B11A689B881385019B586904
:1016E80040F2E93302E0002B00F02B810289013B34
:1016F80012F0020F9BB2F6D01B23037340F2E933BA
:1017080002E0002B00F01D810289013B12F0010F5D
:101718009BB2F6D0037B019B586940F2E93302E0A3
:10172800002B00F00B810289013B12F0020F9BB2E3
:10173800F6D0067340F2E93302E0002B00F0FE8099
:101748000289013B12F0010F9BB2F6D0037B019B8B
:101758009B69002B3FF456A91A689B889361FFF791
:1017680051B9019B9B6913B11A689B881385019B2A
:10177800586940F2E93302E0002B00F0DC8002896E
:10178800013B12F0020F9BB2F6D06B23037340F2B9
:10179800E93302E0002B00F0CE800289013B12F011
:1017A800010F9BB2F6D0037B019B586940F2E933E5
:1017B80002E0002B00F0BC800289013B12F0020F0E
:1017C8009BB2F6D00123037340F2E93302E0002B09
:1017D80000F0AE800289013B12F0010F9BB2F6D0F7
:1017E800037B019B9B69002B3FF4B7A81A689B8871
:1017F8009361FFF7B2B8019B9B6913B11A689B8884
:101808001385019B586940F2E93302E0002B00F090
:101818008C800289013B12F0020F9BB2F6D06B2339
:10182800037340F2E93301E0002B7ED00289013BCB
:1018380012F0010F9BB2F7D0037B019B586940F26D
:10184800E93301E0002B6DD00289013B12F0020F51
:101858009BB2F7D00023037340F2E93301E0002B79
:1018680060D00289013B12F0010F9BB2F7D0037BD5
:10187800019B9B69002B3FF421A81A689B88936100
:10188800FFF71CB8019B9B6913B11A689B881385E5
:10189800019B586940F2E93301E0002B3FD00289EF
:1018A800013B12F0020F9BB2F7D06823037340F29A
:1018B800E93301E0002B32D00289013B12F0010F1D
:1018C8009BB2F7D0037B019B586940F2E93300E0F3
:1018D80013B30289013B12F0020F9BB2F8D0072321
:1018E800037340F2E93300E0B3B10289013B12F01F
:1018F800010F9BB2F8D0037B019B9B69002B3EF440
:101908008EAF1A689B889361FEF789BF24F066F84A
:1019180054E524F063F834E524F060F8ECE724F0AB
:101928005DF8D0E724F05AF8A2E724F057F884E7E6
:1019380024F054F855E724F051F835E724F04EF830
:1019480005E724F04BF8E6E624F048F8B7E624F07B
:1019580045F897E624F042F867E624F03FF848E6B1
:1019680024F03CF816E624F039F8F7E524F036F8C8
:10197800B7E524F033F897E524F030F868E524F06B
:101988002DF848E5019A0A4BD3600123CDE4F319F9
:10199800F0211B7E8DF80C3003A803238DF80E5020
:1019A8008DF80F80D1558DF80D3029F093FFB1E4F3
:1019B8003D0400082DE9F04F4269B24C1388DFF866
:1019C800D082B14E23F040031B041B0C13801388F4
:1019D8009BB223F0380343F03003138013889BB283
:1019E80083B043F040031380019009F043FFDFF810
:1019F800A4E2A649844610274FF47A750120DEF840
:101A08000430C3F30803002B40F01D81EFF311836A
:101A1800002B40F018812368D1F8089000BF226895
:101A28009342F8D1D8F800A005FB0AF2A2EB09020C
:101A3800B2FBFAF205FB03239C45E0D0019D284642
:101A4800FEF78EFEAB6913B11A689B881385019B5C
:101A5800586940F2E93302E0002B00F0388102892E
:101A6800013B12F0020F9BB2F6D06A23037340F2D7
:101A7800E93302E0002B00F02A810289013B12F0D1
:101A8800010F9BB2F6D0037B019B586940F2E93302
:101A980002E0002B00F01E810289013B12F0020FC8
:101AA8009BB2F6D01023037340F2E93302E0002B17
:101AB80000F010810289013B12F0010F9BB2F6D0B1
:101AC800037B019B9B6913B11A689B889361DFF8BC
:101AD800C4916E486C4F4FF0640A4FF0100E4FF4EB
:101AE8007A75D9F80430C3F30803002B40F0D4808A
:101AF800EFF31183002B40F0CF802168826800BF8C
:101B080023689942F9D1D8F8006005FB06F39B1ABF
:101B1800B3FBF6F305FB013101260091D9F8043037
:101B2800C3F30803002B56D1EFF31183002B52D1D6
:101B38002368816800BF22689342F9D1D8F800B0C1
:101B480005FB0BF2521AB2FBFBF205FB0323009ACA
:101B58009B1AB3F57A7FE1D3BAF1010AC1D1019B8F
:101B68004A4D5A69484F138823F040031B041B0C45
:101B78001380138823F038031B041B0C138013886D
:101B88009BB243F04003138009F074FEDFF804C1F0
:101B980081464FF0100E4FF47A760120DCF80430BD
:101BA800C3F30803002B31D1EFF3118373BB236810
:101BB800A96800BF22689342F9D1D8F800A006FBB3
:101BC8000AF2521AB2FBFAF206FB03239945E5D052
:101BD80003B0BDE8F08FEFF3118C8EF312888168A3
:101BE8000368DA0344BF3E60816823683A685FFA95
:101BF8008CFC8CF31188D8F800C01A4405FB0CF350
:101C08005B1AB3FBFCF305FB0233A0E7EFF311818A
:101C18008EF31288D5F808A02B68DB0344BF386020
:101C2800D5F808A023683A68C9B281F31188D8F8B2
:101C380000101A4406FB01F3A3EB0A03B3FBF1F30C
:101C480006FB0233C2E7EFF3118987F31288D1F854
:101C580008A00B68DB0344BF3060D1F808A02368F4
:101C680032685FFA89F989F31188D8F800901A4424
:101C780005FB09F3A3EB0A03B3FBF9F305FB0233F6
:101C8800DAE600BFBC710020B871002010E000E067
:101C9800C071002000ED00E0EFF311828EF312888E
:101CA80086680368D90302D501233B6086682368E8
:101CB8003968D2B282F31188D8F80020194405FB9C
:101CC80002F39B1BB3FBF2F305FB013124E723F07E
:101CD80085FED9E623F082FEF3E600BF10B490E853
:101CE8000600047B40690223A3404B6013685DF83B
:101CF800044B4FF6FE710B40136023F03BB9F8B567
:101D0800174D2B78A52B28D16B78BE2B25D1022215
:101D180029464FF6FF70FEF76BFB124FAC1C22886A
:101D28004AB1A618BE4218D2052A16D92146FEF78E
:101D38005FFB3446F3E721460222FEF759FB0222F5
:101D4800A118FEF755FB0634074B641B1C8041F6AF
:101D58000F53C31A58425841F8BD0020F8BD00BFC0
:101D680000F0030800000408EC2C00202DE9F04FD7
:101D7800DFF864914F4F8BB00326A7EB09071822B1
:101D8800002104A82EF0DDF94B4BCDF810900597F3
:101D98001A69120604D5494A5A6002F188325A6013
:101DA80001228DF824203422DA60454B454C1B88EB
:101DB800ADF800300222694604A823F0D1FE0222C1
:101DC80069464FF6FF70FEF713FBDFF810A1804657
:101DD8004FF0000B544536D30AAC002524F8245D97
:101DE8000222214604A823F0BBFE022221464046D7
:101DF800FEF7FEFA40BAC043ADF80800022202A975
:101E080004A823F0ADFE079860B106ABC0F1040248
:101E1800294618442EF095F9069904A823F046FEA1
:101E2800079508909DF82430089A23B122490B6938
:101E380043F080030B61013E2DD0002A9FD1FFF7AC
:101E48005EFF50B332E065888DF80DB0C5F30B0521
:101E5800AB1DADF808302388C3F30B02ADF80A2098
:101E68001B0B062202A904A88DF80C3023F078FE7B
:101E7800062202A94046FEF7BBFA616880462A4658
:101E880004A823F06DFE616840462A46FEF7B0FAC2
:101E9800143480469EE7002AD1D0052024F0BEFFE6
:101EA800094B0A4A1A600A4B0A4ADA600BB0BDE8C5
:101EB800F08F00BF0000040800200240230167459E
:101EC8004702030868560308FC9F0020EFBEADDEFA
:101ED80000ED00E00400FA0500F003088C5A03083E
:101EE8000378202B024600F10100F9D0092BF7D026
:101EF8002D2B2CD02B2B03BF5378B7EE000A0246AC
:101F0800B7EE000AA3F13001C8B209289FED467A5E
:101F180010D8F2EE046A07EE901AF8EEE77A12F893
:101F2800013FE7EE267AA3F13001C8B20928B0EEE6
:101F3800677AF0D92E2B4CD003F0DF03452B0BD05A
:101F4800F7EE007A67EE276A20EE260A7047537884
:101F5800BFEE000A0246D5E710B451782D2959D0B2
:101F68002B290ABF9178501C901C0024A1F1300342
:101F7800092B53D8002303EB830301EB430310F829
:101F8800011FA1F13002092AA3F13003F3D9B3F5F7
:101F98009A7F28BF4FF49A73072B42D9DFED236A43
:101FA8001A46F7EE007A083A072A67EEA67AFAD8B0
:101FB80003F007032BB1F2EE046A013B67EEA67A41
:101FC800FBD124B3C7EE276A5DF8044B20EE260A3E
:101FD80070475378A3F13001C8B2092802F1010211
:101FE800AAD8F2EE046AF0EE665A07EE901AF8EEF6
:101FF800E77A12F8013F87EEA66AA3F13001C8B26A
:10200800092866EEA56A37EE067AEED994E767EEF8
:10201800276AD9E7901C91780124A7E7F7EE007AA0
:10202800CFE7F7EE007AC5E70000000020BCBE4C01
:10203800B5EEC00ADFED317AF1EE10FACCBF30EE22
:10204800270A30EE670ADFED2E7A20EE270A30B530
:10205800FDEEC07A87B017EE904A054684EAE47030
:10206800002303A9A0EBE4700193009302931DF0F1
:1020780061FE002CACBF20232D2303A88DF800306F
:102088002BF0F4FF012803A924D002282DD003281F
:1020980005BF3023684668468DF801302EF059F8A0
:1020A80068462BF0E3FF0338C4B222466946284647
:1020B8002EF086F800232B5528462BF0D7FF2E222A
:1020C800431C2A540DEB0401E8182EF05FF828464B
:1020D80007B030BD302368468DF801308DF80230E6
:1020E8008DF803302EF035F8DAE7302368468DF89E
:1020F80001308DF802302EF02CF8D1E76F12033A38
:1021080000007A442DE9F041064615460846B6FB1C
:10211800F2F43CB905FB1464124B1B5D00F8013B5B
:10212800BDE8F081B4FBF2F767B90E4B05FB174722
:1021380005FB1464DA5D00F8012B1B5D00F8013B18
:10214800BDE8F081B7FBF2F8B8F1000F02D04046C5
:10215800FFF7D8FF05FB1878024B13F8082000F8A2
:10216800012BE3E7342803082DE9F04714461D4600
:10217800064600234FF47A72204629462CF020FCAC
:10218800DFF848814B4A4C4F88FB00310144C317A4
:1021980082FB002EC3EB611188FB012887FB002717
:1021A8008644464AC3EBEE2EC1EB011C82FB0E2986
:1021B800A0EB8C0C0744424A86F806C0C3EB2747BD
:1021C8004FEAEE7C08EB010ACCEBA90C82FB0782F4
:1021D8004FEAE1780CEB4C0CC8EB6A18AEEBCC0E6E
:1021E800C8EB0818DFF8E8C086F804E0A1EB88011E
:1021F80071718CFB0010F917C1EBE21240F2B55176
:1022080001FB1272C3EBE050B2F5896F4FEA800709
:102218003FDA40F2DA239A4243DCB2F5B77FB4BF23
:102228004FF0000C4FF0010C4FEA4C08254B08EB1F
:102238000C0103EBC1031FFA8CFE588F224908EBEF
:102248000C0301EBC30116310B2301E031F8020D39
:1022580082421BDA013BF9D11A4BC44403EBCC0C84
:102268000123BCF82400B37007F2B2770132121AC6
:10227800BE44F270A6F800E0204629464FF47A7270
:1022880000232CF09DFB3281BDE8F0870133DBB2DF
:10229800E9E74FF0030EF44640F296504FF0060877
:1022A800CCE74FF0020EF44640F229404FF0040804
:1022B800C4E700BFC5B3A29107452EC2ABAAAA2A9C
:1022C80073B06D16280203084C02030889888888B1
:1022D800792D0311104B2DE93048D3E9004554EA14
:1022E80005020BD10346012200201871587198711C
:1022F8009A70DA7018801881BDE83088074B1A6820
:1023080014EB020B45F1000C5A466346FFF72CFF0D
:102318000120BDE8308800BFD01F0020BC7100201C
:10232800F0B402888578164FC37804794179A2F20F
:10233800B27202F0030606EB4606013D05EB860580
:1023480007EB4505013BAE8C8579008940F2B5570E
:10235800920807FB0232931903EB430304EBC30310
:10236800C3EB031301EB8303C3EB031305EB8303F5
:1023780000214FF47A72C2FB0301F0BC704700BF22
:1023880028020308FAB170B48E18044603E0101A44
:1023980014D1B14214D014F8012BA2F14103192B26
:1023A80011F8013BA3F1410598BF2032192D03F123
:1023B8002000ECD9D01A01D1002BEAD170BC7047AB
:1023C800002070BC70471046704700BF4FF0FF32C6
:1023D800FFF7D8BFA0F16103192B98BF20387047C9
:1023E800A0F14103192B98BF20307047202805D051
:1023F800093804288CBF002001207047012070474D
:10240800613819288CBF00200120704741381928ED
:102418008CBF002001207047303809288CBF00206D
:1024280001207047A0F13003092B07D920F02000C4
:10243800413819288CBF00200120704701207047BF
:1024480030B402681146531C036011F8024B016056
:10245800D31C517803609378151D05601B0443EA6B
:102468000123D078234343EA006030BC704700BFA3
:102478000368591C1A46016012F8021B026058785A
:1024880041EA0020704700BF03685A1C02601878B0
:10249800704700BF38B50446006815462CF054FD57
:1024A80022682A44226038BD036810B40A0A5C1CFA
:1024B80004601A7003685A1C026019705DF8044BB6
:1024C800704700BF03685A1C026010B41970036893
:1024D8000A0A5C1C04601A7003680A0C5C1C04601D
:1024E8001A700368090E5A1C026019705DF8044BD3
:1024F800704700BF03685A1C026019700368090A14
:102508005A1C0260197070472DE9F047002488B002
:1025180080460F461E46A14605AD531C039311780D
:1025280039B3252933D1931CCDF8109003935078F3
:1025380030284ED04FF0000AA0F13003DBB2092B4F
:1025480042D96C2819D0642800F0938024D8252813
:102558001CD063D9582876D063281BD131784046DF
:10256800B847039A531C03931178043601340029A1
:10257800D7D1204608B0BDE8F087039B5A1C0392C8
:102588001B78642B7CD02AD8252B54D12521404692
:102598000134B847039AC0E7732833D044D9752863
:1025A8004FD106F1040E30682B4600220A217646E8
:1025B800FDF714FE049A0095534639464046FDF748
:1025C8004BFE039A0444A8E704AA03A91DF0F8FAED
:1025D800B7E7D31C039390784FF0010AACE7732B4D
:1025E80010D05BD9752B3AD0782B96D1A3F158022D
:1025F800B2FA82F2306852092B4610210436FDF7F0
:10260800EDFDD7E73368049A009339460023404626
:10261800FDF722FE04360444039A7EE70028B9D168
:10262800204608B0BDE8F0876E28B3D1039A336816
:1026380004361C6071E72AD9582BD7D0632B8DD06C
:102648006BE77828A6D1A0F15802B2FA82F2306876
:1026580052092B461021FDF7C1FD0436AAE706F101
:10266800040E30682B4600220A217646FDF7B6FD97
:10267800A0E7331D306829461E46FDF781FD99E71E
:10268800331D306829461E46FDF77AFD92E7002B78
:102698007FF443AF204608B0BDE8F0876E2BC6D064
:1026A8003BE700BF0EB400B584B005AB019053F80A
:1026B800042B0649039301A8FFF726FF019B00227C
:1026C8001A7004B05DF804EB03B0704755020008B7
:1026D8000FB430B583B006AB0A490B4853F8042B46
:1026E800096800680193FFF70FFF084C054620684A
:1026F80022F0A0FC0028FAD0284603B0BDE83040FC
:1027080004B07047582C00205C2C002010200020BA
:10271800DFED2B7AB4EEE70AF1EE10FA4ADDDFEDD1
:10272800296A9FED297A01E0B0EE670AB4EEC70A7C
:10273800F1EE10FA70EE667AF6DC9FED247AF4EE8C
:10274800C77AF1EE10FA38D5DFED1E6A9FED207AD0
:1027580001E0F0EE407AF4EEC77AF1EE10FA37EEC7
:10276800A60AF6D4DFED1B7AB4EEE70AF1EE10FA0A
:1027780014DDDFED137A37EEC00A60EE006A9FEDD4
:10278800166A9FED167ADFED167AA6EE867A20EEA7
:10279800266AE6EE877AA6EE270A7047DFED117AF9
:1027A800B4EEE70AF1EE10FA44BFDFED087A37EE2F
:1027B800C00AE2E7F0EE407ABFE7B0EE670AD1E779
:1027C800DB0F4940DB0FC940E4CB1641DB0F49C0A2
:1027D800E4CB16C1DB0FC93F92E741B99730083CFB
:1027E80015A82ABEDB0FC9BF09B909E0194690FB35
:1027F800F1F301FB13030846002BF7D10846704795
:102808000146FBE7F0EEC07AB0EEE07AB4EEE77A84
:10281800F1EE10FAB4BFB0EE676AB0EE476AB5EEF3
:10282800406AF1EE10FA46D0B4EEE77AF1EE10FA0B
:102838008CBFF0EE675AF0EE475AC5EE866A9FEDF8
:102848001F3A9FED1F6A9FED1F4A9FED1F5ADFED4C
:102858001F3ADFED1F4ADFED1F5AA6EEC36AE6EE08
:10286800A34AA6EE864AB7EE006AA6EE845AA6EEFA
:10287800A46AE6EE855AC5EE866AB4EEE77AF1EE0A
:1028880010FA48BFDFED147AF5EEC00A48BF77EEBC
:10289800E66AF1EE10FA48BFDFED107AB5EEC00A2D
:1028A80048BF77EEE66AF1EE10FA48BFF1EE666AC5
:1028B800B0EE660A7047DFED076ADEE739094E3D7C
:1028C800E3B59E3E88FA163E45FE7F3F99FB243FBE
:1028D80069A2163EA7DFA834DB0FC93FDB0F4940CA
:1028E800DFED317A30EE277AFDEEC76A16EE903AC0
:1028F8002033402B02D99FED2D0A7047B4EEE70A2A
:10290800F1EE10FA4DDD9FED2A6ADFED2A6A01E04B
:10291800B0EE677AB4EEE67AF1EE10FA77EE467A20
:10292800F6DC9FED257AF4EEC77AF1EE10FA35D58C
:10293800DFED1F6A9FED217A01E0F0EE407AF4EEB8
:10294800C77AF1EE10FA37EEA60AF6D4DFED167A5A
:10295800B4EEE70AF1EE10FA1BDCDFED197AB4EEFB
:10296800E70AF1EE10FA44BFDFED137A37EEC00A3A
:1029780060EE006A9FED136A9FED137ADFED137A1C
:10298800A6EE867A20EE266AE6EE877AA6EE270A73
:102998007047DFED0F7A37EEC00AE9E7B0EE670A55
:1029A800D4E7F0EE477ABCE7DB0FC93F0000000030
:1029B800DB0FC940E4CB1641DB0F49C0E4CB16C19D
:1029C800DB0FC9BF92E741B99730083C15A82ABE6A
:1029D800DB0F494007EE901AF8EE677A9FED837A8D
:1029E80027EE800A20EE070AFDEEC07A17EE903A2D
:1029F8002033402B00F28C80DFED7D7AB4EEE70ABD
:102A0800F1EE10FA40F3E880B0EE407A9FED796A73
:102A1800DFED796A01E0B0EE677AB4EEE67AF1EEBE
:102A280010FA77EE467AF6DC9FED747AF4EEC77A00
:102A3800F1EE10FA40F1CD809FED6E6ADFED706A1D
:102A480001E0F0EE477AF4EEE67AF1EE10FA37EEAE
:102A5800867AF6D4DFED6B7AB4EEE77AF1EE10FA07
:102A680051DCDFED697AB4EEE77AF1EE10FA44BF93
:102A7800DFED627A37EEC77A27EE076ADFED635A31
:102A8800DFED637ADFED636A9FED635AE6EE257A40
:102A980067EE065AE6EE276AF7EE007AA5EEA67A02
:102AA800F0EE675AE7EE055AE7EE457A87EEA55A43
:102AB800DFED547A30EE277AFDEEC76A16EE903ACB
:102AC8002033402B29D99FED557AF6EE006AB7EEF0
:102AD800006AF7EE004AC4EEA57A002383614361D9
:102AE8000362C36180ED045A67EEA66A27EE866A20
:102AF80027EE877AC0ED006AC0ED026A80ED016AB0
:102B080080ED037A7047DFED3A7A37EEC77AB3E79C
:102B1800B7EE005AF0EE455ACAE7B4EEE70AF1EE0E
:102B280010FA5FDD9FED336ADFED336A01E0B0EE46
:102B3800677AB4EEE67AF1EE10FA77EE467AF6DCCA
:102B48009FED2E7AF4EEC77AF1EE10FA47D59FED95
:102B5800296ADFED2B6A01E0F0EE477AF4EEE67AB7
:102B6800F1EE10FA37EE867AF6D4DFED267AB4EE77
:102B7800E77AF1EE10FA27DCDFED237AB4EEE77A94
:102B8800F1EE10FA44BFDFED1D7A37EEC77A27EE73
:102B9800076ADFED1E4ADFED1E6ADFED1E7AE6EEFC
:102BA800246A67EE064AE6EE267AB7EE006AA4EED5
:102BB800A77AF6EE006A36EE476AF8EE007A27EE54
:102BC800277A66EE266A84E7DFED097A37EEC77A58
:102BD800DDE7B0EE677A3DE7F0EE407A24E7B0EE45
:102BE800677AC2E7F0EE477AAAE700BF27D4D23661
:102BF800DB0F4940DB0FC940E4CB1641DB0F49C06E
:102C0800E4CB16C1DB0FC93FDB0FC9BF92E741B95F
:102C18009730083C15A82ABEF304353F0000008011
:102C280070B406688E4217D90139751E002311F851
:102C3800014F0822634013F0800F4FEA430318BF87
:102C480083F0D503013ADBB2F5D18D42EFD1721C86
:102C58000260337070BC70470023F8E710B44C0969
:102C6800012250F8243001F01F0102FA01F10B4350
:102C780040F824305DF8044B704700BF4B0901F061
:102C88001F0150F82320012303FA01F1114214BF58
:102C980018460020704700BFF0B55B4B5B4A97B001
:102CA8001968914200AF00F0A3805949594A00239E
:102CB8004FF47000C1F888003B607B60136843F4F0
:102CC8008033136003E03B68B3F5A04F09D0136865
:102CD80003F400337B603B6801333B607B68002B67
:102CE800F1D04C4B1B6813F4003318BF01237B60F1
:102CF8007B68012B52D0464C464B474AE260474A14
:102D0800596A11605A6A42F080725A625A6942F4EA
:102D1800FC025A610025032207F10801012341F64C
:102D2800FF764FF09040FD60BE603A73BB7328F0A9
:102D38002BFE4FF6FF7307F108013948BB6028F0F6
:102D480023FE07F108013748374E28F01DFE07F12A
:102D58000801364828F018FE07F10801344828F021
:102D680013FE07F10801334828F00EFE07F10800AA
:102D780028F0BEFEBB683049304AA1FB0313304936
:102D88009B0CF0204FF0070E5C370B60566084F800
:102D980023009560C2F800E0BD46F0BD294A1D4BEE
:102DA800122111605A685A605A685A605A6842F487
:102DB80080625A605A6822F47C125A605A6842F457
:102DC800E8125A601A6842F080721A601A68920112
:102DD800FCD559680F4A21F003015960596841F040
:102DE80002015960536803F00C03082BFAD182E7FB
:102DF80000221A6062B6144B1B6883F30888134BD1
:102E08001B689847FEE700BFFC9F0020EFBEADDEC1
:102E180000ED00E0001002400005FA05704F0020A8
:102E280000040048000800483F190100000C004851
:102E3800001000480014004883DE1B4310E000E047
:102E4800C07100200020024000D8FF1F04D8FF1FD7
:102E580070B50F4C0F4DC0EBC00004EB80046869DF
:102E680026693043686182B09209667BA1600025BB
:102E7800012101A863618DF804608DF805208DF8A3
:102E880006508DF8071028F025FD02B070BD00BF70
:102E9800FC19002000100240074BC0EBC00030B402
:102EA80003EB8000054C056963692B436361017678
:102EB800427630BC704700BFFC1900200010024069
:102EC8002DE9F04F5E4C54F8204083B0002C71D0AF
:102ED800A66D984691465B4B72682265A160236097
:102EE80004F15E014FF4807304F5AF726161A26171
:102EF800E36023610746307E27F06CF9F068A8B1DB
:102F0800514B00215A68904203F11C0300F0928053
:102F180001310C29F6D100207A1CD2B20C21FFF71E
:102F2800BBFF236DF26862632433E364B068D8B1F1
:102F3800454B00215A68904203F11C0378D00131B7
:102F48000C29F7D100257A1CD2B20B212846FFF7AD
:102F5800A3FF2346F27E3D492846FFF779FF236DFC
:102F6800B268A2632833A36494F85D0022F092FA51
:102F7800054694F85C0022F08DFA18F0080F824696
:102F880096F819B01AD0CDB118F0110F4FF00B0305
:102F980007F1010714BF4E213E21EF715A46AB716C
:102FA800284622F03BFB18F0010F45D0636B5BB35A
:102FB800A36B4BB3204603B0BDE8F08F18F0010FA8
:102FC8000CBF4FF02E084FF04E0819F0020F09D031
:102FD80045B10B227B1CAA71EB7128465A46414623
:102FE80022F01CFB19F0010FE0D0BAF1000FDDD080
:102FF80001370C238AF807705A4641468AF806308A
:10300800504622F00BFBD1E7337FB27E8DF80420C7
:103018009B090021012201A88DF805308DF80610C2
:103028008DF8072028F056FC204603B0BDE8F08F45
:10303800CDB288E7C8B26FE7284622F089FBB5E72A
:10304800642C0020AC020308FC190020E51C0008D1
:1030580000B97047F0B595B0054627F0B7FB6E4E3E
:10306800C368026832600446002B00F0C38028461B
:1030780022F010FA694B186018B1292200238271D6
:10308800C371227A664D2E2122F0C8FA306808F002
:1030980081FA27F09FF83068624A038823F0010319
:1030A8001B041B0C038014A91E232B8001270F234C
:1030B8000025138021F84C7D2D230293ADF80C5088
:1030C800ADF80650ADF80E5027F02EFBE379ADF8B9
:1030D800145060229907ADF816500695ADF81C50AB
:1030E800ADF81E50ADF82050ADF82250049200F112
:1030F800838013F0010F14BF022200224FF4807363
:10310800ADF81470ADF81C20ADF82030002304AAE7
:1031180061793068069307F0A3FE3068617927F07B
:10312800E3FA3068436C43F40043436403889BB27A
:1031380043F080030380E3799B0768D56179026ACD
:1031480004238B4022EA03020262026A13430362E9
:103158003268354F13889BB243F001031380207CFB
:1031680000222921FFF798FE3049207C00236022A5
:10317800FFF76EFEE068386028F018FB38680368CF
:103188004FF6FE721340036028F010FB09A828F0E0
:10319800DFFA33686279264938680A913433134470
:1031A800099380221023002509A940F22A3E0E9295
:1031B8000B934FF400724FF400530D95109513952F
:1031C80011950F921293ADF830E028F0CFFA62799A
:1031D80033680C2A98BF1749D86898BF31F812503D
:1031E8003A6815490543DD601368012043F002037E
:1031F8001360087015B0F0BD13F0010F14BF08225A
:103208002A460423ADF81E20ADF816307EE70122C9
:10321800617928F0DBF99BE76C410020581D0020FC
:10322800624100206041002068410020BD04000880
:103238006C3C0020A81E0308644100200348D0F815
:103248003C3113B100F59A7018477047FC190020FB
:103258000348D0F8203113B100F58C701847704737
:10326800FC1900200348D0F804310BB1FC30184792
:10327800704700BFFC1900200348D0F8E8300BB1B4
:10328800E0301847704700BFFC1900200348D0F809
:10329800CC300BB1C4301847704700BFFC19002070
:1032A8000348D0F8B0300BB1A8301847704700BFBA
:1032B800FC1900200348D0F894300BB18C30184723
:1032C800704700BFFC1900200248836F0BB17030B3
:1032D80018477047FC1900200248C36D0BB15430E1
:1032E80018477047FC1900200248036C0BB13830AE
:1032F80018477047FC1900200248436A0BB11C307C
:1033080018477047FC1900200248836803B1184722
:10331800704700BFFC1900201749184B184A194874
:1033280010B4D1F8884044F47004C1F888401C688F
:1033380044F001041C605C6822405A601A6822F05C
:10334800847222F480321A601A6822F480221A6089
:103358005A6822F4FE025A60DA6A22F00F02DA6230
:103368001A6B002410404FF0006218639C608A605A
:103378005DF8044B704700BF00ED00E0001002400C
:103388000CC07FF8CCFC00FF2DE9F04F2DED0E8B23
:10339800DFF8A8A39BB0DAF80430079050469847A6
:1033A800002875D0BAF8A85000228AF85120002DBC
:1033B80041F03884DAF84830BAF93C60BAF9380094
:1033C800DAF82050BAF93A10DAF82440DFF87093A6
:1033D800F71A87EAE772A2EBE772B2F5804FDAF8DC
:1033E8002820DCBFCAF848603346401B091B9B1ADB
:1033F800CAF82C00CAF83010B3489AF85210CAF824
:10340800343015F05DF8D9F80030980041F1FC84AB
:10341800DAED0C5ADFF82CB3DAED0B7AAB4A9BEDF8
:10342800406ADBED416A9BED427ADBF80C311268A9
:10343800B8EEE58ADAED0D5AF8EEE77AF8EEE58AA5
:10344800013377EE867A38EE268A78EE878A9342B9
:10345800CBED407A8BED418ACBED428ACBF80C312B
:1034680002F0CA829A4B05931E78142E03F02A8321
:103478000023DBF814410693062C01F27481DFE87F
:1034880014F0BC15F616F8148F16E108071758152E
:103498008F4BDFF8B0B21C780593072C01F0B6818A
:1034A8009BF82131099353B15F1E8BF82171012CD0
:1034B80001F086841BB0BDEC0E8BBDE8F08F854B08
:1034C8005B79002B01F01682834B1B78013BDBB242
:1034D800072C8BF8213102F0748300230A937F4A6A
:1034E800DBF82C31D2ED006A7D4A9FED7E6AD2F876
:1034F80000907D4A0892079ADBED4AAA9BED499A0B
:10350800DFF844829FED79AADFED79BA9FED79DA89
:103518009FED79BADFED79CA9FED79CA794F7A4E76
:10352800CBF82C21D31A07EE903AF8EE677AB7EE6B
:10353800007AC6EE279A0024744B0693254677EE48
:103548006A8A68EEA68AF4EEC78AF1EE10FA88BF96
:10355800F0EE478A6E4B98ED008A2344D3ED007A4B
:10356800F5EE407AF1EE10FA17D06A4B234493ED4A
:10357800007A78EE476AB0EEE66AF4EEC67AF1EEC3
:1035880010FA08D5F5EEC06AF1EE10FACCBF37EEA6
:10359800878A37EE678A83ED008A5F4B1B889A0714
:1035A80039D0022D37D099F82E105C4A07EE901AC0
:1035B800224492ED007A4A42F8EEE76A07EE902A32
:1035C80026EE877AF8EEE77AB4EEE77AF1EE10FAAB
:1035D8000AD407EE901AF8EE677AF4EEC77AF1EE9D
:1035E80010FA88BFF0EE477A4D4A4E4902EB450281
:1035F80031F91500B2F90C20801A07EE100AB8EE5E
:10360800C77AD807E7EE4A7A41F10A81464B93ED2B
:10361800008A27EE888A089B9BF86021234493ED53
:1036280001EA78EE4EDA002A00F0D0803F4ADBF853
:10363800643107991268CB1A934240F3C78099F80E
:103648004820022A02F01583022D05F00F81384A1E
:10365800126891077AD4374A86ED00DA12689A42DE
:10366800C0F2AE80F7EE007AF4EEE7AAF1EE10FAB7
:1036780040F1AC800899304BD1ED017A93ED007A96
:10368800F0EEE77AF4EEC77AF1EE10FA40F19E8098
:10369800D1ED027AF0EEE77AB4EEE77AF1EE10FABD
:1036A80040F39480D1ED037AF0EEE77AB4EEE77A4E
:1036B800F1EE10FA40F38A801D4B1B689A077FD5FC
:1036C8001849174A63E000BFF86800208C300020D2
:1036D800CC610020446B0020DC2F00206C600020AF
:1036E8000849002000247449586B0020CDCCCC3DFB
:1036F800AE47813F000000000000C842000034438C
:10370800610BB63B24300020183000200C3000201C
:1037180060600020C81E002004490020D41E00203C
:10372800E82F0020B4480020486000207460002082
:10373800B0480020706000207C600020CC68002029
:10374800686B00208C1D0020BC1E0020D74AD84979
:10375800DFF8CCE331F915C09EED008ADFF8C4E349
:1037680086ED00DA02EB450028EE0A8AB0F90C0073
:10377800A0EB0C0007EE900AF8EEE77ADEF80000FE
:1037880027EE888A984278EE4EDABFF66BAFB2F928
:103798000C30B1F900E0C748AEEB030E00688EEAC2
:1037A800EE73A3EBEE73834210DAB1F90230B2F98B
:1037B8000E209A1A82EAE273A3EBE273984205DDBF
:1037C800002318468BF8603108F0B2F9BA4B23444D
:1037D80093ED000A069B29EE000A022D20EE2D0A21
:1037E800A3EC010A069304F08087B44BD6ED006A77
:1037F80093ED007AB24BD3ED007AB24B93ED006AA9
:10380800B14B67EE277A234427EEA87AD3ED007AE6
:1038180067EE277AF0EE665AEDEEA75AB1EE467AD1
:10382800B4EEE57AF1EE10FA08DCB4EEE56AF1EEF2
:1038380010FA8CBFB0EE657AB0EE467A9BED4A6A14
:10384800F7EE007AB4EEE76AF1EE10FAACBF0123A6
:10385800002343B1F0EEE66AF0EEC77AF4EEE67ABA
:10386800F1EE10FA01D586ED007A022D04F02C87CE
:10387800964A974B52F825001B68B0EE4E0A9847B7
:10388800944A954B52F825001B68984799F83730A9
:1038980023B1924B1B88002B01F0BC80B0EE4D8AFF
:1038A8008F4B38EE400A234493ED008A83ED000ADB
:1038B80099F8483030EE480A20EE298A53B3894BEC
:1038C8001B78DB0740F1B186F7EE007AF4EEE7AA41
:1038D800F1EE10FA9BF86031C1F20786002B01F077
:1038E8004981DBF86431079AD31A7F4A12689A42F1
:1038F80010DD7E4BD3ED007AF0EEEDDAF4EEE7DA88
:10390800F1EE10FA42F1BE81002318468BF86031BF
:1039180008F00EF9764B9BF87021234493ED000ACA
:1039280029EE000A20EE088A87ED008A32B9069B44
:1039380086ED00DA03ED01DA87ED00DA0135032DB3
:1039480008F1040807F1040706F1040604F1040469
:103958007FF400AE059B1B78072B01F0DB85012B5C
:1039680002F0348100230B939BF87831002B41F04F
:103978003482604BDFF8B0911C68D9F8003094F8B5
:103988002C50DE0401F172805B4B06931A465B4BA8
:10399800528B93ED006A5A4B5A4ED3ED005AD6ED2E
:1039A800036A594B8BED626A07EE102A574A93ED6A
:1039B800005AD2ED007AD2ED013AD2ED024A8BEDEF
:1039C800606AB8EEC77A35EEC64A012336EEC77A82
:1039D8008BED5F4ACBED635A8BF89031C7EE055AF1
:1039E800238D5A4206EE102A494ADFED4A6A92EDC3
:1039F800005A494A92ED004AB7EE007AF4EEC75AE7
:103A080035EE045AF1EE10FA88BFF0EE475A35EE5B
:103A1800275AB8EEC66AF4EEE65AF1EE10FA07EE47
:103A2800903AB4EEC65AB8BFF0EE665AF1EE10FA04
:103A3800CBED665AB8EE677A01F14F84B4EEC75AF7
:103A4800F1EE10FA88BFB0EE475A314BDFED336A1A
:103A5800D3ED017A304B93ED014A77EE847A25EE67
:103A6800265A77EEA37AB4EEE76AF1EE10FA08DC8C
:103A7800B4EEE77AF1EE10FA8CBFB0EE676AB0EEFA
:103A8800476A234A638DD2ED027A9FED247A5A421F
:103A980004EE102A74EEA77AB8EEC44A26EE076A36
:103AA800F4EEC47AF1EE10FA4BD43FE0E82F002090
:103AB800B4480020786000201C600020585F002077
:103AC800000000209060002028600020605F002037
:103AD8005C5F0020B45F0020B05F00200449002034
:103AE800F41E0020186F0020746000208060002001
:103AF800346000200849002024710020C46F002091
:103B0800B42F0020D0620020286100201830002047
:103B18000C30002000000000243000206F12833A8F
:103B28004860002070600020686B002007EE103AA3
:103B3800B8EE474AB4EEE74AF1EE10FA88BFB0EEA5
:103B4800674AEB4BDFEDEB7A5B7824EE274A0BB93B
:103B5800B1EE444A002D41F01387B7EE003AE64B28
:103B680008931A78002A02F0BC87E44BDFEDE47A68
:103B7800D3ED024AD3ED016A93ED037A66EE244A47
:103B8800E5EE264AE4EE074A63EE244AF4EEE74AF5
:103B9800F1EE10FAB4BFF0EE673AF0EE643A98BF6F
:103BA800F0EE647A012ACDED124A02F0C38793ED54
:103BB800067AD3ED052AD3ED076A26EE077AA5EE35
:103BC800227AA4EE267A23EE077AB4EEE77AF1EEAB
:103BD80010FAB4EEE37A8CBFF0EE676AF0EE476A4B
:103BE800F1EE10FA88BFF0EE676AB4BFF0EE637AC0
:103BF800F0EE477A022A8DED137A00F0DE8093ED1D
:103C08000A7AD3ED092AD3ED0B3A26EE077AA5EE08
:103C1800227AA4EE237A23EE077AB4EEE67AF1EE5E
:103C280010FAB4EEE77A8CBFF0EE663AF0EE473A57
:103C3800F1EE10FA98BFF0EE636AA8BFF0EE477A8B
:103C4800032A8DED147A00F0B88093ED0E7AD3ED47
:103C58000D2AD3ED0F3A26EE077AA5EE227AA4EEC6
:103C6800237A23EE077AB4EEE67AF1EE10FAB4EE90
:103C7800E77A8CBFF0EE663AF0EE473AF1EE10FACA
:103C880098BFF0EE636AA8BFF0EE477A042A8DED7C
:103C9800157A00F09280D3ED123AD3ED112A93ED04
:103CA800137A66EE233AE5EE223AE4EE073A63EE3B
:103CB800233AF4EEE63AF1EE10FAF4EEE73A8CBF66
:103CC800B0EE667AB0EE637AF1EE10FA98BFF0EED5
:103CD800476AA8BFF0EE637A052ACDED163A6CD094
:103CE800D3ED163AD3ED152A93ED177A66EE233AFB
:103CF800E5EE223AE4EE073A63EE233AF4EEE63ACA
:103D0800F1EE10FAF4EEE73A8CBFB0EE667AB0EE58
:103D1800637AF1EE10FA98BFF0EE476AA8BFF0EEAA
:103D2800637A062ACDED173A47D0D3ED1A3AD3ED88
:103D3800192A93ED1B7A66EE233AE5EE223AE4EE71
:103D4800073A63EE233AF4EEE63AF1EE10FAF4EEAF
:103D5800E73A8CBFB0EE667AB0EE637AF1EE10FA0D
:103D680098BFF0EE476AA8BFF0EE637A072ACDED58
:103D7800183A22D093ED1E7AD3ED1D2AD3ED1F3ABF
:103D880026EE077AA5EE227AA3EE847A27EE037A46
:103D9800B4EEE67AF1EE10FAB4EEE77A8CBFB0EE44
:103DA800666AB0EE476AF1EE10FA8DED197A98BF9F
:103DB800F0EE466AA8BFF0EE477A77EEE67AF7EEBD
:103DC800006AF4EEE67AF1EE10FACBED4A7A44F3A3
:103DD800118286EEA77A022ADDED137A67EE244A6D
:103DE80067EE877ACDED124ACDED137A2DD0DDED51
:103DF800147A67EE877A032ACDED147A25D0DDEDA3
:103E0800157A67EE877A042ACDED157A1DD0DDED97
:103E1800167A67EE877A052ACDED167A15D0DDED8C
:103E2800177A67EE877A062ACDED177A0DD0DDED81
:103E3800187A67EE877A072ACDED187A05D0DDED76
:103E4800197A27EE877A8DED197A2E4B1B6813F0B5
:103E5800805C01F0FF82F6EE005ACBED665A002A2C
:103E680002F06286284D294C9BED636A284B9BF92A
:103E78009011284E28489BED625AD5ED004AB4F9B6
:103E88000650069C0078648B96F800E00A94BDEE14
:103E9800C66A07EE101AD978D9F80030DBED5F6AE8
:103EA800DBED607A16EE106ABDEEC56A03F0100409
:103EB80003F4805803F480030C9300F00107B8EE74
:103EC800C77A16EE103A0D48002940F0C9879DEDD3
:103ED800125A90ED006A002C41F0268425EE866A7D
:103EE8000E49A5EE076AB0EE675AA6EE265A17E005
:103EF8007C3000206F12833AAD610020986000206A
:103F0800000000001C710020946000203C3C002050
:103F1800F43B0020F04B0020186F002040300020B8
:103F2800BDEEC56A16EE105A16EE104AB542A8BF85
:103F38003446AB42C8BF1C4606EE104AB8EEC66A05
:103F4800012A81ED006A00F0DC8090ED046A9DEDA5
:103F5800135A25EE866AA5EE076AB0EE675AA6EEF2
:103F6800265ABDEEC56A16EE105A16EE104AB5422C
:103F7800A8BF3446AB42C8BF1C4606EE104AB8EE8E
:103F8800C66A022A81ED016A00F0BB8090ED086ADA
:103F98009DED145A25EE866AA5EE076AB0EE675ABB
:103FA800A6EE265ABDEEC56A16EE105A16EE104A4F
:103FB800B542A8BF3446AB42C8BF1C4606EE104AFD
:103FC800B8EEC66A032A81ED026A00F09A8090ED85
:103FD8000C6A9DED155A25EE866AA5EE076AB0EEC5
:103FE800675AA6EE265ABDEEC56A16EE105A16EEA8
:103FF800104AB542A8BF3446AB42C8BF1C4606EEBD
:10400800104AB8EEC66A042A81ED036A79D090EDA9
:10401800106A9DED165A25EE866AA5EE076AB0EE7F
:10402800675AA6EE265ABDEEC56A16EE105A16EE67
:10403800104AB542A8BF3446AB42C8BF1C4606EE7C
:10404800104AB8EEC66A052A81ED046A59D090ED87
:10405800146A9DED175A25EE866AA5EE076AB0EE3A
:10406800675AA6EE265ABDEEC56A16EE105A16EE27
:10407800104AB542A8BF3446AB42C8BF1C4606EE3C
:10408800104AB8EEC66A062A81ED056A39D090ED65
:10409800186A9DED185A25EE866AA5EE076AB0EEF5
:1040A800675AA6EE265ABDEEC56A16EE105A16EEE7
:1040B800104AB542A8BF3446AB42C8BF1C4606EEFC
:1040C800104AB8EEC66A072A81ED066A19D090ED43
:1040D8001C6A9DED195A65EE865AE7EE055AE6EE1A
:1040E800A57AFDEEE77A17EE900A8642A8BF064643
:1040F8008342D8BF334607EE903AF8EEE77AC1ED2F
:10410800077A002F00F0B887CD4B1B68002B40F0D2
:10411800C087CC4B1B788BB1089F387858B1CA4DF3
:10412800CA4E0024E0B23368B5EC010A98473878E3
:1041380001348442F6DBC64B1B689847059B1B7805
:10414800072B01F0D7810025D9F800305F0501F170
:104158002381C04B1B78BBB1BF4A069BB2F906202E
:104168005B8B9A4210DCBD4B1B78012B01F040851C
:10417800192B01F03D850E2B06D0082B04D0B84E24
:104188000023B360CBF838319BF8C64124B1B54B56
:104198001B889E0741F0FF849BF8CC31002B41F02F
:1041A800A080069A947F002C00F00186022C01F072
:1041B8001884032C41F01C8492F82020C2EB421191
:1041C80002EB8102D20092B20699CF7F0237FFB28A
:1041D800002B00F01E86002A00F01B86A2490C68FE
:1041E800B2FBF4F214B2ABF8FC41002F03F0B88430
:1041F80007EE904AF8EEE77AF7EE006A86EEA77ABD
:10420800974E012FDBED846AD6ED007A77EEE67AD9
:1042180067EE877ACBED807A21D0D6ED017ADBED97
:10422800856A77EEE67A022F67EE877ACBED817A98
:1042380015D0D6ED027ADBED866A77EEE67A032FA3
:1042480067EE877ACBED827A09D0D6ED037ADBED7B
:10425800876A77EEE67A67EE877ACBED837A059AF6
:104268001278092A03F01786002C40F3A6859FB31D
:104278009BED847ADBED807A77EE877A012FCBEDA0
:10428800847AC6ED007A21D09BED857ADBED817AC0
:1042980077EE877A022FCBED857AC6ED017A15D0B5
:1042A8009BED867ADBED827A77EE877A032FCBED6A
:1042B800867AC6ED027A09D0DBED877A9BED837AA0
:1042C80077EE877ACBED877AC6ED037A013F022F26
:1042D800B8BF0227FAB20992002B099F18BF02271C
:1042E800624BDFED676A1A68059B91781878137836
:1042F80007EE903AF8EEE77AB0EE007A67EEA67A23
:10430800F4EEC77AF1EE10FA40F3E387DFED596A6D
:1043180037EEC77AB0EE676AA7EE266AF0EE466A0D
:1043280096ED007A9FED546A27EE066AF0EEC65ABB
:104338008BED526ACBED555A99B107EE101AB8EECB
:10434800C75A9FED4F7A66EE064A25EE075AB7EE32
:10435800007A37EE457A64EEA54AA4EE857A26EE11
:10436800076A9FED467A537926EE877A27EE067A12
:10437800CBB1DFED436A9FED436A65EEA65A06EEC0
:10438800903AF8EEE66A65EEA65AF4EEC65AF1EEF1
:1043980010FA01F3DE82B7EE006A76EE655AC6EED1
:1043A800256A27EE267A0C289FED378ADFED376AD3
:1043B80001F05780B4EEC87AF1EE10FA98BFB0EE6B
:1043C800478AB4EEE68AF1EE10FAB8BFB0EE668A14
:1043D8008BED4C8A002F00F00681B0EE007AF4EEE7
:1043E800C77AF1EE10FA05DD37EEC77ADFED216AFC
:1043F800E7EE267A96ED017ADFED1F6A27EE267A38
:10440800F0EEC75A8BED537ACBED565A99B106EEBA
:10441800901A9FED1B6AF8EEE66A27EE075A66EED9
:10442800866AB7EE006A36EE666A25EE255AA5EE6C
:10443800266A27EE067ADFED116A937928E000BF35
:104448003C2F0020184F002040300020E44B002073
:10445800EC4B00207C1B00203C3C00207C300020E2
:10446800D062002004490020643000200C4900205C
:104478000000C842D7A368416F12033B00004843BD
:104488000AD7233CA4707D3F00C0F94400C0F9C49A
:1044980067EEA67A67EE877AABB107EE103AB8EE08
:1044A800C77A1FED096A5FED096A27EE257A27EEBC
:1044B800067AB4EEE67AF1EE10FA41F33C825FED4B
:1044C800146A67EEA67A0C2800F0E8875FED126A96
:1044D8001FED127AF4EEE67AF1EE10FA88BFF0EEEC
:1044E800667AF4EEC77AF1EE10FAB8BFF0EE477AC2
:1044F800012FCBED4D7A76DD53785FED1F6A07EE1D
:10450800903AF8EEE77AB0EE007A67EEA67A537A38
:10451800F4EEC77AF1EE10FA05DD37EEC77A5FEDF3
:104528002B6AE7EE267A96ED027A5FED2D6A27EE82
:10453800267AF0EEC75A8BED547ACBED575A9BB1D9
:1045480006EE903A1FED326AF8EEE66A27EE075A51
:1045580066EE866AB7EE006A36EE666A25EE255A7A
:10456800A5EE266A27EE067A5FED3C6AD37967EEF8
:10457800A67A67EE877AFBB107EE103AB8EEC77AEB
:104588001FED416A5FED416A27EE257A27EE067A2C
:10459800B4EEE67AF1EE10FA01F3C981B5EEC07A0D
:1045A800F1EE10FA02F18D84B7EE006A36EE477A22
:1045B800C6EE076A67EEA67A0C2800F08E875FEDD4
:1045C8004E6A1FED4E7AF4EEE67AF1EE10FA88BFE5
:1045D800F0EE667AF4EEC77AF1EE10FAB8BFF0EEB4
:1045E800477ACBED4E7A092800F02787069B93F887
:1045F8002140002C40F0DB8600238BF8CC31BF4BE8
:104608001B7823B9BE4CA378002B41F08A82059B06
:104618001C78072C7EF44BAF07F02CF9B94B059AA0
:10462800401B1478D880FEF742BF9BF86031002BFE
:104638003FF470A9002318468BF8603107F078FA28
:10464800FFF768B9B04B1A78DBF81851AF4F9FEDF8
:10465800B07AE8003B1883ED007A002A78D0AD499B
:10466800B0EE476AF0EE476A0023F1EC017A0133B5
:1046780067EEA77A05EE903AB4EEE77AF1EE10FA13
:10468800F8EEE55AB8BFB0EE677A934276EEA76ABD
:10469800A7EEA56AE9D1F5EEC06A3B18F1EE10FA6B
:1046A80083ED007A54DDC6EE265A9B4B9B4A12884E
:1046B800F7EE007A75EEE75AD3ED007A65EEA77A41
:1046C800FDEEE77A17EE903A812B42F3718393421D
:1046D800A8BF134607EE903AF8EEE77A904B4119D7
:1046E80003EB810393ED057AD3ED003A93ED066A67
:1046F80093ED014AD3ED046AD3ED034A93ED025AD0
:10470800A3EEA77AA4EE276A66EEC76AA7EE646AE4
:10471800BDEEC77AE5EE276A17EE101A812983EDF8
:10472800056AC3ED066A42F347838A42A8BF0A4670
:1047380007EE902AF8EEE77AFCEEE77ACDED087AF4
:10474800BDF820303A18938015B9132E03F0EB8486
:10475800152E41F0E1836B4BDBF8144138441A46BF
:10476800838822F815306F4B013483FB04231A1910
:10477800E317C3EBA203C3EBC303E41ACBF814415A
:104788006949DBF81C31079C68480A680078CBF84F
:104798001C41E31A1A440A60002840F0D78007EE4B
:1047A800903A634DDFF8A081624EB8EEE78A05F5CE
:1047B800F07405F51377F5EC017A9AED070ADAF843
:1047C8000832F8EEE77A204627EE800A9847A4F1E7
:1047D800E000DAF828319847A4F17000DAF8983147
:1047E8009847D5F8EC00DAF8AC309847D6ED007A5F
:1047F800A8EC010AE0EE087A2434A742E6EC017A34
:10480800D9D1059B1C78072C7EF44AAE07F032F804
:10481800059A3C4B1478079A801A1880FEF740BE18
:104828009BED557AB1F90000DBED566AB1F902E06B
:10483800414AF4EEC76A80EAE0738EEAEE71A3EBB0
:10484800E073F1EE10FAA1EBEE71B8BFF0EE476A33
:104858008B42B8BF0B4607EE103A1378B8EEC77A0A
:1048680027EE0A7A002B00F05C81344B93ED005A56
:10487800B5EEC05AF1EE10FA40F3E885304BD3EDAF
:10488800004AF5EEC04AF1EE10FA40F3DF8534EE47
:10489800C77A66EECB5A87EE246AC5EE856AB7EE0C
:1048A800007AB4EEC76AF1EE10FA88BFB0EE476A34
:1048B800B5EEC06AF1EE10FA76EE876AB8BFB0EED0
:1048C8004D6A66EE266AF4EEC76AF1EE10FA88BF02
:1048D800F0EE476AF5EEC06AF1EE10FAB8BFF0EEF6
:1048E8004D6A184B93ED007A67EE877AA7EEA68A91
:1048F800FEF791BE0123FEF7EBBD00BFE8400020A4
:10490800BE640020D061002092300020883300204F
:10491800000000008C1D0020943000209030002002
:10492800B0320020932449921C5F00208A30002076
:10493800F8680020205F00205460002050600020AC
:10494800586000204C6000205C6B002007EE903A15
:104958009E4A9F4C9F49A04FCDF820B0F8EEE78AB9
:10496800069204F5B875904600268B46059BDAED4D
:10497800077A1B78172B6DD094ED007AB8EEC78AAA
:10498800082B28EE278A07D1B0EE480A09932AF0A7
:104998001BFC099BA8F80000D9F8002091000BD552
:1049A800002E03F04887B0EE480ADAF8083205F11D
:1049B80070009847B0EE408AB0EE480ADAF828311D
:1049C800A5F170009847DAF8983128469847059B72
:1049D8001B78032BB0EE408A37D0D4F8F000DAF811
:1049E800AC30B0EE480A9847D7ED007AABEC010A34
:1049F800E0EE287A0136032E05F1240508F10208B5
:104A080004F10404E7EC017AB0D1059BDDF820B08D
:104A18001C78F8E6714B724A234493ED007AD2ED84
:104A2800007A704B67EE277AF7EE006AF4EEE67AC2
:104A3800F1EE10FA93ED007A88BFF0EE667A67EE31
:104A4800877A27EE888AFEF72BBF2AF0BDFBA8F8E5
:104A58000000C2E794ED007A0AEB4602B8EEC78A76
:104A6800128FA8F8002028EE278A95E75E4B5F4E44
:104A78001B78D6ED037A13F0010F5D4B069304BF44
:104A88001B8BABF884315B4B1B8807EE103AB8EEF2
:104A9800C77AF4EEC77AF1EE10FA41F2D087564A97
:104AA800128807EE102AB8EEC77AF4EEC77AF1EE4C
:104AB80010FAC1F2A980514B514A93ED006AD2ED28
:104AC800006A9BF99031CBED626A76EE665A012B4B
:104AD800CBED606ACBED5F5A8BED636A01F0B0866F
:104AE800079BCBF89431002237EEC77AFCEEE77AC1
:104AF80044498BED667A17EE903AABF8843101237E
:104B080091ED005A8BF890313F4B9A4241F2C7879A
:104B18003E4BD3ED007AD3ED013AD3ED024AFEF7CE
:104B28005DBF3B4B93ED006AB4EEEB6AF1EE10FA11
:104B380040F1F287F7EE005A75EEC65A3CEEC77A96
:104B480065EE8C5A334BA7EE256A93ED007A26EE74
:104B5800076AB5EEC06AF1EE10FA40F27784CBEE40
:104B6800065AB7EE007AB0EE476AA6EEE56AF0EEAE
:104B7800466AA8E6284AD2ED007AB0EEC87AB4EEC2
:104B8800E77AF1EE10FA7EF7C5AE244AD2ED007A44
:104B9800B0EEED7AB4EEE77AF1EE10FA7EF7BAAE3F
:104BA8001F4AD8ED007A92ED007AF0EEE77AF4EE3B
:104BB800C77AF1EE10FA7EF5ADAE01220799CBF86F
:104BC80064118BF86021FEF790BE00BFD061002011
:104BD800F86800205C6B0020205F0020E01E0020A9
:104BE8004460002040600020186F0020D062002040
:104BF800247100202C6100202E610020B42F002099
:104C080018610020346100208FD003001830002084
:104C18005C600020506000208460002080600020DC
:104C280088600020804C8148814B82490893264641
:104C38001B68059006944F780478B6F906004FF47F
:104C48007A71B1FBF3F3C3EB431603EB8603DE0083
:104C5800B6B2B54202F0B380DAF87CE0BAF938208F
:104C6800DAF860300EF1010107EE902A13440129A9
:104C7800CAF87C10CAF86030F8EEE77A02F0AC8027
:104C8800DAED1B5ADAED1D6A07EE101A37EEE56AFF
:104C9800B8EEC75A012D86EE057A37EE257A77EEFB
:104CA800C77A8AED1C7AE7EE866A8AED1B7AF0EEFF
:104CB800667ACAED1E6ACAED1D6A02F09385DAF8B3
:104CC80090E0BAF93A20DAF864300EF1010107EE03
:104CD800902A13440129CAF89010CAF86430F8EEF3
:104CE800E77A02F09480DAED205ADAED226A07EECC
:104CF800101A37EEE56AB8EEC75A012D86EE057A26
:104D080037EE257A77EEC77A8AED217AE7EE866A5A
:104D18008AED207AF0EE667ACAED236ACAED226A35
:104D280002F08885DAF8A4E0BAF93C20DAF86830AD
:104D38000EF1010107EE902A13440129CAF8A410C4
:104D4800CAF86830F8EEE77A02F07C80DAED255A86
:104D5800DAED276A07EE101A37EEE56AB8EEC75A99
:104D6800012D86EE057A37EE257A77EEC77A8AED39
:104D7800267AE6EE276A8AED257AF0EE667ACAED9B
:104D8800286ACAED276A02F02085069BDFF8C8B0BA
:104D9800D880BAF8A830059A013B1478AAF8A83048
:104DA800089900234B608B60CB60FEF776BBABF8AD
:104DB800FC41002B3FF423AC1F4E0227FFF790BAAB
:104DC8001E4B1F4A19681288174BC96919805A80E7
:104DD8001BB0BDEC0E8BBDE8F08F1A4B1B7813F09F
:104DE800010F194B089340F0CD831A78002A00F080
:104DF800C185920015491648DFF860902AF0A4F89A
:104E0800144B0693FFF780B9084B0593DFF848B0B9
:104E1800B6E4BBF8FC41013C24B2002CABF8FC41E1
:104E2800C7DD054EFFF723BAD0610020CC61002012
:104E3800586B0020446B0020D0620020BC4A002040
:104E4800EE2C0020186F0020AD610020F02C00200F
:104E580040300020247100208C1D0020686B002049
:104E6800002C01F06782002F42F09486BEF1000FFB
:104E780042F0108590ED006A9DED125AAE4925EE7C
:104E8800866AFDEEE44AA5EE076AB0EE675AA6EE1A
:104E9800265A14EE903ABDEEC56A16EE105A16EE72
:104EA800104AB542A8BF3446AB42C8BF1C4606EEFE
:104EB800104AB8EEC66A012A81ED006A00F0DF8068
:104EC80090ED046A9DED135A25EE866AA5EE076AF1
:104ED800B0EE675AA6EE265ABDEEC56A16EE105A0F
:104EE80016EE104AB542A8BF34469D42B8BF1C46CC
:104EF80006EE104AB8EEC66A022A81ED016A00F091
:104F0800BE8090ED086A9DED145A25EE866AA5EEDE
:104F1800076AB0EE675AA6EE265ABDEEC56A16EEC7
:104F2800105A16EE104AB542A8BF34469D42B8BF83
:104F38001C4606EE104AB8EEC66A032A81ED026ADC
:104F480000F09D8090ED0C6A9DED155A25EE866A5D
:104F5800A5EE076AB0EE675AA6EE265ABDEEC56AF8
:104F680016EE105A16EE104AB542A8BF34469D42B6
:104F7800B8BF1C4606EE104AB8EEC66A042A81ED90
:104F8800036A7CD090ED106A9DED165A25EE866A6C
:104F9800A5EE076AB0EE675AA6EE265ABDEEC56AB8
:104FA80016EE105A16EE104AB542A8BF34469D4276
:104FB800B8BF1C4606EE104AB8EEC66A052A81ED4F
:104FC800046A5CD090ED146A9DED175A25EE866A46
:104FD800A5EE076AB0EE675AA6EE265ABDEEC56A78
:104FE80016EE105A16EE104AB542A8BF34469D4236
:104FF800B8BF1C4606EE104AB8EEC66A062A81ED0E
:10500800056A3CD090ED186A9DED185A25EE866A1F
:10501800A5EE076AB0EE675AA6EE265ABDEEC56A37
:1050280016EE105A16EE104AB542A8BF34469D42F5
:10503800B8BF1C4606EE104AB8EEC66A072A81EDCC
:10504800066A1CD090ED1C6A9DED195A65EE865AC9
:10505800E7EE055AE6EEA57AFDEEE77A17EE900A36
:105068008642A8BF06468342D8BF334607EE903A29
:10507800F8EEE77AC1ED077A002A3FF445A89200D6
:105088002E492D4829F060FF2D4B1B68002B3FF45B
:1050980040A82C4B1B78192B07D801212A4A01FA62
:1050A80003F31A40002A41F0EF87DFF8B480274E57
:1050B800D9F80030990655D5F27AFF2A04D0244B46
:1050C8001B78934201F2E582B6F90850F27DA8F800
:1050D8000050FF2A01F0AF841D4B1B78934241F228
:1050E800AA841C4B33F91240A8F8024008201EF08D
:1050F8003BFAB8B39BF8C031012B02F08086164BFF
:1051080096F9160096F90A705A881B88134910FBFD
:1051180003F317FB02F281FB020781FB0301D2179D
:10512800DB17C2EB2712C3EB21132A441C44A8F84F
:105138000020A8F8024015E040300020F02C0020A4
:105148003C2F0020402F002032C13003343700208C
:10515800DC5B00203C3C0020B44800201F85EB515C
:1051680030300020B8F90070B6F90600B8F90250DE
:10517800B6F91210B8F90440B6F91E20B6F9043091
:10518800B8F90EE0B842A8BF3846A942A8BF2946D8
:10519800A242A8BF2246BB42D8BF0346A8F80030A7
:1051A800B6F91030B8F90670B8F90800AB42C8BFB4
:1051B8001946B6F92A30A8F80210B6F91C10B8F941
:1051C8000C50BB42A8BF3B46A142C8BF0A46B6F92D
:1051D8003640A8F80420B6F92820B8F90A10844205
:1051E800A8BF0446BA42C8BF1346B6F94220A8F879
:1051F8000630B6F93430B6F94E708A42A8BF0A466E
:105208008342D8BF2346A8F80830B6F94030B6F92B
:105218005A00AF42A8BF2F468B42D8BF1346A8F802
:105228000A30B6F94C30B6F958207045A8BF704618
:10523800AB42C8BF1F46C24BA8F80C709645B8BF12
:105248001046A8F80E009B8913B3BE4DBE4FBF4E43
:1052580005F11004B5F9023000EE103A3846B8EE00
:10526800C00AFBF769F829F0AFFFB6F90430B6F9C0
:10527800062000B2984207F1240706F10C0603DB6A
:1052880082421346A8BF034625F8023FAC42E1D14B
:10529800AF4B1B78013B182B01F2D882DFE813F0E3
:1052A800490AD60AD60A4609D60AD60AD60A390AB1
:1052B800D60AD60AD60AD60AD60A190AFE09D60A7C
:1052C800D60AD60AD60A4609290AD60AD60A190AD1
:1052D800490AF0EE676AFFF723B8B0EE465AFEF7C0
:1052E800B4BB9C499C4AD1F8EC10126844F6206083
:1052F8008142A8BF0146B1F57A7FB8BF4FF47A71F1
:1053080089B212F0100FABF8CE11D9F8002000F0D6
:105318007684D00441F1F587904A17687C8E64083A
:105328008F4E9048DBF8D021D6ED037AA0FB01011F
:105338008809642191FBF0F11429BDEEE77A0BEBA3
:105348004206A8BF142101329142CBF8D02117EEB2
:1053580010EADCBF0022CBF8D0210BEB4202A6F802
:10536800D4E1B2F9D42107EE102AB8EEC77A77EE65
:10537800C77AFDEEE77ACDED087ABDF9201081EA0B
:10538800E172A2EBE172A24202F3048276494FF085
:105398007E520A60FEF705BFDAF80830002B3EF4AB
:1053A800D8AE7249A1F14C009847FEF7D2BE1E2133
:1053B8006948FDF763FC00283FF41EA96C4B1B8865
:1053C8005B063FF519A99BF82032A34242F04085BD
:1053D800654B9BED890AD3ED018ADBED4E5A9FEDB3
:1053E800656ADFED656A20EE657A68EE007AA8EEF8
:1053F800287AE5EEA87AB4EEC67AF1EE10FA88BFFC
:10540800B0EE467AB4EEE67AF1EE10FAF4EEC67A29
:10541800B8BFB0EE667AF1EE10FA88BFF0EE467AC1
:10542800F4EEE67AF1EE10FAB8BFF0EE667A8BED9C
:105438004C7ACBED4E7AFFF7DFB8FDEEC87A4F4ACB
:1054480017EE903A9480D380FFF7D0B8DFED4C6A1E
:10545800FFF747BAD9F800305D023EF5FCACFEF71D
:10546800FEBCB4EEC87AF1EE10FA98BFB0EE478AE7
:10547800BDEEC77AB4EEE68ADFF800E1F1EE10FA85
:1054880017EE103AB8BFB0EE668A8BED4C8AAEF8CC
:105498000030002F7EF4A1AFFFF7A8B89FED357A52
:1054A800DFED356A3549F4EEC77AF1EE10FA98BFA8
:1054B800B0EE677AFDEEE77AB4EEE67AF1EE10FA2E
:1054C80017EE903AB8BFB0EE667A012F8BED4D7AA1
:1054D8004B803FF711A8FFF789B8BDEEE77A274B55
:1054E80017EE102A9A80FFF76AB8002B3EF412AA2A
:1054F800FEF7F7B906F0BEF9059B0B991B781F4A12
:10550800401A072B90807EF41EAE06F0B3F90546CC
:10551800FEF71ABE06F0AEF9184B06931A46059B1D
:105528000A991B78401A012B508000F05183072BF1
:105538007EF418AA06F09EF90B90FEF715BA00BF84
:105548005C6600202E3000201C2E002034370020FE
:10555800402F0020C40600201C71002008490020AC
:10556800D0620020D34D621000000020186900208E
:105578000449002000C0F94400C0F9C4D0610020EB
:10558800000000001B78002B00F0F481DBED563A98
:105598009BED556ADBED607AF04A9BED5F7AD2EDC0
:1055A800005A9BED534ADBED524AED48ED49F4EEC3
:1055B800C63AF3EE046AF1EE10FA37EEA65A00F195
:1055C800A58390ED026A26EE446AF0EE674AE6EE9D
:1055D800074AF4EEC54A34EEE66AF1EE10FA48BF1F
:1055E800B0EE656A012B81ED006A00F0C38190ED91
:1055F800066A26EE446AF0EE674AE6EE074AF4EEDB
:10560800C54A34EEE66AF1EE10FA48BFB0EE656AB4
:10561800022B81ED016A00F0AD8190ED0A6A26EE59
:10562800446AF0EE674AE6EE074AF4EEC54A34EEFD
:10563800E66AF1EE10FA48BFB0EE656A032B81ED19
:10564800026A00F0978190ED0E6A26EE446AF0EE49
:10565800674AE6EE074AF4EEC54A34EEE66AF1EE2A
:1056680010FA48BFB0EE656A042B81ED036A00F0BA
:10567800818190ED126A26EE446AF0EE674AE6EE02
:10568800074AF4EEC54A34EEE66AF1EE10FA48BF6E
:10569800B0EE656A052B81ED046A00F06B8190ED30
:1056A800166A26EE446AF0EE674AE6EE074AF4EE1A
:1056B800C54A74EEE66AF1EE10FA48BFF0EE656A84
:1056C800062BC1ED056A00F05581D0ED1A6A66EE29
:1056D800C46AF0EE674AE6EE874AB3EE046AF4EE6F
:1056E800C54A74EEC66AF1EE10FA48BFF0EE656A74
:1056F800072BC1ED066A00F03D81D0ED1E6A9A4B7A
:10570800DFF86C92069326EEC44AE4EE077AF4EECC
:10571800C57A77EEC67AF1EE10FA48BFF0EE657AF0
:10572800C1ED077AFEF7F0BC002F41F03D8225EE6F
:10573800866A8C49A5EE076AB0EE675AA6EE265A25
:10574800BDEEC56A16EE105A16EE104AB542A8BF4D
:105758003446AB42C8BF1C4606EE104AB8EEC66ACD
:10576800012A81ED006A3FF48AAC90ED046A9DED50
:10577800135A25EE866AA5EE076AB0EE675AA6EEBA
:10578800265ABDEEC56A16EE105A16EE104AB542F4
:10579800A8BF3446AB42C8BF1C4606EE104AB8EE56
:1057A800C66A022A81ED016A3FF469AC90ED086A85
:1057B8009DED145A25EE866AA5EE076AB0EE675A83
:1057C800A6EE265ABDEEC56A16EE105A16EE104A17
:1057D800B542A8BF3446AB42C8BF1C4606EE104AC5
:1057E800B8EEC66A032A81ED026A3FF448AC90ED30
:1057F8000C6A9DED155A25EE866AA5EE076AB0EE8D
:10580800675AA6EE265ABDEEC56A16EE105A16EE6F
:10581800104AB542A8BF3446AB42C8BF1C4606EE84
:10582800104AB8EEC66A042A81ED036A3FF427AC31
:1058380090ED106A9DED165A25EE866AA5EE076A68
:10584800B0EE675AA6EE265ABDEEC56A16EE105A95
:1058580016EE104AB542A8BF3446AB42C8BF1C4634
:1058680006EE104AB8EEC66A052A81ED046A3FF4CE
:1058780006AC90ED146A9DED175A25EE866AA5EEE2
:10588800076AB0EE675AA6EE265ABDEEC56A16EE4E
:10589800105A16EE104AB542A8BF3446AB42C8BFEC
:1058A8001C4606EE104AB8EEC66A062A81ED056A5D
:1058B8003FF4E5AB90ED186A9DED185A25EE866A1F
:1058C800A5EE076AB0EE675AA6EE265ABDEEC56A7F
:1058D80016EE105A16EE104AB542A8BF3446AB422F
:1058E800C8BF1C4606EE104AB8EEC66A072A81ED04
:1058F800066A3FF4C4AB90ED1C6A9DED195A65EE3B
:10590800865AE7EE055AE6EEA57AFDEEE77A17EE37
:10591800900A8642A8BF06468342C8BF1E4607EEC5
:10592800906AF8EEE77AC1ED077AFFF7A5BBDFEDDD
:105938000F6AFEF73FBEB5EEC07AF1EE10FA01F13C
:10594800C482B7EE006A36EE477AC6EE076AFEF7FB
:10595800B8BDDFED066AFEF724BD00BF94600020E5
:105968009860002040300020247100200000C842C8
:10597800686B0020CB4BDFF890930693FEF7C4BB0F
:10598800C94A5379002B3EF4E8A8C84B1B78002B72
:105998003EF4E3A81278DFEDC64A07EE902AC54A1E
:1059A800B8EE677A128807EE903A06EE902AF8EE7B
:1059B800E77AF8EE666A67EE277AB7EE007A87EE3E
:1059C800A63AB4EEE43AF1EE10FA88BFB0EE643AC3
:1059D800B4EEC73AF1EE10FAB8BFB0EE473AFEF7A8
:1059E800BEB8BBF8CE2102F57A7292B2FEF7ECBBD4
:1059F800B14A5288FEF7E8BBB04A059207EE103A62
:105A08001278AF490691B8EEC77AF7EE006A00231C
:105A1800132AB1F904009AED070ABBF81041CBF834
:105A28000C3186EE879A01F06182A64BA64A02EBFA
:105A380084050021CBF80011CBF8041167EE897AB0
:105A480093ED001AD3ED053A93ED122A93ED173A28
:105A5800D3ED091AD3ED0E4A93ED016A93ED064A88
:105A680093ED0A7AD3ED0F5AD3ED132AD3ED186AC2
:105A780093ED045AD3ED030A69EE288A29EE088AC1
:105A8800E1EE273AA2EE283AE1EE884AA6EE274A46
:105A9800E7EE085A93ED167A93ED0D6A93ED021A24
:105AA800D3ED0C1AC5ED003AE2EEA86A25EE635A6A
:105AB80027EE437A93ED0B2AD3ED152AC5ED204A3C
:105AC800A0EEE34A26EE646AD3ED143A83ED054A64
:105AD800A1EE275AF0EE477AE1EEE45AA2EE086A00
:105AE800E2EEC36AE3EEA87A83ED065AC3ED0E5AD6
:105AF80083ED0F6A85ED403AC3ED176AC3ED187A56
:105B0800CBF80811631C03F01F03ABF81031069B98
:105B18009880059BFDF7A8BC6C4B93ED006AFFF7D6
:105B280018B86B4E3278013A0A2A20D8DFE812F00A
:105B3800FC0678072D0712071F001F0034066507AB
:105B4800D7060B00BC06634B1B78002B02F0FD82C6
:105B58001A201DF009FD002842F0F7825E4B1B78E1
:105B6800002B42F0F2820923337026F093FF237949
:105B7800012B00F02986022B7EF449AD3378012BE6
:105B88007EF445AD544B1B78002B7EF440AD26F0D7
:105B980061FCFEF73CBD514B9FED517AD3ED087A7D
:105BA800F4EEC77AF1EE10FA00F2FF849FED4D7A19
:105BB8004D4ED6ED037A77EE877AC6ED037AFEF777
:105BC800EBBA05F057FE0A90FDF789BC3C4B0693EB
:105BD80005F050FE454ADBF8743112680B90C31A81
:105BE800CBF8740106989A1A8380C280FDF7BCBE70
:105BF8003F4B9B7B002B3EF4C2AAFEF7C5BAD000F0
:105C08003FF587ABFEF7CDBABBF884219A4200F284
:105C1800178526201DF04CFC002840F01185354BD7
:105C2800354AD3ED007A354B92ED007A1B78CBEDEF
:105C3800627A8BED637A002B01F0A68577EE676AAE
:105C48009BF99031CBED5F6A0133CBED607A02F0BE
:105C5800F980079BCBF8943100229FED227A2849DE
:105C68008BED667AFF2391ED005A8BF89031FEF7A1
:105C78004BBF012005F05CFFDBF86431079AD31AAB
:105C8800FDF7E2BC1F4BD8ED007A93ED007AF0EEF9
:105C9800E77AF4EEC77AF1EE10FA7DF73BAEFDF73E
:105CA80033BE00BF24710020A0480020CE6200202F
:105CB800713DAA3FB8620020DC5B0020CC61002067
:105CC800D06100201C330020B0300020506000203C
:105CD800BC6400207E300020956F0020F45E002018
:105CE8008FC2753C00000000D062002064300020A4
:105CF8005C660020C46F00201C610020F04B00206F
:105D08003061002088600020686B002090ED016AF7
:105D180026EE646AB0EE674AA6EE074AB4EEC54AB4
:105D280034EE666AF1EE10FA48BFB0EE656A012BF0
:105D380081ED006A3FF41EAE90ED056A26EE646AB6
:105D4800B0EE674AA6EE074AB4EEC54A34EE666A74
:105D5800F1EE10FA48BFB0EE656A022B81ED016AD8
:105D68003FF408AE90ED096A26EE646AB0EE674A21
:105D7800A6EE074AB4EEC54A34EE666AF1EE10FAAA
:105D880048BFB0EE656A032B81ED026A3FF4F2ADBD
:105D980090ED0D6A26EE646AB0EE674AA6EE074AF1
:105DA800B4EEC54A34EE666AF1EE10FA48BFB0EEBA
:105DB800656A042B81ED036A3FF4DCAD90ED116A4E
:105DC80026EE646AB0EE674AA6EE074AB4EEC54A04
:105DD80034EE666AF1EE10FA48BFB0EE656A052B3C
:105DE80081ED046A3FF4C6AD90ED156A26EE646A4B
:105DF800B0EE674AA6EE074AB4EEC54A74EE666A84
:105E0800F1EE10FA48BFF0EE656A062BC1ED056A9F
:105E18003FF4B0ADD0ED196A66EEE46AB0EE674AB9
:105E2800A6EE874AB3EE046AB4EEC54A74EE466A33
:105E3800F1EE10FA48BFF0EE656A072BC1ED066A6D
:105E48003FF498ADD0ED1D6ACC4BDFF85093069324
:105E580066EEE44AE4EE877AF4EEC57A77EEC67A1F
:105E6800F1EE10FAB8BFF0EE657AC1ED077AFEF7E9
:105E78004BB9C34DDBED017A9BED006A28886B694D
:105E880077EEA77AF0EE006AB0EE677AA6EE267A89
:105E980001380BEBC002D6EE267A083A1033F6EE3C
:105EA800003A27EE237A67EEA37A8BED207ACBEDC2
:105EB800217ADFF8E4B25D460BF1800192ED027AB7
:105EC80092ED036AD5ED036AD5ED027A53ED014AE6
:105ED80013ED025A37EE674A76EEC65A77EE277AFE
:105EE800E4EE845A0138A2F10802E5EE047A05F1DD
:105EF800080503F1080336EE267A01F10801E4EEFD
:105F0800877AE5EE475A67EEA37A25EEA37AC1EDC4
:105F1800007A81ED017AD1D1142E7EF424AC05F0FB
:105F2800A9FC069A974B801A5880DBF81441FEF7B3
:105F38001ABCDBF818C1BBF81071934BC7F12008E5
:105F48005FFA88F807EB4C1503EB85055FEA9803C1
:105F580002F0F680013318018C498D4A05EB000EDA
:105F680005F1100313ED024A13ED035A13ED016A0C
:105F780013ED047A51ED024A51ED035A51ED016ACD
:105F880051ED047A64EE244A65EE255A66EE266AD7
:105F980067EE277A10339E4542ED024A42ED035AD6
:105FA80042ED016A42ED047A01F1100102F110029A
:105FB800D8D17849A0F11002154401EB020E5A44D9
:105FC80018F0030309D0B5EC017AFEEC017A67EE0C
:105FD800277A013BE2EC017AF5D1002F41F00280EB
:105FE800142E7EF4C0AB05F045FC069A654BDBF831
:105FF8001441801A5880FEF7B6BB614D2A88D5F83F
:1060080004E04FEA520C4FEA8C01D7080BEB01036E
:106018000BEB820400F0A08001F1100201375C480C
:1060280003EB0717224410330EF1100604F1100198
:1060380051ED032A51ED043A10ED043A10ED032A0C
:1060480051ED026A11ED016A10ED020A10ED018AA4
:1060580012ED044A12ED035A53ED044A53ED035A64
:1060680013ED027A53ED017A52ED020A12ED011A8C
:1060780073EE238A72EE221A40ED048A40ED031A69
:1060880070EE268A78EE061A40ED028A40ED011A73
:1060980074EE848A75EE851A43ED048A43ED031A7B
:1060A80077EE208A77EE811A43ED028A43ED011AD2
:1060B80073EE633A75EE655A16ED035A32EE623A9C
:1060C80074EE644A65EE631A16ED044A23EE052A57
:1060D80064EE652AE3EE041A10339F4224EE843AF4
:1060E800A3EE842A00F1100006F11006A5EE853A09
:1060F80001F1100102F11002E4EE852A41ED071AC0
:1061080001ED082A02ED073A42ED082A56ED055A34
:1061180016ED065A70EE666A38EE466A30EEC77AB1
:1061280071EE677A26EE253A65EEE63A25EE674A7D
:1061380067EE054AE6EE053AA6EE853AA7EE254A49
:10614800E7EEA54A01ED063A41ED053A02ED064AA9
:1061580042ED054A7FF46CAF1FFA8CF67246314661
:106168000D4824F017FC31466A68204624F012FCDA
:10617800059B1B78142B7FF4D8AED0E62471002041
:1061880098300020D0610020B0300020403200203C
:106198009C1D0020303200208C1D0020686B0020E0
:1061A800D94D2A78970802F0C781D84807F1010C21
:1061B8004FEA4C1C00EB0C0E00F12003A0F170011B
:1061C80013ED076A53ED056A13ED037A53ED017A6F
:1061D80053ED025A13ED084A53ED064A13ED045ADB
:1061E80026EE066A66EEA66A27EE077A67EEA77AB3
:1061F800A4EE046A20339E45E4EEA46A01F110017E
:10620800A5EE057AE5EEA57AF1EEC65AB1EEE66A94
:10621800F1EEC76AB1EEE77A41ED085A01ED076A77
:1062280041ED066A01ED057ACAD1ACF120030344B9
:106238000BEB071712F0030118BF08330FD053ED0B
:10624800017A13ED027A67EEA77A0139E7EE077A49
:1062580003F10803B1EEE77AA7EC017AEFD1142E27
:1062680001F0D0870134CBF81441FEF7EDB9A84D01
:10627800A848AA68A98927F099FE059B1E78142EBC
:1062880001F0D787DBF814410134CBF81441F1E56C
:10629800DBF81821A04BA149A14C1846D30019449A
:1062A8001A448B88016800EE103A10EE103A643BED
:1062B800C82BA8BFC823782BB8BF782307EE903A1D
:1062C800B8EEC07AF8EEE77A04EB820477EE670A54
:1062D80077EE876A67EE877A20EEA67AB8EE400AEC
:1062E800C7EE870A2046D4F81880E769256A94ED36
:1062F800058A26F001FC059B84ED058A1E78C4F802
:106308001880142EE761256201F08987DBF81831BF
:10631800844ADBF81441013382FB0312A2EBE37CCD
:106328000CEB4C02A3EB020C0134CBF818C1CBF8F0
:10633800144100E6BEF1000F41F0DC8090ED006AE8
:106348009DED125A784925EE866AFDEEE44AA5EEDF
:10635800076AB0EE675AA6EE265A14EE903ABDEEDA
:10636800C56A16EE105A16EE104AB542A8BF344652
:10637800AB42C8BF1C4606EE104AB8EEC66A012AF0
:1063880081ED006A3DF4BDAE90ED046A9DED135AAF
:1063980025EE866AA5EE076AB0EE675AA6EE265A7B
:1063A800BDEEC56A16EE105A16EE104AB542A8BFE1
:1063B80034469D42B8BF1C4606EE104AB8EEC66A7F
:1063C800022A81ED016A3DF49CAE90ED086A9DEDCC
:1063D800145A25EE866AA5EE076AB0EE675AA6EE4D
:1063E800265ABDEEC56A16EE105A16EE104AB54288
:1063F800A8BF34469D42B8BF1C4606EE104AB8EE08
:10640800C66A032A81ED026A3DF47BAE90ED0C6A00
:106418009DED155A25EE866AA5EE076AB0EE675A15
:10642800A6EE265ABDEEC56A16EE105A16EE104AAA
:10643800B542A8BF34469D42B8BF1C4606EE104A76
:10644800B8EEC66A042A81ED036A3DF45AAE90EDAF
:10645800106A9DED165A25EE866AA5EE076AB0EE1B
:10646800675AA6EE265ABDEEC56A16EE105A16EE03
:10647800104AB542A8BF34469D42B8BF1C4606EE36
:10648800104AB8EEC66A052A81ED046A3DF439AEB1
:1064980090ED146A9DED175A25EE866AA5EE076AF7
:1064A800B0EE675AA6EE265ABDEEC56A16EE105A29
:1064B80016EE104AB542A8BF34469D42B8BF1C46E6
:1064C80006EE104AB8EEC66A062A81ED056A3DF462
:1064D80018AE90ED186A9DED185A25EE866AA5EE5D
:1064E800076AB0EE675AA6EE265ABDEEC56A16EEE2
:1064F800105A16EE104AB542A8BF34469D42B8BF9E
:106508001C46FDF7DCBD00BF923000200C1E0020A9
:10651800983000208C1D0020586B00208833002004
:10652800D86A00205655555540300020C84BB8F958
:1065380008101A6802B111609B69B8F90A20002B8B
:1065480000F0F3801A60032604220225D9F80030EF
:10655800990600F1DC86DB027DF5DBADBD4BDE7B09
:10656800112E3DF7D6ADBC4C34F9163000EE103A7A
:106578002846B8EEC00A17F089F804EB460401274C
:10658800C6F11206E819B742C0B207F101073DF497
:10659800C0AD34F9023F00EE103AB8EEC00A17F069
:1065A80075F80E2FEED1FDF7B4BDF0EEE76AB7EE41
:1065B800005A35EE665A9FEDA94ADFEDA95A9FEDBC
:1065C800A96A9FEDA97A9BED720AF1EEC54AE6EE3B
:1065D800845AF5EEC07AA6EEA56AF1EE10FAA6EE98
:1065E800867A48BFDFEDA17A27EE247A48BF37EED6
:1065F800C77A27EE000A28F0E7FDB0F5617F01F3BE
:10660800B78007EE900AB8EEE70ADFED997A20EE38
:10661800270A07EE904AB8EEE78AFDEEC07A17EE31
:10662800903A2033402B41F2A9809FED920A28F03E
:10663800CBFD00B207EE900AB8EEE77AFFF7B8BADA
:106648009BF89C21002A7FF4EAAA8B4B8B4993ED97
:10665800007AD1ED007A9BF99031CBED627A77EE32
:10666800676A012BCBED607ACBED5F6A8BED637ABD
:1066780001F0BA85079BCBF89431814B9FED7D7A69
:1066880093ED005A8BED667A01238BF89031FEF773
:106698003BBA714B33F91250FEF718BD6C4BB8F981
:1066A80000101A6802B111609A69B8F9021002B1B3
:1066B80011601A6BB8F9041002B111609B6CB8F93B
:1066C8000620002B01F05D871A60052606220425A6
:1066D8003CE76C4D002435F9023F00EE103AE0B279
:1066E800B8EEC00A013416F0D1FF062CF3D12046CB
:1066F80031E0654D002435F9023B00EE103AE0B276
:10670800B8EEC00A013416F0C1FF042CF3D12046BC
:1067180021E04F4BB8F906101A6802B111609B6965
:10672800B8F90820002B7FF40DAF032604220225B8
:106738000CE7484B9B7B002B41F01B82534B1B788B
:1067480013F0010341F01582414A1268002A01F052
:10675800708713600120D9F800309A0604D44C4A97
:106768001278052A40F03684851C461CEDB2F6B234
:10677800B8F9003000EE103AB8EEC00A16F086FFFD
:10678800B8F9023000EE103A3046B8EEC00A16F0FA
:106798007DFFD9F80030DEE625F014FD3D4B0021E1
:1067A80005208DE80300A3F10802029153200FF0A1
:1067B80059F900287FF4DBA9374A082310603370A1
:1067C8002379012B7DF423AF344F304B1B78DC0742
:1067D80040F1B380DBF828223B689A423FF6CEA905
:1067E8003378012B3DF413AFDFF8B88098F8002018
:1067F800002A3DF40CAF0B2B18D801229A4040F622
:10680800030112EA010416D112F4C06F0ED0093B3D
:10681800012B0BD8452025F015FDFF2025F012FD92
:106828001F4825F0FBFC204625F00CFD1A4B3A6862
:106838005A600B233370002388F80030FDF7E7BE59
:10684800DBF89421079B9A1AFEF74EB9002082E7DD
:106858006C6600205C6600203C3C0020306E99BCD1
:106868002716983D843459BEA40DC93FDB0F494013
:10687800D06D393A00000000B42F002018610020C4
:10688800346100203230002036300020186F00209C
:10689800402F0020E8040308B82F0020BC71002016
:1068A8005C280308956F0020AB4AAC4F52683968E2
:1068B800C8328A4205D325F0A3FC00283FF457A923
:1068C800A378032B01F0EE862379012293423270DC
:1068D8003FF47BAF022B3FF455A9FDF798BE1A2071
:1068E8001CF042FE00283FF440A99D4B1B88002B5A
:1068F8007FF43BA99B4B45201F6825F0A3FC0E2085
:1069080025F0A0FC384625F043FD079F384625F0C2
:106918003FFD954A954B12681A6038460A23337032
:1069280025F008FEFFF721B9914B1B78DF0701F12D
:106938001E862379012BCDD1884F1CF021FD00281C
:106948003FF448AF3B6803F59C530833CBF8283233
:10695800FFF714B925F036FC864A0292A2F10C031F
:10696800252101930091A2F10A035021163A4920EA
:106978000FF078F800287FF4FAA8774B4FF0FF3132
:1069880007221860596032701AE7DFF8CC81734F1C
:1069980025F018FCD8F804303A6864339342BFF401
:1069A800E6A8402025F0F4FB00287FF4E0A8D8F8FA
:1069B8000030714FDFF8C4A14FF040090FE025F017
:1069C80041FCDAF80020D8F80030013A0133B9F177
:1069D8000109CAF80020C8F8003001F0D386FB5C32
:1069E8001846002BEBD100234FF0FF32C8F80030D7
:1069F8000423C8F804203370E2E625F0E3FB0EF028
:106A080075FB00283FF4B3A825F0FAFB00283FF4F3
:106A1800AEA8554A554B12681A600A233370CFE660
:106A28004E4F4D4A3B68536054490023136003227C
:106A38000B603270C4E6B6F91440FEF755BB504BF4
:106A4800504AD3ED006A504B92ED006A1B78CBEDAB
:106A5800626A8BED636A002B00F0BF8276EE665A9D
:106A68009BF99031CBED5F5A0133CBED606A01F0B1
:106A78007A80079BCBF89431002237EE677AFCEED8
:106A8800E77A42498BED667A17EE903AABF8843193
:106A9800FF2391ED005A8BF89031FEF735B83C4B47
:106AA800DFED3C7A1C683C4B9BED667AC3ED007ABF
:106AB800F0EE674AC3ED017AC3ED027AF0EE673A69
:106AC800FCF78CBF04F0D6FE059B06901E78142EAA
:106AD80005BF324BDBF81441DBF814411C80FCF78E
:106AE800CBBC2F4BDFED2F7A1B68CBED4A7A13F026
:106AF800805C40F05D86D9F8003013F4800C00F01B
:106B08000A844FF0000CB6EE007A67EE877AF4EE4E
:106B1800E75AF1EE10FA48BFF0EE675A40F148869E
:106B2800CBED665AFDF79BB9114B187800F00107B9
:106B3800FDF7E7BA73EEE77AB7EE007AF4EEC77AB4
:106B4800F1EE10FACBED4A7A41F3548384EEA77A3A
:106B58008DED127AFDF779B9B82F0020BC710020AD
:106B68009C6F0020986F0020AC6F0020A46F00205D
:106B7800186F00203A030308D40203088C6F002022
:106B8800C46F00201C610020F04B00203061002001
:106B9800084900200000000018300020D0610020C3
:106BA8001C71002000000080B8F1000F01F0A281E4
:106BB80025EE866AC749A5EE076AB0EE675AA6EEC3
:106BC800265ABDEEC56A16EE105A16EE104AB542A0
:106BD800A8BF3446AB42C8BF1C4606EE104AB8EE02
:106BE800C66A012A81ED006A3DF48EAA90ED046A16
:106BF8009DED135A25EE866AA5EE076AB0EE675A30
:106C0800A6EE265ABDEEC56A16EE105A16EE104AC2
:106C1800B542A8BF3446AB42C8BF1C4606EE104A70
:106C2800B8EEC66A022A81ED016A3DF46DAA90EDBC
:106C3800086A9DED145A25EE866AA5EE076AB0EE3D
:106C4800675AA6EE265ABDEEC56A16EE105A16EE1B
:106C5800104AB542A8BF3446AB42C8BF1C4606EE30
:106C6800104AB8EEC66A032A81ED026A3DF44CAABE
:106C780090ED0C6A9DED155A25EE866AA5EE076A19
:106C8800B0EE675AA6EE265ABDEEC56A16EE105A41
:106C980016EE104AB542A8BF3446AB42C8BF1C46E0
:106CA80006EE104AB8EEC66A042A81ED036A3DF47E
:106CB8002BAA90ED106A9DED165A25EE866AA5EE70
:106CC800076AB0EE675AA6EE265ABDEEC56A16EEFA
:106CD800105A16EE104AB542A8BF3446AB42C8BF98
:106CE8001C4606EE104AB8EEC66A052A81ED046A0B
:106CF8003DF40AAA90ED146A9DED175A25EE866AAE
:106D0800A5EE076AB0EE675AA6EE265ABDEEC56A2A
:106D180016EE105A16EE104AB542A8BF3446AB42DA
:106D2800C8BF1C4606EE104AB8EEC66A062A81EDB0
:106D3800056A3DF4E9A990ED186A9DED185A25EE0B
:106D4800866AA5EE076AB0EE675AA6EE265ABDEE29
:106D5800C56A16EE105A16EE104AB542A8BF344658
:106D6800AB42C8BF1C4606EE104AB8EEC66A072AF0
:106D780081ED066A3DF4C8A990ED1C6A9DED195A8B
:106D880065EE865AE7EE055AE6EEA57AFDEEE77A55
:106D980017EE902A9642A8BF16469342D8BF3346AC
:106DA80007EE903AF8EEE77AC1ED077AFDF7ACB94D
:106DB800DFED497AFDF792BC8223FDF7C3BCBAF92F
:106DC8003830CAF8202007EE903A0122F8EEE77A28
:106DD800CAF86030CAF87C200023012DCAED1C7A5D
:106DE800CAED1B7ACAF8743001F0AB83B5427DF462
:106DF80066AFBAF93A30CAF8643007EE903A002222
:106E08000123F8EEE77ACAF82420CAF89030002364
:106E1800012DCAED217ACAED207ACAF8883001F02E
:106E28009783B5427DF47EAFBAF93C30CAF8683032
:106E380007EE903A00220123F8EEE77ACAF82820F4
:106E4800CAF8A4300023012DCAED267ACAED257AA6
:106E5800CAF89C307DF499AF9FED208A032C2AD084
:106E68004FB107EE907AF8EEE77AF4EEC87AF1EED1
:106E780010FA01F1D6831A4BDFF86CB01A68069B3A
:106E88009BF82011D880DAF8683003EB560393FB9F
:106E9800F6F60023CAF8286093621363D36229B117
:106EA800104B1B6833F480637DF473AF012021F02D
:106EB800D5FFFDF76EBFB0EE480A28F085F900B29D
:106EC800CEE7F7EE006AFDF775BBF7EE006AFDF74F
:106ED800F8BA00BF40300020000002430000000064
:106EE800BC4A0020004900208C1D0020B14DB24E44
:106EF80095ED004A95ED057AD5ED014A95ED066ABE
:106F0800D5ED046A95ED035AD5ED025A67EE897AF4
:106F180006EB8403A4EE277AA4EEA76A66EEC76A96
:106F2800A5EE476AE5EEA76A20EE070A85ED056A31
:106F3800C5ED066A29EE088A69EE288A83ED007A8B
:106F480028F042F9D5ED0E5AD5ED176A95ED091AD4
:106F5800D5ED121A95ED0F5A95ED187A95ED0A2A86
:106F6800D5ED132A95ED0D6AD5ED167A95ED0C3A07
:106F7800D5ED0B3A95ED154AD5ED144AE1EE085AD0
:106F8800002206EB8401E8EEA16A00B2CBF80021EA
:106F9800A2EE085ACBF80421CBF80821A8EEA27A71
:106FA80026EE656A67EEE67AA3EE655AA3EE886A6E
:106FB800A6EEC47AE8EEA47A85ED0E5AC1ED205A01
:106FC80085ED0F6AC1ED406A85ED177AC5ED187A2F
:106FD800FEF798BD0546FFF7BEBA76EEC65AF0EE44
:106FE800466A3DE5744B4FEA88055FEA97082944ED
:106FF80003EBCC1C5D4437D008F101084FEA0818B0
:107008000CEB080E0CF1100301F1100005F1100251
:1070180013ED024A13ED035A13ED016A13ED047AD6
:1070280050ED024A50ED035A50ED016A50ED047AD2
:1070380064EE244A65EE255A66EE266A67EE277ADC
:1070480010339E4542ED024A42ED035A42ED016A71
:1070580042ED047A00F1100002F11002D8D1A8F133
:107068001008C4444144454417F003073EF4B8AF40
:10707800BCEC017AF1EC017A67EE277A013FE5EC86
:10708800017AF5D1FEF7ACBF4C4B1B88DC0541F10A
:1070980061804B4E4B4B96ED017A0F93D6ED006A0B
:1070A800D6ED027AB3F90670069BBDEEC77A198B46
:1070B800FDEEE66A17EE103AFDEEE77A16EE902A34
:1070C800ADF84A3017EE903AADF84820ADF84C309C
:1070D8003D4A3E4CB2F90230B2F900203C489FEDDF
:1070E8003D7AD0ED007A3C48DFF8FC8000780E90BD
:1070F8004FF47A7503F5E16305FB03F302F5E162EA
:1071080005FB02F284FB03651D44DB17C3EBE52393
:107118000F9D77EEC77A84FB02642E88FDEEE77A2E
:10712800761AA3F5FA731444ADF86030D21717EE47
:10713800903AADF850600F9EADF84E30C2EBE422A5
:1071480028462C466D88B3890089A4886D1AA2F553
:10715800FA725B1AADF86220ADF852507289F5895F
:10716800ADF85C30401A0E9BADF858007F1A00202D
:10717800641A521A691AADF85670ADF85440ADF851
:107188005A20ADF85E10C8F80000C8F80400C8F826
:107198000800C8F80C00002B01F040820F4B104E7D
:1071A800CDF840900F4D0A961F468146CDF844B061
:1071B80059E000BF1C330020B030002004490020F3
:1071C800D06200203C3C0020B4480020C5B3A29106
:1071D800403000200080BB44412F00202C1F00209D
:1071E80034370020442F0020303000201AAB03EB46
:1071F800440030F9200C38800A9B95F902E00E44CF
:107208001EFB00F053F82660012303FA04F4B64B82
:1072180083FB003EC0170C9B3442C0EB6E100CBFC2
:1072280001244FF0FF3498420EDB0D9B02FB03F262
:10723800AD4B83FB0263D217C2EB6313A3EB0C03C2
:107248001BB28342A8BF034638F8112003FB04236E
:1072580028F811300E9B09F10109994505F1070538
:1072680007F1020761DAA879002835D1297895F95C
:1072780005200D924E000A9A95F9043095F803E01E
:107288006C78701802EB8000C2888088121A92B25B
:10729800954802FB03F380FB03C0DB17C3EB6013C5
:1072A8004FEA520CA3EB0C031BB20C93BEF1000F78
:1072B8009CD01AAB03EB440BB7F900003BF920BC98
:1072C800584511DA8644704503DCF3455846A8BF93
:1072D800704600B238808FE71630C0B21CF044F90F
:1072E8000028C3D13880B5E786DDA0EB0E0EDE4559
:1072F80003DB7045A8BF704683460FFA8BF03880D1
:107308007AE77A4A1768B7F93240FEF709B828468B
:107318001546FFF72DBAB6EE007AF4EEC75AF1EE2D
:1073280010FA3FF7F0ABFCF79ABD0A9EDDF84090E3
:10733800DDF844B096F90A10B8F800306C486A4A8B
:10734800047811FB03F3F17A82FB0302FF294FEA69
:10735800E373C3EB621200F000848C4240F2FD83B9
:107368000F9B33F9111096F91600B8F80230114442
:10737800A8F800105C4AF17D10FB03F382FB0302BE
:10738800FF294FEAE373C3EB621200F0E3838C42F8
:1073980040F2E0830F9B33F9111096F92200B8F8F8
:1073A80004301144A8F802104F4A96F8231010FB35
:1073B80003F382FB0302FF294FEAE373C3EB621274
:1073C80000F0C5838C4240F2C2830F9B33F9111041
:1073D80096F92E00B8F806301144A8F80410424A6D
:1073E80096F82F1010FB03F382FB0302FF294FEAE4
:1073F800E373C3EB621200F0A7838C4240F2A483CC
:107408000F9B33F9111096F93A00B8F80830114477
:10741800A8F80610344A96F83B1010FB03F382FBD9
:107428000302FF294FEAE373C3EB621200F089837A
:107438008C4240F286830F9B33F9111096F946006F
:10744800B8F80A301144A8F80810274A96F84710E7
:1074580010FB03F382FB0302FF294FEAE373C3EB3C
:10746800621200F06B838C4240F268830F9B33F901
:10747800111096F95200B8F80C301144A8F80A1007
:10748800194A96F8531010FB03F382FB0302FF29F5
:107498004FEAE373C3EB621200F04D838C4240F273
:1074A8004A830F9B33F9111096F95E00B8F80E3035
:1074B8001144A8F80C100C4A96F85F1010FB03F35F
:1074C80082FB0302FF294FEAE373C3EB621300F068
:1074D8002F83A14280F02C830F9A32F91120134494
:1074E800A8F80E30FDF7E4BD1F85EB5108490020D0
:1074F800DC5B002090ED006A9DED124AE14925EE23
:10750800866AFDEEE43AA4EE076AB0EE674AA6EE94
:10751800264A13EE903AB4EEC45AF1EE10FAB0EEE1
:10752800446A88BFB0EE646ABDEEC66A16EE105AA9
:1075380016EE104AB542A8BF3446AB42C8BF1C4637
:1075480006EE104AB8EEC66A012A81ED006A3CF4DC
:10755800D8AD90ED046A9DED134A25EE866AA4EE37
:10756800076AB0EE674AA6EE264AB4EEC45AF1EEB0
:1075780010FAB0EE446A88BFB0EE646ABDEEC66A1F
:1075880016EE105A16EE104AB542A8BF34469D4270
:10759800B8BF1C4606EE104AB8EEC66A022A81ED4C
:1075A800016A3CF4AEAD90ED086A9DED144A25EEF3
:1075B800866AA4EE076AB0EE674AA6EE264AB4EEDB
:1075C800C45AF1EE10FAB0EE446A88BFB0EE646AAD
:1075D800BDEEC66A16EE105A16EE104AB542A8BF9E
:1075E80034469D42B8BF1C4606EE104AB8EEC66A3D
:1075F800032A81ED026A3CF484AD90ED0C6A9DED9E
:10760800154A25EE866AA4EE076AB0EE674AA6EE2A
:10761800264AB4EEC45AF1EE10FAB0EE446A88BFB6
:10762800B0EE646ABDEEC66A16EE105A16EE104A3F
:10763800B542A8BF34469D42B8BF1C4606EE104A64
:10764800B8EEC66A042A81ED036A3CF45AAD90ED9F
:10765800106A9DED164A25EE866AA4EE076AB0EE1A
:10766800674AA6EE264AB4EEC45AF1EE10FAB0EE16
:10767800446A88BFB0EE646ABDEEC66A16EE105A58
:1076880016EE104AB542A8BF34469D42B8BF1C4604
:1076980006EE104AB8EEC66A052A81ED046A3CF483
:1076A80030AD90ED146A9DED174A25EE866AA4EE7A
:1076B800076AB0EE674AA6EE264AB4EEC45AF1EE5F
:1076C80010FAB0EE446A88BFB0EE646ABDEEC66ACE
:1076D80016EE105A16EE104AB542A8BF34469D421F
:1076E800B8BF1C4606EE104AB8EEC66A062A81EDF7
:1076F800056A3CF406AD90ED186A9DED184A25EE32
:10770800866AA4EE076AB0EE674AA6EE264AB4EE89
:10771800C45AF1EE10FAB0EE446A88BFB0EE646A5B
:10772800BDEEC66A16EE105A16EE104AB542A8BF4C
:1077380034469D42B8BF1C4606EE104AB8EEC66AEB
:10774800072A81ED066A3CF4DCAC90ED1C6A9DEDDD
:10775800194A65EE865AE7EE045AE6EEA57AB4EEC3
:10776800E75AF1EE10FAC8BFF0EE647AFCF7B9BC3C
:1077780007EE904A9FED440AB8EEE78AFAF7C8FF89
:1077880020EE080AFEF753BF77EEC76AF0EE477A95
:10779800FEF756BABA8E9FED3D7A07EE902AF8EEBC
:1077A800E77A3B4A67EE877AC2ED007AFCF7F9BCC4
:1077B800B7EE007A77EE677AF4EEE75AF1EE10FA50
:1077C80088BFF0EE675AFFF7ABB901297FF744ABE2
:1077D80007EE10EAB8EEC77AC7EE876AB1EEE68A16
:1077E800FFF73CBB012940F3AC8607EE10EAB8EE80
:1077F800C77AC7EE876AB1EEE68A032C14D04FB178
:1078080007EE907AF8EEE77AF4EEC87AF1EE10FA1D
:1078180000F10787DAF8603003EB560393FBF6F3C1
:10782800CAF82030FFF7E2BAB0EE480A27F0CCFCDD
:1078380000B2E4E7012940F38B8607EE10EAB8EEC0
:10784800C77AC7EE876AB1EEE68A032C14D04FB127
:1078580007EE907AF8EEE77AF4EEC87AF1EE10FACD
:1078680000F1DF86DAF8643003EB560393FBF6F396
:10787800CAF82430FFF7D5BAB0EE480A27F0A4FCBE
:1078880000B2E4E74030002084F9223F6F12833AC7
:107898000000002090ED006A9DED124ABA4925EEDD
:1078A800866AFDEEE43AA4EE076AB0EE674AA6EEF1
:1078B800264A13EE904AB4EEC45AF1EE10FAB0EE2E
:1078C800446A88BFB0EE646ABDEEC66A16EE105A06
:1078D80016EE103AB542A8BF3346AC42C8BF23469D
:1078E80006EE103AB8EEC66A012A81ED006A3DF448
:1078F800C6AB90ED046A9DED134A25EE866AA4EEA8
:10790800076AB0EE674AA6EE264AB4EEC45AF1EE0C
:1079180010FAB0EE446A88BFB0EE646ABDEEC66A7B
:1079280016EE105A16EE103AB542A8BF3346A542D5
:10793800B8BF234606EE103AB8EEC66A022A81EDB1
:10794800016A3DF49CAB90ED086A9DED144A25EE62
:10795800866AA4EE076AB0EE674AA6EE264AB4EE37
:10796800C45AF1EE10FAB0EE446A88BFB0EE646A09
:10797800BDEEC66A16EE105A16EE103AB542A8BF0A
:107988003346A542B8BF234606EE103AB8EEC66A9B
:10799800032A81ED026A3DF472AB90ED0C6A9DED0D
:1079A800154A25EE866AA4EE076AB0EE674AA6EE87
:1079B800264AB4EEC45AF1EE10FAB0EE446A88BF13
:1079C800B0EE646ABDEEC66A16EE105A16EE103AAC
:1079D800B542A8BF3346A542B8BF234606EE103AC3
:1079E800B8EEC66A042A81ED036A3DF448AB90ED0F
:1079F800106A9DED164A25EE866AA4EE076AB0EE77
:107A0800674AA6EE264AB4EEC45AF1EE10FAB0EE72
:107A1800446A88BFB0EE646ABDEEC66A16EE105AB4
:107A280016EE103AB542A8BF3346A542B8BF234662
:107A380006EE103AB8EEC66A052A81ED046A3DF4EE
:107A48001EAB90ED146A9DED174A25EE866AA4EEEA
:107A5800076AB0EE674AA6EE264AB4EEC45AF1EEBB
:107A680010FAB0EE446A88BFB0EE646ABDEEC66A2A
:107A780016EE105A16EE103AB542A8BF3346A54284
:107A8800B8BF234606EE103AB8EEC66A062A81ED5C
:107A9800056A3DF4F4AA90ED186A9DED184A25EEA2
:107AA800866AA4EE076AB0EE674AA6EE264AB4EEE6
:107AB800C45AF1EE10FAB0EE446A88BFB0EE646AB8
:107AC800BDEEC66A16EE105A16EE103AB542A8BFB9
:107AD8003346A542B8BF234606EE103AB8EEC66A4A
:107AE800072A81ED066A3DF4CAAA90ED1C6A9DED4D
:107AF800194A65EE865AE7EE045AE6EEA57AB4EE20
:107B0800E75AF1EE10FAC8BFF0EE647AFDEEE77AB4
:107B180017EE903A9E42A8BF1E469C42D8BF3446F4
:107B280007EE904AF8EEE77AC1ED077AFDF7A4BAB6
:107B3800B6F95C20D3E4B6F95010B5E4B6F94410B0
:107B480097E4B6F9381079E4B6F92C105BE4B6F985
:107B580020103DE4B6F914101FE4B6F9081002E449
:107B68000A4EFCF77CBBDBF89421079B9A1AFEF7B8
:107B780084BF074BB8F90A201B68002B00F0598511
:107B88001A600120FEF7E7BD40300020D0620020D7
:107B98006C66002090ED006A9DED124A25EE866A1B
:107BA800A4EE076AB0EE674AA6EE264AB0EE446A2B
:107BB800B8F1000F00F06C83BEF1000F06D0B4EEF0
:107BC800445AF1EE10FAC8BFB0EE646AFDEEE44A1A
:107BD800BDEEC66A14EE904A16EE103A9C4214EEB8
:107BE800905A00F31785B342A8BF334606EE103A01
:107BF800B849B8EEC66A012A81ED006A3CF484AA45
:107C080090ED046ADDED134A25EE866AA4EE876AD4
:107C1800F0EE674AE6EE264AB0EE646ABEF1000F5F
:107C280000F0EE84B4EEE45AF1EE10FA40F3E88482
:107C38002346B342A8BF334606EE103AB8EEC66AEA
:107C4800022A81ED016A3CF45FAA90ED086ADDED35
:107C5800144A25EE866AA4EE876AF0EE674AE6EED5
:107C6800264AB0EE646ABEF1000F00F0BF84B4EE9D
:107C7800E45AF1EE10FA40F3B9842346B342A8BFA0
:107C8800334606EE103AB8EEC66A032A81ED026A58
:107C98003CF43AAA90ED0C6ADDED154A25EE866AA9
:107CA800A4EE876AF0EE674AE6EE264AB0EE646A0A
:107CB800BEF1000F00F09084B4EEE45AF1EE10FA31
:107CC80040F38A842346B342A8BF334606EE103AEF
:107CD800B8EEC66A042A81ED036A3CF415AA90ED51
:107CE800106ADDED164A25EE866AA4EE876AF0EE84
:107CF800674AE6EE264AB0EE646ABEF1000F00F06D
:107D08006184B4EEE45AF1EE10FA40F35B84234642
:107D1800B342A8BF334606EE103AB8EEC66A052A43
:107D280081ED046A3CF4F0A990ED146ADDED174A80
:107D380025EE866AA4EE876AF0EE674AE6EE264AE2
:107D4800B0EE646ABEF1000F00F03284B4EEE45A7B
:107D5800F1EE10FA40F32C842346B342A8BF334611
:107D680006EE103AB8EEC66A062A81ED056A3CF4BA
:107D7800CBA990ED186ADDED184A25EE866AA4EEC7
:107D8800876AF0EE674AE6EE264AB0EE646ABEF10C
:107D9800000F00F00384B4EEE45AF1EE10FA40F359
:107DA800FD832346B342A8BF334606EE103AB8EE29
:107DB800C66A072A81ED066A3CF4A6A990ED1C6AFA
:107DC800DDED194A65EE865AE4EE875AE5EEA67AA5
:107DD800BEF1000F00F0DA83F4EEC57AF1EE10FA86
:107DE80040F1D4832346B342A8BF33461D4607EE6D
:107DF800905AF8EEE77AC1ED077AFCF785B936496B
:107E080096F916700B8896F90A20B1F902003349E1
:107E180017FB03F3524200FB02F081FB03721211BD
:107E280081FB0071DB17C017C0EB2110991AD31A18
:107E380001440344691A1C44A8F80010A8F8024039
:107E4800FDF790B9DBF89421079B9A1AFDF705BF57
:107E580007EE904AB8EEE79ADFED217A8BF82042D8
:107E680029EE279AB0EE490AFAF73AFDFDEEC97AEB
:107E78001C4A17EE903A2033402BF0EE408A82EDF0
:107E8800010A00F26283B0EE490AFAF741FC8BED71
:107E9800890AFDF7A2BA96ED000A089327F094F92B
:107EA800114A1249D2F8EC20DFF844E081FB023194
:107EB800D217C2EBA11207EE902AF8EEE77AAEF8D5
:107EC8000000FDEEE77A089B17EE902AAEF8022034
:107ED800FCF7CAB940300020B44800201F85EB5198
:107EE80035FA8E3C00000020C4060020D34D6210F5
:107EF800D061002025EE866AA5EE076AB0EE675AC3
:107F0800A6EE265ABDEEC56A16EE101A8B4200F38D
:107F1800A681B142A8BF314606EE101AB8EEC66A6D
:107F2800BCF1000F00F05D84CE49012A81ED006AA2
:107F38003CF4EAA890ED046A9DED135A25EE866A92
:107F4800A5EE076AB0EE675AA6EE265ABDEEC56AD8
:107F580016EE104AA34200F37C81B442A8BF34460F
:107F680006EE104AB8EEC66ABCF1000F00F01084A5
:107F7800022A81ED016A3CF4C7A890ED086A9DEDDC
:107F8800145A25EE866AA5EE076AB0EE675AA6EE81
:107F9800265ABDEEC56A16EE104AA34200F35D816B
:107FA800B442A8BF344606EE104AB8EEC66ABCF121
:107FB800000F00F02184032A81ED026A3CF4A4A892
:107FC80090ED0C6A9DED155A25EE866AA5EE076AB6
:107FD800B0EE675AA6EE265ABDEEC56A16EE104AEE
:107FE800A34200F33881B442A8BF344606EE104AD3
:107FF800B8EEC66ABCF1000F00F0DF83042A81EDF9
:10800800036A3CF481A890ED106A9DED165A25EE9E
:10801800866AA5EE076AB0EE675AA6EE265ABDEE46
:10802800C56A16EE104AA34200F30F81B442A8BFF6
:10803800344606EE104AB8EEC66ABCF1000F00F0EE
:108048004A83052A81ED046A3CF45EA890ED146A1F
:108058009DED175A25EE866AA5EE076AB0EE675AB7
:10806800A6EE265ABDEEC56A16EE104AA34200F3E4
:10807800EA80B442A8BF344606EE104AB8EEC66A93
:10808800BCF1000F00F0A383062A81ED056A3CF4D9
:108098003BA890ED186A9DED185A25EE866AA5EE64
:1080A800076AB0EE675AA6EE265ABDEEC56A16EE06
:1080B800104AA34200F3CB80B442A8BF344606EE70
:1080C800104AB8EEC66ABCF1000F00F05183072AC7
:1080D80081ED066A3CF418A890ED1C6A9DED195ACA
:1080E80065EE865AE7EE055AE5EEA67AFDEEE77AE2
:1080F80017EE902A934204DCB24217EE903AA8BFDA
:10810800334607EE903AF8EEE77ABCF1000F7FF4B9
:1081180072AE0C9B002B7FF46EAE0A9B9D42B8BFDB
:10812800F0EE647A67E69FED500A504B25EE800A20
:108138001C4627F049F8E080DBF81441FCF713BB34
:108148004B494C4A8E46FDF73BBF079824F0F2F99D
:10815800FDF70BBD484B9FED496A93ED007A484BFC
:10816800D9F80010D3ED003A434BD3ED017A444BD4
:1081780093ED014A404BD3ED026A414BD3ED024ADD
:10818800404B37EE237A93ED005AD3ED015A77EE40
:10819800847A37EE057A77EEA57A76EEA46A27EE2A
:1081A800067A67EE867A66EE866ABDEEC77AFDEED7
:1081B800E77AFDEEE66A17EE100A17EE903ACDED73
:1081C8000A6ABDF92820ADF84800ADF84A30C8045D
:1081D8002D4BADF84C200F9300F1BE81069AB3F9F0
:1081E8000670118BFEF774BFDBF89421079B9A1A6F
:1081F800FEF743BA254B1B6813F0805C7EF483AC12
:10820800FEF779BC03F036FB0599184B0E780699F2
:108218002A78DBF81441401A9880FEF723B803F057
:1082280029FB059A114B1678069A801A5880FEF792
:108238006DB803F01FFB059A0C4B1678069A801A46
:108248005880FEF71FB81C4616E71C46F1E61C4688
:1082580035E71C4684E61C46C8E61C46A3E61946D4
:108268005AE600BF403000200000C842D06100201C
:10827800303200208C1D00200C3000203333333F77
:1082880018300020243000203C3C00201C710020C5
:10829800BEF1000F06D0B4EE445AF1EE10FAC8BF92
:1082A800B0EE646ABDEEE44ABDEEC66A14EE104A4A
:1082B80016EE103A9C4214EE107A00F3D181B342C4
:1082C800A8BF334606EE103AB8EEC66ABCF1000FF6
:1082D80000F0A782EF49012A81ED006A3BF414AF50
:1082E80090ED046A9DED134A25EE866AA4EE076AAE
:1082F800B0EE674AA6EE264AB0EE446ABEF1000F19
:1083080005D0B4EEC45AF1EE10FA00F39581BDEE33
:10831800C66A16EE103AA342B8BF234680F28D8192
:1083280006EE103AB8EEC66ABCF1000F00F0D08233
:10833800022A81ED016A3BF4E7AE90ED086A9DEDF3
:10834800144A25EE866AA4EE076AB0EE674AA6EEDE
:10835800264AB0EE446ABEF1000F05D0B4EEC45A06
:10836800F1EE10FA00F36D81BDEEC66A16EE103A12
:10837800A342B8BF234680F2658106EE103AB8EEF4
:10838800C66ABCF1000F00F09982032A81ED026AE7
:108398003BF4BAAE90ED0C6A9DED154A25EE866A5F
:1083A800A4EE076AB0EE674AA6EE264AB0EE446A23
:1083B800BEF1000F05D0B4EEC45AF1EE10FA00F386
:1083C8004581BDEEC66A16EE103AA342B8BF2346F1
:1083D80080F23D8106EE103AB8EEC66ABCF1000F95
:1083E80000F08082042A81ED036A3BF48DAE90EDA3
:1083F800106A9DED164A25EE866AA4EE076AB0EE6D
:10840800674AA6EE264AB0EE446ABEF1000F05D0D0
:10841800B4EEC45AF1EE10FA00F31D81BDEEC66A3F
:1084280016EE103AA342B8BF234680F2158106EE35
:10843800103AB8EEC66ABCF1000F00F0E881052AD0
:1084480081ED046A3BF460AE90ED146A9DED174A25
:1084580025EE866AA4EE076AB0EE674AA6EE264ABB
:10846800B0EE446ABEF1000F05D0B4EEC45AF1EE86
:1084780010FA00F3F880BDEEC66A16EE103AA34271
:10848800B8BF234680F2F08006EE103AB8EEC66A0E
:10849800BCF1000F00F08781062A81ED056A3BF4E4
:1084A80033AE90ED186A9DED184A25EE866AA4EE63
:1084B800076AB0EE674AA6EE264AB0EE446ABEF1F5
:1084C800000F05D0B4EEC45AF1EE10FA00F3D080D4
:1084D800BDEEC66A16EE103AA342B8BF234680F234
:1084E800C88006EE103AB8EEC66ABCF1000F00F07C
:1084F8000382072A81ED066A3BF406AE90ED1C6AFA
:108508009DED194A65EE865AE7EE045AE6EEA57A1D
:10851800BEF1000F40F0B180FDEEE77A17EE903A19
:108528009C4240F3B18007EE907AF8EEE77ABCF10E
:10853800000F7FF460ACECE5574F07F18003FDF7BF
:1085480079BE9FED568AFFF758B99FED540A9EE40D
:108558009FED528AFFF779B90699B3F90670098B2E
:108568008F42BCBF5242ADF84C20FEF7B1BD80200F
:1085780017F03EFD08B120F075F90DF0C1FBFDF7CD
:10858800F6BA052606220425FDF7E0BFFDEEE77AD8
:1085980017EE903AA342FFF62AAC24E4BDEEC66A71
:1085A80016EE103AA342BFF6FDAB2346FFF7FDBB1C
:1085B800BDEEC66A16EE103AA342BFF6CEAB23460E
:1085C800FFF7CEBBBDEEC66A16EE103AA342BFF661
:1085D8009FAB2346FFF79FBBBDEEC66A16EE103A67
:1085E800A342BFF670AB2346FFF770BBBDEEC66A69
:1085F80016EE103AA342BFF641AB2346FFF741BB44
:10860800BDEEC66A16EE103AA342BFF612AB234679
:10861800FFF712BB14EE903AFFF7E8BA204EFEF7C8
:1086280089BE069BAAF8A860D880DFF86CB0FCF772
:10863800B7BB0120FEF78FB82346B342A8BF334625
:108648006EE62346B342A8BF334696E62346B342B6
:10865800A8BF3346BEE62346B342A8BF3346E6E684
:1086680014EE103A2EE62346B342A8BF33460BE772
:108678002346B342A8BF334633E7B4EEE75AF1EED8
:1086880010FA7FF749AF2346B342A8BF33461F46C7
:1086980049E700BF403000208C1D0020000000008A
:1086A80034370020DFF8B082D8F8000020F0AEF8A8
:1086B800994B1B780022022BC8F800207EF404A9ED
:1086C80020F00EFBFEF700B99BF87031002B7BF40D
:1086D80041A9FBF72CB90C9C002C7FF4B2AC0A9C86
:1086E800A542B8BFB0EE646AABE48C4A8C4B106804
:1086F8001B6898478B4BD6ED006A93ED007A8A4B3E
:10870800D3ED007A894B83ED020A894B67EE277A0D
:10871800234427EEA87AD3ED007A864B67EE277AB2
:10872800F0EE665AE7EEAD5A93ED006AB1EE467A7E
:10873800F4EEC75AF1EE10FA08D4F4EEC65AF1EE88
:1087480010FA8CBFB0EE467AB0EE657A7A4B1B7899
:10875800012B02D0192B7BF471A8DFED787AF4EEA7
:10876800E7DAF1EE10FACCBF01230023FBF771B86A
:108778000C9C002C7FF4ABAC0A9CA542B8BFB0EEB1
:10878800646AA4E4FB5C002B7DF4F1A9FEF72BB925
:108798000C9C002C7FF4ECAB0A9CA542B8BFB0EE51
:1087A800646AFFF7E5BB0C9B002B7FF475AE0A9B50
:1087B8009D42B8BFB0EE646A6EE60C9C002C7FF454
:1087C8001DAC0A9CA542B8BFB0EE646A16E40C9CC6
:1087D800002C7FF459AC0A9CA542B8BFB0EE646A7D
:1087E80052E40C9900297FF49FAB0A998D42B8BFD7
:1087F800B0EE646AFFF798BB0C9C002C7FF4DBABEF
:108808000A9CA542B8BFB0EE646AFFF7D4BB0C9BC4
:10881800002B7FF414AE0A9B9D42B8BFB0EE646A89
:108828000DE60C9B002B7FF455AD0A9B9D42B8BF0B
:10883800B0EE646A4EE5132B05D1B0EE480A26F077
:10884800C3FC069B1880B0EE480ADAF808323C48A8
:108858009847059B1B78132BB0EE408A7CF4ACA894
:1088680026F0B2FC069B5880FCF7A6B8DFED357AF7
:10887800B4EEE7EAF1EE10FA4BDCDFED337AB4EE52
:10888800E7EAF1EE10FA44D4304AD2ED007AB1EEBC
:10889800677AF4EEC7DAF1EE10FA37D4F4EEE7DAD5
:1088A800F1EE10FA88BFF0EE67DA294A86ED00DAB1
:1088B80012689A42BAF6D6AEFAF7FEBE0C9B002BA7
:1088C8007FF463AD0A9B9D42B8BFB0EE646A5CE575
:1088D8000C9B002B7FF42CAD0A9B9D42B8BFB0EED9
:1088E800646A25E50C9B002B7FF47CAD0A9B9D42B6
:1088F800B8BFB0EE646A75E50C9B002B7FF4F9AD48
:108908000A9B9D42B8BFB0EE646AF2E5F0EE47DA22
:10891800CBE7DFED10DAC8E7603000200460002004
:1089280018600020585F0020000000200C30002054
:108938002860002090600020402F00200000964210
:10894800D86A002000C0F84400C0F8C48C60002039
:108958007060002000000000906F00202DE9F047B3
:10896800B0F908400C81E4B2442C8AB00D46174691
:1089780000F03284064642D9812C00F06F8300F261
:108988009480542C00F0C78040F2D1806E2C00F007
:10899800F183802C40F0CE80724B93F8009009F15F
:1089A800020919F0FF0900F093806F4B6F4F704E6A
:1089B800DFF8E4A1994403F101080A2416E0322CF7
:1089C80001F06482A4F13C00C0B2132841F268822D
:1089D80000232A68511C296014702A68C14502F1D5
:1089E80001012960137073D018F8014B0A2CE6D1E5
:1089F800BAF80030FF2BA8BFFF23DBB2E9E7052C4C
:108A080000F0D8831ED8022C7DD040F20783032CB7
:108A180000F0A783042C40F08D8056492846224652
:108A2800F9F738FD00212846F9F764FD2A68002186
:108A3800531C01242B602046234611706B810AB019
:108A4800BDE8F087242C5CD040F29E82282C00F0F0
:108A58004D83382C6ED10A68474B0124511C29607C
:108A680014702A6805211019286011702A680A21D3
:108A78001019286011702A680021101928601170D7
:108A88002A6819781019286011702A6859781019FD
:108A9800286011702A68997813192B602346117081
:108AA80020466B810AB0BDE8F087A02C17D040F2B1
:108AB8008A82B82C00F05383FE2C3BD12F4C04F152
:108AC800080634F8021B2846F9F714FDA642F8D127
:108AD8000124234620466B810AB0BDE8F087284B65
:108AE80008461968F9F7EEFC264B28461968F9F785
:108AF800E9FC254B196828460124F9F7E3FC2346CD
:108B0800E8E7224BF6E70422214928460124F9F731
:108B1800C1FC2346C4E70B6800215A1C2A6019705F
:108B28002A68012413192B6023461170B8E7522CC8
:108B38003FF47CAF2946204607F07EFB0028C7D1CA
:108B4800742C00F07E82772C28D1336872689A42A0
:108B58001BBF5A1C3260014619780E4A284620F07D
:108B6800FDFAB5E7AD61002008050308676666668B
:108B780050240020666300205B630020D061002041
:108B8800ACF7FF1FB0F7FF1FB4F7FF1FE06400202A
:108B98003C2903083983020878240020F52C00F0CA
:108BA8004783292C376801F0FD81392C01F0E881D1
:108BB800212C01F0A88172680B3CD31BEF2C00F22A
:108BC8002B8401A151F824F02F9900082194000862
:108BD8002194000821940008219400082194000899
:108BE8002194000821940008219400082194000889
:108BF8002194000821940008219400082194000879
:108C08002194000821940008219400082194000868
:108C18002194000821940008219400082194000858
:108C28002194000821940008D9980008219400088C
:108C380075980008219400085398000821940008AA
:108C48002194000821940008339A00082194000810
:108C5800BD990008219400088B9900082194000808
:108C6800659900082194000841980008219400089B
:108C7800ED97000821940008A197000821940008A6
:108C8800219400082194000821940008D98A00083A
:108C98002194000875970008219400082194000881
:108CA8007B9E000821940008E19D0008219400089B
:108CB80021940008219400082194000821940008B8
:108CC8002194000821940008219400083B9E000884
:108CD80021940008F19C00082194000821940008C0
:108CE800A39D0008219400082194000821940008FD
:108CF8002194000821940008219400082194000878
:108D08003F9D000821940008059B00082194000855
:108D18005B9A000821940008259C0008219400080B
:108D2800C19B0008A39B0008879B000821940008AA
:108D38002194000821940008219400082194000837
:108D48002194000821940008219400082194000827
:108D58002194000821940008219400082194000817
:108D68002194000821940008219400082194000807
:108D780021940008219400082194000821940008F7
:108D880021940008219400082194000821940008E7
:108D980021940008219400082194000821940008D7
:108DA80021940008219400082194000821940008C7
:108DB80021940008219400082194000821940008B7
:108DC80021940008219400082194000821940008A7
:108DD8002194000821940008219400082194000897
:108DE8002194000821940008219400082194000887
:108DF8002194000821940008219400082194000877
:108E08002194000821940008219400082194000866
:108E18002194000821940008219400082194000856
:108E28002194000821940008219400082194000846
:108E38002194000821940008219400082194000836
:108E48002194000821940008219400082194000826
:108E58002194000821940008219400082194000816
:108E68002194000821940008219400082194000806
:108E78002194000821940008C79C00082194000848
:108E88005F9700083597000821940008219400088E
:108E980021940008219400082194000821940008D6
:108EA80021940008219400082194000821940008C6
:108EB800219400082194000821940008D9960008FC
:108EC80021940008A196000821940008059600083E
:108ED800EB950008CF95000821940008B595000887
:108EE800219400088D95000821940008E594000855
:108EF80021940008B79400082194000821940008E0
:108F08009594000867940008539400082B9400086F
:108F180003940008E19300082194000821940008B4
:108F28002194000821940008219400082194000845
:108F38002194000821940008219400082194000835
:108F48002194000821940008219400082194000825
:108F58002194000821940008C79300082194000870
:108F6800219400086F9300082194000821940008B8
:108F7800219400080993000821940008219400080E
:108F880021940008EF920008202C7FF4D3AD0B68E1
:108F9800954C591C627829601A702B682278591CE4
:108FA80029601A702B68A278591C29601A702189C7
:108FB8002846F9F79FFA2B686279591C29601A70BC
:108FC8002A68A17934E5822C7FF4B4AD0B68874A0E
:108FD800874C1178844A581C2860197011892846D2
:108FE800F9F788FA834B2A681B88FF2B02F10101E5
:108FF800A8BFFF2329601370A16881F3100189B20B
:109008002846F9F777FA216801F30F0189B2284653
:10901800F9F770FA784B2A68197809E5012C7FF47A
:1090280089AD0B680022591C29601A702B685A1CDC
:109038002A601C702A682521531C2B602346117056
:109048002EE5336872689A421BBF5A1C326001468B
:1090580019786A4A284620F081F839E5684B1E7865
:10906800033616F0FF063FF433AD664B664F1E44D9
:1090780003F101094FF00A0820E0B8F1500F00F0A1
:109088000C87B8F1320F00F02187A8F13C00C0B27C
:10909800132840F21F87002421462B685A1C2A6097
:1090A800284683F80080F9F725FA21462846F9F77B
:1090B80021FA4E453FF40CAD19F8018BB8F10A0FAF
:1090C800DBD1524B9C68196804EB84044FF6FF739C
:1090D80064009C42A8BF1C469942A8BF194624EACE
:1090E800E47421EAE171A4B289B2D6E70B68DFF82B
:1090F8003C81474E591C022229601A702B680627AA
:109108005A1C2A601F702B680A22591C29601A7081
:109118002B6801241A192A601C70B8F80010284618
:10912800F9F7E8F9B8F802102846F9F7E3F92B68D7
:109138001A192A601F702B685022191929601A7091
:109148002B680022191929601A7031882846F9F706
:10915800D1F971882846F9F7CDF92346A0E42D4BBB
:10916800C8E40B685A1C0A601C700B685A1C0A6019
:109178001C705BE41F4B0A681B881D4CFF2BA8BFA3
:10918800FF23511C29601370A16881F3100189B273
:109198002846F9F7AFF9204B28461988F9F7AAF9B4
:1091A800216801F30F0189B228460124F9F7A2F9D1
:1091B800234675E40B2219492846F9F76BF908226A
:1091C80017492846F9F766F9012407221549284660
:1091D800F9F760F9234663E4002A3FF479AC124BAF
:1091E8001360012423465BE4A0480020CE620020DF
:1091F800E4460020B8620020EF3B002021840208EA
:10920800AD6100201805030848240020042400202C
:1092180038240020E0380020EC3B002044290308D3
:10922800502903085C29030815020108D82F0020DB
:10923800336872689A4240F0CF86BF4BFF221A709B
:109248004FF00009BD4C13F087FF49462022BC4867
:1092580084F8009026F075FF8DF804909DF804308E
:10926800072B00F21587DFF81083B54E4A469DF8A4
:10927800043003EB430308EBC3035B7CE3B19DF8C5
:10928800043003EB430308EBC30320215B699BB164
:109298009DF8043003EB430308EBC303586946F811
:1092A80022001CF013FA237856F823001CF056FA13
:1092B80022780132D2B222709DF804300133DBB239
:1092C8008DF804309DF80430072BD0D92B68591C31
:1092D80029601A70002F3FF4FBAB9A4B3B600124C6
:1092E8002346FFF7DDBB984B1B78DB0700F1948022
:1092F800012401F05BF901F001FA2346FFF7D0BB26
:109308003046F9F7B5F83368ADF804001A46591C29
:10931800316012F8021B32608DF806105A788DF809
:109328000720DA1C32609A788DF808201A1D3260FE
:10933800DA788DF809205A1D32601B798DF80A30C9
:1093480001A80023ADF80C30F8F7EAFF7F4A7A4B02
:109358001268801A4FF0010461F10001C3E90401A9
:109368002346FFF79DBB7B1C33603B780F2B53D8FC
:10937800BA1C3260C3EBC303754A7978D154F91C1F
:1093880031601344BA785A703A1D3260FA789A708C
:109398007A1D32603A79DA70BA1D32607A791A71B8
:1093A800FA1D3260BA795A7107F108023260FA7907
:1093B8009A71012418F0BEFF2346FFF771BB3046AF
:1093C800F9F756F8634FF8813046F9F751F8012458
:1093D800B8812346FFF764BB3046F9F749F85E4F7A
:1093E80038823046F9F744F878823046F9F740F881
:1093F8000124B8822346FFF753BB3B467A1C3260F0
:1094080013F8020B3360FB1C79783360BA7811F0DB
:1094180033FC00287FF45CAB4FF0FF342346FFF7A2
:109428003FBB3B467A1C32604C4A13F8021B117052
:109438003360484A7B789370FB1C3360484BBA789A
:109448009A7001242346FFF72BBB464B4649186800
:109458004E22012425F078FD2346FFF721BB3A462A
:109468007B1C3360414B12F8021B197032607A780A
:109478005A70FA1C3260BA789A703046F8F7F8FFDA
:109488003B4B0124D8802346FFF70ABB3046F8F748
:10949800EFFF374F38803046F8F7EAFF78803046DC
:1094A800F8F7E6FF0124B8802346FFF7F9BADFF89A
:1094B800CC8098F80030002B3FF40AAB2D4F0024E5
:1094C8003046F8F7D5FF19F0BDFA98F80030A7EC48
:1094D800010A01349C42F3DBFFF7FABA0D2B9BD14A
:1094E8007B1C33603C78072C96D8DFF89480304694
:1094F8000C27F8F7BDFF07FB04F708EB0704A0806B
:109508003046F8F7B5FFE0803046F8F7B1FF33682A
:1095180020811A46591C316012F8021BA172326070
:109528005B78E3723046F8F78BFF012448F80700B0
:109538002346FFF7B5BA00BFC01F00201B3A002022
:10954800F05C002039950108186F0020BC710020DC
:10955800F4370020E82F0020CC4B0020446B00207B
:10956800F82F002008490020D0210308E02F002010
:1095780020610020F02C00200C4B0020AD61002061
:10958800343700207B1C33603878060600F1838569
:10959800BD4B1B78DC073FF59BAA032828BF00209A
:1095A800012400F0E7FF2346FFF77ABAB64B1B7891
:1095B800D8073FF58DAA012401F046FC01F09EF87A
:1095C8002346FFF76DBAB04B1B78DA073FF580AA40
:1095D800AE4A1378012443F0040313702346FFF7BF
:1095E8005FBAA94B1B78D9073FF572AAA84B4FF46D
:1095F800C87201241A802346FFF752BA092B7FF755
:109608000BAFDFF8C8823B467A1CD8F800403260BE
:1096180013F8022B227033607B78A370FB1C336035
:10962800BB78642BA8BF64233A1D63713260FB7852
:10963800642BA8BF64237A1DA37132603B79E37160
:10964800BB1D33607B79642BA8BF6423FA1D23728A
:109658003260BB79E37007F108033360FB7923714B
:109668003046F8F705FF726833686081D11A00291F
:109678000CDD591CD8F800003160521A002A1978FC
:10968800417203DD9A1C32605B784370012419F043
:10969800CFFF2346FFF704BA7E4B1868FB1C02462F
:1096A8002137991E316013F8031C1170591E31605F
:1096B80013F8021C5170336013F8011C91700333C6
:1096C8009F4202F10302ECD119F05AF8FFF700BAF1
:1096D800C3F34704122C3FF69FAEBCB10AAB0DF1A1
:1096E800020803EB44094746A9F126093046F8F772
:1096F800BFFE27F8020F4F45F8D1674B38F8022F05
:1097080023F8022F4745F9D1112C09D8634A630081
:10971800023B13440021223223F8021F9A42FBD154
:109728005F4A01231C461370FFF7BAB97B1C5D49D9
:1097380033600A783B78002A40F0C18404220A701A
:10974800594A9B00138002F095F8584B0124986100
:109758002346FFF7A5B9564F002330463B60F8F77C
:109768006FFE012438602346FFF79AB93B46791CFF
:109778003160504913F8020B88703360787848706C
:1097880093423FF4A5A9FB1C3360484BBA781A7280
:1097980001242346FFF784B90722B3FBF2F2C2EB98
:1097A800C2041B1B7FF438AED2B202F1FF385FFA55
:1097B80088F8002A3FF48CA9DFF8FC9008F101082A
:1097C8001C467B1C33603C4B97F90010002793F92B
:1097D80002208A4203F1080300F035840137062F7E
:1097E800F5D119E67B1C33603B780E2B3FF614AE9F
:1097F800BA1C3260787803283FF60EAE2F4906224D
:1098080002FB03F28B18FC1C58713460B87888543A
:109818003A1D3260FA785A707A1D32603A799A7035
:10982800BA1D32607A79DA70FA1D3260BA791A7123
:1098380001242346FFF734B97B1C3360204B3A7868
:109848005A7501242346FFF72BB93046F8F710FE66
:109858001C4F38603046F8F70BFE78603046F8F752
:1098680007FE0124B8602346FFF71AB9164F0023F4
:109878003B603046F8F7E4FD3B68012403433B6056
:109888002346FFF70DB900BF186F0020883000206D
:109898002E72002008490020F25B0020F45B0020B3
:1098A800185C0020E6350020EC3B0020C01F00209B
:1098B800E03800200830002050710020EC380020EB
:1098C80024710020882C0020E06400200C4900202E
:1098D8007B1C33603C78132C3FF69EADBB1C336079
:1098E80078781FF075FC00283FF496ADBC4B0278E1
:1098F80003F82420FA1C326003EB8403BA785A7008
:109908003A1D3260FA789A707A1D32603A79DA70C4
:10991800002019F0CDFDB34B80F001000124187030
:109928002346FFF7BDB8B049102B4FF0000228BFFF
:1099380010230A604A608A60CA600A74002B3FF4E8
:10994800C7A83268013913440132326012F8010C99
:1099580001F8010F9342F7D1FFF7BAB87A1C3260C9
:109968003C781F2C3FF658AD052B7FF455AD30469B
:10997800F8F766FD9D4B43F8240011F0EFF9FFF767
:10998800A7B89A4C04F140073046F8F771FD3368E0
:10999800A4F88000591C1A46316012F8021B84F89A
:1099A800821032605B7884F883300434BC42EBD197
:1099B800FFF78EB87B1C8E4C33603B7823723046A1
:1099C800F8F756FDA0833046F8F752FD208330465D
:1099D800F8F74EFD32686083531C33601278E274E6
:1099E8007268D31A032B00F36F833368D11A0529E1
:1099F8000EDD5A1C32601B78E3723046F8F720FD02
:109A08003368E0605A1C32601B78237433687268CC
:109A1800D21A002A7FF75CA85A1C32601B7884F897
:109A2800213001242346FFF73BB87B1C3360714982
:109A380038780870D21A002A7FF74AA8BB1C33600E
:109A48007B78003318BF012301244B702346FFF7AE
:109A580027B87B1C3360684CDFF8BC813B7888F8FA
:109A6800053030462768F8F703FD38843046276804
:109A7800F8F7FEFC72683368F883D11A072915DDF8
:109A88003046F8F7F5FCA8F80A003046F8F7F0FC7D
:109A9800A8F80C0030462768F8F7EAFC78843046C6
:109AA8002768F8F7E5FC33687268B884D11A032987
:109AB8000BDD3046F8F7DCFCA8F80E003046F8F766
:109AC800D7FC33687268A8F81000D21A002A05DD9E
:109AD800591C226831601B7882F8263000F070FD2E
:109AE8001DF036FE454B1B68002B00F00C832068E8
:109AF800012418F06BFC2346FEF7D2BF3B467A1CC4
:109B08003260DFF8148113F8022B88F802203360E2
:109B18003B4A7B781370FB1C33603A4CBB7823714B
:109B28003B1D3360FB78092BA8BF09233046A3707F
:109B3800F8F79EFC336872682080D11A012905DD88
:109B48003046F8F795FC33687268E0819A4207D08E
:109B58005A1C32601B78003318BF012388F807307D
:109B680000F02EFD336872689A423EF4B1AF5A1C79
:109B780032601B78E37001242346FEF791BF7B1CFB
:109B880033603B78002B00F091824FF400400124B1
:109B980023F0D6FF2346FEF783BF1B4B1B7813F039
:109BA80001017FF439AC7B1C33603878012407F05D
:109BB800F9FE2346FEF774BF3B467A1C3260134A0F
:109BC80013F8021BD1703360114A7B785371FB1C68
:109BD8003360104BBA78DA7001242346FEF760BF71
:109BE800705D00207C1B0020C42F0020683A0020F4
:109BF800247100207C3000200849002064300020B7
:109C0800DC2F0020CC4B0020186F0020E82F00200C
:109C18009C4A0020F82F0020446B00203046F8F7BB
:109C280027FC3046F8F724FC3046F8F721FC30468C
:109C3800F8F72AFC3368C44C1946581C226830606F
:109C480011F8020B82F82C003160597882F836102E
:109C5800D91C31609B7882F837303046F8F714FC0D
:109C68003046F8F711FC3046F8F70EFC3046276806
:109C7800F8F7FEFB788730462768F8F7F9FB336872
:109C880072683887D11A01290ADD591C22683160A7
:109C98001B7882F82E303046F8F7F6FB3368726886
:109CA800D31A032B09DD30462768F8F7E1FB7886DD
:109CB80030462668F8F7DCFBB086206804E53B46AA
:109CC8007A1C326013F8024B3360FB1C78783360DF
:109CD800B978002C00F03C82012C7EF4F9AE07F034
:109CE8001FFF2346FEF7DCBE7B1C336097F800801D
:109CF800B8F1110F3FF690ABBB1C3360934C7B78E7
:109D080004F818303046F8F7B3FB40F6CA03984217
:109D1800A8BF184640F2EE23984204EB4801B8BFAA
:109D280018460124A0F2EE222346192092FBF0F2F5
:109D38004A70FEF7B5BE864B1B68002B3EF4C8AED2
:109D480012F0CCF8FF283EF4C3AE3046F8F790FB8B
:109D58003F2840F2F0817F4F00243C7033687268DE
:109D6800B880D21A012A7EF7B3AE1A46591C316060
:109D780012F8021BB9700AA8326000225C7800F859
:109D8800242D12F07DF89DF80430A3423EF4A0AED5
:109D9800204612F099F8FEF79BBE6F4B1B78012BFB
:109DA8003EF696AE7B1C39463360DFF8CC8111F85D
:109DB800023B88F80230FB1CD21A3160012A7878FD
:109DC800336040F3AB813046F8F752FB0124A8F822
:109DD80000002346FEF764BE7B1C33605F4B3A7875
:109DE800DFF898811A700023C8F800303046F8F779
:109DF80027FB3268D8F8003059495A4C0343501CA5
:109E0800C8F80030306013780B723046F8F730FB32
:109E180020603046F8F72CFB60603046F8F728FBE6
:109E2800A0603046F8F724FB3046F8F721FBFEF730
:109E38004FBE3B467A1C4C4C326013F8022B227101
:109E480033607B7863713046F8F712FB3368208003
:109E58005A1C32601B78A3713046F8F709FB336847
:109E680060805A1C32601B78E37101242346FEF798
:109E780017BE3E4B07F108010137376017F8012C70
:109E880003F8012FB942F7D1FEF722BE3388FF2B22
:109E9800A8BFFF23DBB2FEF79CBD354BFFF712B915
:109EA8001AF0D8FC00283EF493AD03780A2B28D882
:109EB800B0F9023087FB0312DB17C3EBA2039BB296
:109EC800FF2BA8BFFF23DBB2FEF783BD97E8120084
:109ED800FFF7FAB81AF0BEFC00283FF4DCA80378B4
:109EE8000A2B3FF6D8A8B0F90430B0F9061003EBF6
:109EF800830383F3500421EAE171A4B289B2FFF726
:109F0800CCB80023DFE73B467A1C3260194C13F8C3
:109F1800022B627033607B782370FB1C3360BB7844
:109F2800A3703046F8F7A4FA33682081591C1A4602
:109F3800316012F8021B617132605B78A3710124F1
:109F48002346FEF7ADBD00BF08490020805E002013
:109F58001C6F0020206F0020BC6400207C30002093
:109F680024710020882C00203861002023710020F3
:109F78003C240020A0480020BE640020E0640020AB
:109F88007B1C33603B780A2B4ED03046F8F77CFABE
:109F98003046F8F779FA01243046F8F775FA23467F
:109FA800FEF77EBD7B1C33603B780A2B0FD0502B0D
:109FB8007FF437AF3046F8F75BFA684F38803046A1
:109FC800F8F756FA012478802346FEF769BD304633
:109FD800F8F74EFA624FF1E75A1C194632606148A9
:109FE80011F8022B027031605B784370042A04D99F
:109FF800FF2A7EF41BADFFF723B95B490978994224
:10A0080005D8022A7EF412ADFF2B7EF40FAD2B6823
:10A0180001241A192A601C70002F3EF459AD534BC5
:10A028003B602346FEF73CBDBB1C3360504B7A783F
:10A038001A70FA1C3260BA785A703A1D3260FA788F
:10A048009A70FEF745BD09EBC70A30468AF8021038
:10A05800F8F70EFA336829F837001A46591C3160A8
:10A0680012F8021B8AF8031032605A788AF8042022
:10A07800DA1C32609A788AF806201F1D376001348E
:10A08800DB788AF80530A0457FF49BABFEF720BD4E
:10A098004A46FFF71BB900F07F00032828BF0020BD
:10A0A800012407F059FD2346FEF7FABC314A13682C
:10A0B800012423F4004313602346FEF7F1BC042A6D
:10A0C8007EF406ADFFF73CBB3046F8F7D1F9A08423
:10A0D8003046F8F7CDF933687268E084D11A03295D
:10A0E8007FF784AC1A46591C316012F8021BA1771D
:10A0F80032605B7884F820303046F8F7B9F9336875
:10A108007268608472E41C481C491D4A1D4B036038
:10A1180001240B6013602346FEF7C2BC1A4BB978C2
:10A128001A88012412FB00F2234692FBF1F2A8F8E8
:10A138000020FEF7B5BCC40800F007030134013362
:10A14800E4B2124F204619467B701AF0EDFA04E685
:10A15800012418F0F9FA2346FEF7A2BC382400209F
:10A16800D82F0020C01F0020AD6100202D0201085B
:10A178005B630020004900205C5F0020B05F002086
:10A1880018600020F5030008A86F0020206F002049
:10A1980038B50B4C23688BB15A68821A002A0546D9
:10A1A80004DA0CE05A68AA1A002A07DB9A682260C7
:10A1B80018461A6890472368002BF3D138BD38BD7C
:10A1C800783600200B4B002210B4027203F1DC0435
:10A1D800012102E0072A09DC9979890702D5197952
:10A1E800815401329C4203F11403F3D15DF8044B0E
:10A1F800704700BF3827030818230370704700BF53
:10A2080030B4012330253324312132224570C47102
:10A218004171C2700372037083710371837030BC23
:10A22800704700BF2DE9F0478C4B1B78DB070746CA
:10A2380044D58B4B8B4D1C788B4E012C59D01CD39D
:10A24800022C07D189498A4A09881288914201D982
:10A2580001241C70EB7AE3B12B89D3B1854B1B78B1
:10A26800BBB107F09BFC002800F09B802B7B83424E
:10A278002CBF0121002131700CE07C497E4A0988FD
:10A2880010886A7B801A8842E2DAEB7A0024002B75
:10A29800E2D131782A79632A06D8022C774E00F069
:10A2A800BA803378002B5DD1754AAB7A8C4238BFBF
:10A2B8000C461470002B4CD1BDE8F0876B4B694DF0
:10A2C80019885B88E878CB1A83EAE3728142A2EBAB
:10A2D800E3721DD32B788B421AD3614B1C78E01E96
:10A2E800012861D96749097802294FD0012C5E4EAF
:10A2F800A5D15F4A5D491288687B0988121A914284
:10A3080039DD5D4A12888A42A4D200241C70A1E774
:10A31800B1EB400FE1DC524B1C78E11E012940F201
:10A328009480022ADEDC57494F4E0878DFF84481D2
:10A33800DFF844C1DFF838E1002103240228347033
:10A348001C7088F80010ACF80010AEF8001081D12D
:10A358001FE0012C71D0022C0BD10720BDE8F0477B
:10A368001EF07CBD7068381A474B984258DD7270F1
:10A378009AE7BDE8F08702241C706BE7022AD2DD59
:10A388004049097802294FF0040464D13949364E0E
:10A3980009783E48022ACCBF00220122C28081806F
:10A3A8004BE70221317075E7022A9BDC95F800C063
:10A3B80091FBFCFC0CF1010CBCF1080FDFF8B4A018
:10A3C800304EA87895F801E096F800802A4CDFF81E
:10A3D800A090254EA8BF4FF0080C8AF800C01FFABD
:10A3E8008CFA10FB0AF01EFB0AFE80B2DFF88CA084
:10A3F8002080A9F800E000244FF0640EB8F1020FA5
:10A4080034701C70CAF804408AF801E07FF439AF50
:10A418000FFA8CF1BDE73078A0B90123776033706B
:10A42800C2F164021A4B00FB02F083FB0023C01741
:10A43800A0EBA3506430707036E70820BDE8F04701
:10A448001EF00CBD7368F81A8EE7032C96D10D49DF
:10A45800097802299AD0044EFCE600BF186F002044
:10A46800A0240020A0480020B0240020B8620020CA
:10A47800A4240020CE620020A2240020A8240020CA
:10A48800EF3B0020CC6100207F969800D06100202F
:10A498006BCA5F6B2DE9F0470569C3681D4028D07A
:10A4A8000F4606464FF000484FF00009B5FA85F30D
:10A4B80028FA03F2D2431B3B32611540042B16D80D
:10A4C800DFE803F03129211903007B6A002B32D021
:10A4D80003F1FF3A1FFA8AFAC7F824903C6A34B1AC
:10A4E80023682046514698476468002CF8D1002D0F
:10A4F800DCD1BDE8F0873868716B036889B298478A
:10A50800002DD3D1F5E77868B16B036889B2984715
:10A51800002DCBD1EDE7B868F16B036889B2984795
:10A52800002DC3D1E5E7F868316C036889B2984714
:10A53800002DBBD1DDE7F36A1FFA83FACEE700BF2F
:10A5480008B5012102201BF019F9094B1B7803F00B
:10A558000503052B08D0002101201BF00FF900216D
:10A5680008461BF00BF9FEE718F080FBF3E700BF85
:10A57800602C0020022828BF022010B4084C094B88
:10A58800207000EB8002C0EBC20207495DF8044B63
:10A59800013003EB4203C0B20B601EF031BD00BFB7
:10A5A800606300207A6300200849002008B516F08F
:10A5B80017FBF7F7DBFBBDE8084016F0F9BA00BF58
:10A5C80038B5434B5A899989914224BF00225A8150
:10A5D800198ADA89914224BF0022DA81DA788AB3AB
:10A5E800072A2FD03B493C4D91F853000124002104
:10A5F8000A282C709C70D9713DD00C2865D0DFEDED
:10A60800377A8ABB364C9FED370AA278002918BFE3
:10A61800F0EE407A062A04D8334901EB820191ED25
:10A62800000A217959B3013A032A4DD8F7EE007A86
:10A6380087EE800A24F0C8FD2388984228BF184670
:10A64800208038BDD97921B198780428B8BF042072
:10A658009870204890F853000A280CD00C28CED1C6
:10A66800DFED227A002ACDD0072ACBD00A282CD1B8
:10A67800DFED1F7AC6E70A20DFED1E7AC1E79B7877
:10A68800154A07EE103A1178B8EEC77A27EE277AFE
:10A6980007EE901AF8EEE77A67EE877AB4EEE70AE3
:10A6A800F1EE10FA10DDC0EE077AFDEEE77A17EE4C
:10A6B800903A102BA8BF1023012BB8BF0123DBB29F
:10A6C8008B4238BF0B46137038BDDFED0B7A99E724
:10A6D800446B0020CC680020DC2F00206F12033967
:10A6E800CC4B00206F120338280503080AD7A3397A
:10A6F8000F506E3A5304E9386F12833A2DE9F04748
:10A70800AA4FAB4E16F06CFABE421ED2DFF81C837D
:10A71800DFF81C934446258862197DB14A450DD25D
:10A72800052D0BD933886188C3F30B03994200F0D8
:10A73800E280144625886219002DEFD171683046F1
:10A7480014361BF026FABE42E4D39A4A1378A3F1D2
:10A75800170102290FD9984911F83300002840F051
:10A76800F680D8000144497829B1944911F833306A
:10A77800002B00F01481924B5A78022A40F2E180B3
:10A78800002290495A701A788F48022A016000F214
:10A79800D48002EB82018D4BC2EBC10203EB420372
:10A7A800998C5A8C8A4C9142236001D300225A8496
:10A7B800884B9A78042A00F0E98032B91A88B2F5F1
:10A7C800F07F84BF4FF4F0721A80834DFFF7F8FED4
:10A7D8002B68824A1A40002A00F0E480D80700F16A
:10A7E800D080590400F1C8801A0700F1C0809B048A
:10A7F80000F1B68022F092FA10B979481DF09EFD5A
:10A8080080201BF0FDF94FF400701BF0F9F94FF4AC
:10A8180000301BF0F5F94FF480201BF0F1F94FF4EC
:10A8280000101BF0EDF94FF000701BF0E9F94FF044
:10A8380080601BF0E5F918F0FBFE00213022694822
:10A8480025F07FFC206818F0CBF8674B276803F1E8
:10A85800500102E0043399426DD01A78002AF9D1E8
:10A868009C78D8788442F5D26049614B0D7961496A
:10A8780061480A70614E624C0460C822642111FB71
:10A888000521002259609A60DA601A615A619A615A
:10A89800DA6183F8202083F8212037600DF08EFEDE
:10A8A800584B9FED595A1B88584A9FED596A507961
:10A8B800584906EE903AF8EEE66A1388C5EE265A2D
:10A8C80007EE103A53881279C1ED005A07EE903A14
:10A8D800B8EEC77A504BF8EEE77A18725A7227EE3C
:10A8E800067A67EE867ABDE8F04783ED017AC3ED14
:10A8F800007A16F05DB963799B077FF41AAF716827
:10A9080094F804A030461BF044F93388BAEB133F9F
:10A9180004D01436BE42FFF4FDAE16E773887068A3
:10A92800AA1FC3F30B039A4204F10601A8BF1A46F3
:10A9380024F00AFBEDE7012296E700221A70234B68
:10A948002EE7204902EB420201EB82011BE7D80007
:10A958000C186468002C7FF405AF1724147001E705
:10A968002E481BF04DF940201BF04AF942E72C48CD
:10A978001BF046F92B683AE72A481BF041F92B6887
:10A9880032E729481BF03CF92B682AE79A8AB2F586
:10A998007A7FBFF41AAF4FF47A729A8215E71823B8
:10A9A8001370E8E643F008032B6017E78C5A030896
:10A9B800685603087C300020C41E030844140308AA
:10A9C80060630020866400200C4900207A63002020
:10A9D80008490020CC4B0020E064002009600002F8
:10A9E80050710020FC200020705D0020386100209C
:10A9F800F43B00207C1B0020E81F002030210020B1
:10AA0800EE2F0020501F0020C0C9FB48C41F0020A3
:10AA180017B7D138541F00203C5F002009400002BE
:10AA280001600002092000020860000202F0030829
:10AA38000000040808B516F0D3F8F7F797F916F0F0
:10AA4800B7F8FFF75BFE0120BDE808401EF0D8BA52
:10AA58002DE9F047B24C636820469847002800F07B
:10AA6800C180B04B1B780122042B84F83C2000F0F5
:10AA7800BB80B4F91610B4F91820B4F91A30216360
:10AA88006263A363A84B1B88002B69D0A74DD4ED44
:10AA98000C7AD5ED004A95ED050A95ED015A95ED2C
:10AAA800067AD5ED035A95ED026AF8EEE76AD5ED18
:10AAB800047AA4EEA60AA5EE267A67EEC07AA5EE79
:10AAC800C07AE6EE267A85ED057AC5ED067A24F099
:10AAD8007BFBD4ED0D6AD5ED094A95ED0E0A95ED8F
:10AAE8000A5A95ED0F7AD5ED0D7AD5ED0C5A95EDFC
:10AAF8000B6A2063F8EEE66AA4EEA60AA5EE267AAB
:10AB080067EEC07AA5EEC07AE6EE267A85ED0E7A73
:10AB1800C5ED0F7A24F058FBD4ED0E6AD5ED124A34
:10AB280095ED170A95ED135A95ED187AD5ED167A25
:10AB3800D5ED155A95ED146A6063F8EEE66AA6EE4F
:10AB4800A40AA6EE857A67EEC07AA0EE657AE6EEEC
:10AB5800867A85ED177AC5ED187A24F035FBA0635F
:10AB6800734FA17F73480DF0ABFC3B88002B7DD160
:10AB7800714E3568714B1B685B0743D4B5F900709B
:10AB8800216B636BA06B6E4A6E4E92ED026AD2ED3A
:10AB9800006AD2ED015AC91B2163B5F90270DB1BAB
:10ABA8006363B5F904703568C01B07EE900AB8EE08
:10ABB800E75A07EE901AB8EEE77A07EE903AF8EE01
:10ABC800E77A36EE056A36EE877A77EEA57A0135AA
:10ABD800A06382ED026A82ED007AC2ED017A3560E7
:10ABE800BDE8F087BDE8F087574BB4F91600B4F913
:10ABF8001810B4F91A2018802063598061639A806C
:10AC0800A2633FE7514F3B88322B79D0002B5BD1B1
:10AC18004F480378002BB1D0DFF83CE1F169326A84
:10AC28008EFB01730027C9170770C1EB23118EFB38
:10AC38000203D217C2EB2312736A29806A80A08AA2
:10AC480044498EFB03E2DB17C3EB22131B1AAB80CC
:10AC5800CF6015F0C5FFF7F789F815F0A9FFFFF7E2
:10AC68004DFD01201EF0CCF9356887E7324E226B86
:10AC78003568B3F5C87F4FF0000323632B8039880C
:10AC880018BF7068B7F8008008BF0020B1F5C87F0A
:10AC980018BFB368616B02440B440020B8F5C87F45
:10ACA80060637260B360688035D0D4F838E0F168CA
:10ACB800A0637144B8F1010FA880F1604ED008F18B
:10ACC800FF38A7F8008055E7F169226B0020206360
:10ACD80028803B880A44322B616BF261606368808C
:10ACE80068D0326AD4F838E0A0631144726A3162DD
:10ACF8007244012BA880726262D0013B3B8087E7D7
:10AD0800144B2988D8686A88AB883182B06172820E
:10AD1800B3820021D9E7A36BF360A063A880CEE7D4
:10AD2800BC480020CC610020B8360020BC3600208A
:10AD38002E720020EC480020E81F0020686B0020DD
:10AD4800305F00202C5F0020D0610020F820002018
:10AD5800F5200020E82F00201F85EB51DFF894C074
:10AD6800DFF88CE0C8328CFB02A9C833D217C2EBDB
:10AD7800E9128CFB03A9DB17C3EBE913C8316B801D
:10AD88002A808CFB013CA28ACB17C3EBEC139B1ADD
:10AD9800AB80CEF80C0015F023FFF6F7E7FF15F0AF
:10ADA80007FFFFF7ABFC40461EF02AF9B7F8008012
:10ADB800356884E7A26B3162A0637262A8809CE761
:10ADC80009490A4A08700B2013701EF047F83568C5
:10ADD800338A718A064A2B806980B08AB169A88053
:10ADE8003B88D16089E700BFFA200020F4200020CA
:10ADF800E82F00201F85EB5138B50C4C0C4DAC42A8
:10AE080006D26168204614341AF0C3FEAC42F8D367
:10AE1800084A094B094C1460002209491A705A70F3
:10AE280008480860BDE838400FF098BF6856030826
:10AE38008C5A030808490020606300207A630020C8
:10AE48000C4900208664002008B5FFF7D5FF15F0EF
:10AE5800C7FEF6F78BFFBDE8084015F0A9BE00BF96
:10AE6800F0B50C292BD8DFE801F06F2A2A2A4C2AE2
:10AE78002A2A2B2A2A2A0700046AB2F80CE09788A3
:10AE88001668674D24F480540462036A4468C169F3
:10AE980023F4005343EA0E3321F4E641A84243EA7F
:10AEA800073341EA062100F0B58005F50065A842A0
:10AEB80000F0B08092684460C16102640362F0BD32
:10AEC800046A96899588D2F800E0554F24F4807476
:10AED8000462036A4468C16923F4007343EA0623E1
:10AEE80021F07301B84243EA052341EA0E017ED0FE
:10AEF8004C4DA8427BD092684460C161C263036232
:10AF0800F0BD046A96899588D2F800E0444F24F091
:10AF180010040462036A4468816923F0200321F065
:10AF2800807143EA061321F4E641B84243EA051367
:10AF380041EA0E2148D03B4DA84245D09268446072
:10AF4800816182630362F0BD046A9389B2F804E008
:10AF58001768334E24F001040462056A4468816965
:10AF680043EA0E0321F4803125F002059BB221F05B
:10AF78007301B04243EA050341EA070114D0294DA1
:10AF8800A84211D005F54065A8420DD005F58065A9
:10AF9800A84209D005F58065A84205D092684460AA
:10AFA800816142630362F0BDD689158A578A23F00E
:10AFB800080333433D43D68824F4407423F0040344
:10AFC800ADB233432C43E9E7D589178AD68823F0F5
:10AFD800800343EA051324F44064558A23F04003B0
:10AFE80044EA870443EA061344EA8504A6E7D589B8
:10AFF800178AD68823F4006343EA052324F44054CF
:10B00800558A23F4806344EA071443EA062344EA92
:10B01800051470E7158A24F4804444EA851449E746
:10B02800002C0140003401402DE9F04FC8220021D6
:10B0380083B07848784CDFF80492784D784E794F91
:10B04800DFF8FC8125F07DF877487849DFF8F4E1EE
:10B05800DFF8F4C100221359834200F0C180B3F134
:10B06800804F00F0BF80AB4200F0C880B34200F0D0
:10B07800C780BB4200F0C680734500F0C5806345B9
:10B0880000F0C480434500F0C380DFF8C0A15345F9
:10B098007ED00AF5806A534508BF092379D0143257
:10B0A800F02AD8D15C4C624D624E604F04F1F00832
:10B0B80002E01434A04568D0A379002BF9D0237995
:10B0C8004FEA131909F1FF39B9F1050F03F00F031E
:10B0D800EFD835F8190040FA03F2D207E9D54FF056
:10B0E800010A0AFA03F3013B184023F0B9FC16F8E9
:10B0F80009305149184411EBC002DAD051F8300038
:10B10800DFF84CE1217A00F138439B0A1EF803303E
:10B1180003F01F0E5B09022B0AFA0EFA69D0032B03
:10B1280062D0012B03D17B694AEA03037B619388D0
:10B138000093B3FA83F3C3F11F039BB2DA0800EB61
:10B14800820203F00703D2F820E09B004FF00F0CB7
:10B158000CFA03FC2EEA0C0EC2F820E0D2F820E02C
:10B1680001FA03F343EA0E0313626946002302223D
:10B1780014348DF804208DF805308DF806308DF8DC
:10B18800073020F001FCA04596D103B0BDE8F08F50
:10B19800082309EBC3034FF0010B93F820A00AF032
:10B1A8001F034FEA5A1ABAF1020F0BFA03F30BD036
:10B1B800BAF1030F0ED0DA457FF471AFD1F814A0BD
:10B1C80043EA0A034B616AE7D1F818A043EA0A0385
:10B1D8008B6164E7D1F81CA043EA0A03CB615EE700
:10B1E8000023D6E70123D4E7FB694AEA0303FB619E
:10B1F8009DE7BB694AEA0303BB6198E70223C8E7F6
:10B208000323C6E70423C4E70523C2E70623C0E7F0
:10B218000723BEE7206E00203827030800040040FB
:10B228000008004000100040002C014000100240BF
:10B2380004240308102403082C67002028050308A9
:10B248000040014000140040003401400044014027
:10B258003027030801490248FFF71CB9C06E0020D7
:10B268000040014001490248FFF714B9986E0020D8
:10B278000034014001490248FFF70CB9986E0020DC
:10B288000034014001490248FFF704B9706E0020FC
:10B298000004004002494FF08040FFF7FBB800BFB0
:10B2A800486E002001490248FFF7F4B8206E0020DC
:10B2B800002C014001490248FFF7ECB8206E00203D
:10B2C800002C01402DE9F04104684A4DA30AAB4225
:10B2D80072D009D8B3F5801F6AD04A3DAB425AD123
:10B2E8004FF0700E022608E0434DAB4268D003359C
:10B2F800AB4252D14FF0C00E042647794FEA970C63
:10B30800002961D0B000634685190227D4F80C8063
:10B318009F400CEB4503BFB2384D03F1040C47EADC
:10B32800080745F8231045F82C20E760EFF3118152
:10B33800502282F31288821905EBC202136973B393
:10B3480013620433821905EBC202576917B11F60F3
:10B3580053690433821905EBC202976917B11F605C
:10B3680093690433821905EBC202D76917B11F60CC
:10B37800D36904330027CAB21F6082F311883044AE
:10B3880005EBC000036A6BB9E3684FF6FE72134021
:10B39800E360BDE8F081BDE8F081BDE8F08105EB30
:10B3A8000E03CFE7E36843F00103E360BDE8F081F3
:10B3B8004FF0480E0126A0E74FF0200E00269CE72C
:10B3C8004FF0980E032698E7BF08022306FA03F009
:10B3D800BB40DB43E768094D9BB23B4087190CEB48
:10B3E800470CE3600CF1040345F82C1045F82320C2
:10B3F8009CE700BF4B0010004D001000206E00209D
:10B4080030B503685C4D18885C4CB4FBF2F2013926
:10B41800013AAB4294B283B089B282B266D058483E
:10B42800834263D0B3F1804F60D0A0F59830834257
:10B438005CD000F58060834258D0524883425BD08C
:10B4480000F5806083427DD022F4407200F58C3094
:10B4580092B283421A80D9621C850ED0484A934220
:10B468000BD002F54062934207D002F58062934206
:10B4780003D002F58062934201D100221A8601228C
:10B488005A611A883C4992B242F001028B421A80F2
:10B4980062D0B3F1804F61D03B4A934260D002F54D
:10B4A800806293425ED002F5006293425CD002F55E
:10B4B800806293425AD002F59032934258D002F5F6
:10B4C8004062934256D002F5806293421ED002F544
:10B4D8008062934208BF092219D002A84FF00123C5
:10B4E80040F8043D20F0F6F903B030BD254822F0BD
:10B4F8007002834292B2A3D101201A80D9621C85BE
:10B5080058611A8892B202431A80C5E708221F4B75
:10B5180003EBC20301A893F821408DF804400123EE
:10B5280000228DF805308DF807308DF8062020F0C0
:10B53800D1F91B2CD8D1164B019301A820F0CAF9D8
:10B5480003B030BD01201A80D9621C8558611A8861
:10B5580092B202431A809CE70022D8E70122D6E77C
:10B568000222D4E70322D2E70422D0E70522CEE75D
:10B578000622CCE70722CAE7002C014000A24A04B1
:10B588000034014000100040000400402805030872
:10B5980019010001204B98422DD0B0F1804F2CD0DA
:10B5A800A3F5943398422AD003F58063984228D0B3
:10B5B80003F50063984226D003F58063984224D0AF
:10B5C80003F59033984222D003F54063984220D087
:10B5D80003F58063984207D003F58063984208BF5B
:10B5E800092202D00020704708220C4B03EBC2034B
:10B5F80093F8200070470022F7E70122F5E70222BE
:10B60800F3E70322F1E70422EFE70522EDE706223C
:10B61800EBE70722E9E700BF002C014028050308F3
:10B628002DE9F04F013085B0C3B203930B46029168
:10B638008B4C8C4E002B00F09A8032208A4D8B4F19
:10B64800DFF82C9221F084FF4FF4FA7A4FF0100CB7
:10B658004FF47A70D9F80430C3F30803002B40F094
:10B66800DE80EFF31183002B40F0D9802968A268AF
:10B6780000BF2B689942F9D1D7F800E000FB0EF320
:10B688009B1AB3FBFEF300FB01314FF0010E019151
:10B69800D9F80430C3F30803002B40F08780EFF398
:10B6A8001183002B40F082802B68A16800BF2A68B4
:10B6B8009342F9D1D7F800B000FB0BF2521AB2FB53
:10B6C800FBF200FB0323019A9B1AB3F57A7FDFD3C1
:10B6D800BAF1010ABED1039B002B40F0BD804FF4A4
:10B6E8007A7ADFF88C9150464FF0100CD9F8043074
:10B6F800C3F30803002B75D1EFF31183002B71D12D
:10B708002968A26800BF2B689942F9D1D7F800E0F0
:10B7180000FB0EF39B1AB3FBFEF300FB01314FF065
:10B72800010E0191D9F80430C3F3080313BBEFF3FA
:10B738001183FBB92B68A16800BF2A689342F9D12D
:10B74800D7F800B000FB0BF2521AB2FBFBF200FB79
:10B758000323019A9B1AB3F57A7FE3D3BAF1010A5E
:10B76800C4D1029B013B0293002B7FF466AF05B066
:10B77800BDE8F08FEFF311888CF31288A168236875
:10B78800DB0344BFC6F800E0A1682B6832685FFAA3
:10B7980088F888F31188D7F800801A4400FB08F36A
:10B7A8005B1AB3FBF8F300FB0233D2E7EFF311881F
:10B7B8008CF31288A1682368DB0344BFC6F800E055
:10B7C800A1682B6832685FFA88F888F31188D7F87F
:10B7D80000801A4400FB08F35B1AB3FBF8F300FB84
:10B7E800023370E7EFF311828CF31288D4F808E083
:10B7F8002368D90303D501233360D4F808E02B6804
:10B808003168D2B282F311883A68194400FB02F316
:10B81800A3EB0E03B3FBF2F300FB01317FE7EFF379
:10B8280011828CF31288D4F808E02368D90303D571
:10B8380001233360D4F808E02B683168D2B282F370
:10B8480011883A68194400FB02F3A3EB0E03B3FB1B
:10B85800F2F300FB013118E7184621F0E7FC3EE758
:10B8680010E000E0B8710020BC710020C071002019
:10B8780000ED00E0204B5B68C3F3080330B4BBB9AC
:10B88800EFF31183A3B91D4B1D4C1868A16800BFC5
:10B898001A689042F9D11B4B1C684FF47A7202FB6C
:10B8A80004F3591AB1FBF4F130BC02FB00107047E5
:10B8B800EFF31182102383F3128811498C680B6807
:10B8C80013F4803F104B02D0012018608C680B499C
:10B8D800D2B20D68186882F311880A4B19684FF4C0
:10B8E8007A72284402FB01F31B1B30BCB3FBF1F353
:10B8F80002FB0030704700BF00ED00E0BC71002083
:10B9080010E000E0C0710020B87100202DE9F84F68
:10B918008046FFF7AFFF254E2549DFF8A0E0254A0E
:10B92800254D844610274FF47A740120DEF8043040
:10B93800C3F30803D3B9EFF31183BBB90B68D2F88B
:10B9480008A000BFD1F800904B45F7D1D6F800B059
:10B9580004FB0BF9A9EB0A09B9FBFBF904FB0393F8
:10B96800A3EB0C034345E1D3BDE8F88FEFF3118A4D
:10B9780087F31288D2F808B01368DB0344BF286045
:10B98800D2F808B00B68D5F800905FFA8AFA8AF303
:10B998001188D6F800A0994404FB0AF3A3EB0B0323
:10B9A800B3FBFAF304FB0933DAE700BFC0710020E8
:10B9B800BC71002010E000E0B871002000ED00E04C
:10B9C8002DE9F04FDFF830C1474A4849484E494D04
:10B9D8008046102718F1FF38C0F08480DCF8043066
:10B9E800C3F30803002B5CD1EFF31183002B58D16C
:10B9F8000B68946800BF08688342F9D1D6F80090B4
:10BA08004FF47A7000FB09FEAEEB040EBEFBF9FEA4
:10BA180000FB03EEDCF80430C3F308034FF47A7438
:10BA28000120FBB9EFF31183E3B90B68D2F808A042
:10BA380000BFD1F800904B45F7D1D6F800B004FB11
:10BA48000BF9A9EB0A09B9FBFBF904FB0393A3EB78
:10BA58000E03B3F57A7FBDD2DCF80430C3F30803D4
:10BA6800002BDFD0EFF3118A87F31288D2F808B0E1
:10BA78001368DB0344BF2860D2F808B00B68D5F818
:10BA880000905FFA8AFA8AF31188D6F800A09944E0
:10BA980004FB0AF3A3EB0B03B3FBFAF304FB093330
:10BAA800D5E7EFF3118487F31288D2F8089013686A
:10BAB800D80303D501232B60D2F808900B682868B7
:10BAC800E4B284F31188D6F800A04FF47A7400EB3E
:10BAD800030E04FB0AF3A3EB0903B3FBFAF304FB1D
:10BAE8000E3E97E7BDE8F08F10E000E0BC71002043
:10BAF800C0710020B871002000ED00E030B4EFF311
:10BB08001183102282F312880649074C0A680748F5
:10BB1800013200250A602560DBB2026883F31188D0
:10BB280030BC7047BC710020B871002010E000E004
:10BB38000F4B1B88014643B90E4B0F4A1B78106800
:10BB48000BB981F0010119F00FBE0C4B5A691AB1FB
:10BB580018B91A68106058747047094A186811882B
:10BB6800084A92FBF1F2012102605974704700BF44
:10BB78009471002096710020987100209C7100201B
:10BB8800B471002020A107001D4B70B59C68236D7F
:10BB9800626BDD69C2B1A36B2BB12B0702D5236D94
:10BBA80008221A6270BD2A06F7D5A26A616A8A421B
:10BBB80020D0511CA069A162825C2069266D814257
:10BBC8003285EAD3A362E8E7A906E4D5E26A22B19E
:10BBD800988C216B80B29047DDE7E1699B8C6069A6
:10BBE800DBB24E1CE6614354E169E368994228BF21
:10BBF800E261D0E7226D136823F080031360CCE77D
:10BC0800642C00201D4B70B55C68236D626BDD6988
:10BC1800C2B1A36B2BB12B0702D5236D08221A6280
:10BC280070BD2A06F7D5A26A616A8A4220D0511CE3
:10BC3800A069A162825C2069266D81423285EAD3BF
:10BC4800A362E8E7A906E4D5E26A22B1988C216BE1
:10BC580080B29047DDE7E1699B8C6069DBB24E1CDE
:10BC6800E6614354E169E368994228BFE261D0E79D
:10BC7800226D136823F080031360CCE7642C002046
:10BC88002DE9F04FBF4B1E788BB0002E40F0BC80E2
:10BC9800BD4BBE4C1D78DFF814A3DFF81493DFF812
:10BCA800148305F00105A4F10A0B54F80A3CBBB152
:10BCB800CC2707FB06B7184619F0C8F980B154F825
:10BCC8000A0C19F0BBF914F8023C8BB9242831D0BE
:10BCD800F5B154F80A3C184619F0B8F90028EED125
:10BCE8000136032E04F1CC04DFD10BB0BDE8F08F90
:10BCF800012B23D0022B2BD0032B37D0042B67D05A
:10BD0800052B40D0062B4FD054F80A2C1346D2E707
:10BD180054F80A3C23281A4600F087819C4991F878
:10BD280032108142C7D19B4BCAF80090C3F80C80EF
:10BD38001346C0E7012304F8023CCAE74D2854F82B
:10BD48000A2C0CBF0223002304F8023C1346B2E776
:10BD580000233C2804F8023C45D03E28D4D10122D7
:10BD6800032304F8012C04F8023CB2E7C02814D8D5
:10BD78000022042304F8050C04F8040C04F8062C2B
:10BD880004F8023CA5E714F8063C14F8052C9A427E
:10BD98002FD814F8043C834203D0002304F8023C53
:10BDA80097E7062304F8023C14F801ECBEF1000FF3
:10BDB80000F08081BEF1010F00F0C481013600233C
:10BDC800032E04F8023C04F1CC047FF46EAF8CE738
:10BDD80014F8043C04F8030C5840052304F8040C38
:10BDE80004F8023C75E7032204F8013C04F8022C2D
:10BDF8006FE714F8042CF9184240013304F8042CB6
:10BE080004F8063C887264E7634B186800283FF41E
:10BE18006CAF19F0F5FDDFF8A0A1604DDFF89C913B
:10BE2800DAF8000019F012F900283FF45EAFDAF8EA
:10BE3800000019F003F909281BD03F2819D02B68F6
:10BE4800002B66D1042800F0A8810C2800F0E680B9
:10BE58007F28E5D0A0F12002D2B25E2AE0D80BB943
:10BE68002028DDD05A1C09F803002A6007F012FFC9
:10BE7800D6E72C68002C5AD1494B264603F5907B0F
:10BE8800002E08BF1E4608335B45F9D1002E00F08E
:10BE98007881A3F108083068D8F80020075D135DA1
:10BEA8009F42204402EB040140F06981671E4F4421
:10BEB80022460BB9FD2A5CD907F8013F01322A60F6
:10BEC80010F8013F11F801EF9E45F2D00AB1B045D4
:10BED80012D0344807F0E6FEB04508D356F8080BF0
:10BEE80007F0E0FE092007F0D5FE4645F6D92E48B2
:10BEF80007F0D8FE2A680024944291D2661E4E4468
:10BF080016F8010F07F0C6FE2B6801349C42F7D3E0
:10BF180086E70C2800F082800A2851D00D284FD0DF
:10BF28007F2800F0FC80FF2B3FF67AAF92E71C4F8A
:10BF38004FF0000807F5907B464602E008375F455A
:10BF48000DD0224639684846F6F71CFA0028F5D184
:10BF5800B846002EF2D13E4608375F45F1D1002E93
:10BF680099D1B8F1000F3FF45BAF0E4807F09AFE85
:10BF7800B4E7511C202009F80200296009F80130B3
:10BF88000A46A4E7E8400020186F00201658002051
:10BF98005071002000ED00E0102D0020182E002028
:10BFA800981703086829030870290308FC9F0020D4
:10BFB800EFBEADDE0400FA05142D0020182D002078
:10BFC80007F0F1FE23217D4824F0D2F8002800F084
:10BFD800E280A0EB0900286088B1431E19F803101D
:10BFE800202940F0E88009EB030204E012F8011D63
:10BFF800202948D10346581E002BF7D12B604FF457
:10C0080080720021484624F09CF86D4B1B78002B69
:10C018003FF46BAE6B4807F045FE01E76A4807F04E
:10C0280041FE684807F03EFEFAE668496848C97864
:10C03800684ADFF8D0E19362003118BF012101702E
:10C048006549D1624021136382F8341082F8355073
:10C05800624963480B602C32CEF80020584A01230D
:10C06800137008F081FB574807F01CFE4FF400607E
:10C0780021F066FD5B4B93F83230232B00F0938060
:10C0880014F8023C3EE62B60574C002204F5907BE6
:10C0980009F8032002E008345C4578D02168484656
:10C0A80007F0F8FC0028F6D05C4570D26368984722
:10C0B8000023A3E74D4BADF822E00FCB0DF1280C80
:10C0C80002AF87E80F004CF824ED14F8051C14F8AB
:10C0D800033C069404EB010E624639464FF0010C0E
:10C0E80006A8CDF81CE0ADF820308DF824C0FCF788
:10C0F80035FCE8B9019F002304F8023C002F3FF407
:10C10800EFAD54F80A0C1CF0E3FA013654F80A0CA7
:10C11800B847032E04F1CC047FF4C7ADE5E5013B35
:10C12800002233482B6009F8032007F0BBFD77E6AF
:10C13800029A304B03923946A4F10A0002931CF08C
:10C1480041FAD7E714F8053C14F8032C0694234465
:10C1580007936E2A4FF0000308930993ADF8202047
:10C168007FF42CAE06A8F6F78FF906A8F6F780F943
:10C1780006A8F6F77DF906A8F6F77AF91EE622462C
:10C18800A4E61D48A3F1080807F08CFDA6E61B48A5
:10C1980007F088FD8CE728681EE7084806F0B3FE1C
:10C1A8000BB0BDE8F08F164A14F8023CC2F80C80B8
:10C1B800CAF80090A6E5034666E700BF182D0020E0
:10C1C800E8400020702903087829030860630020EC
:10C1D80028250020E81F00201D4D0208142D0020EE
:10C1E800A429030850710020981703089405030830
:10C1F800A029030838720020682903088429030845
:10C2080000ED00E0102D00202DE9F04F2DED068BFC
:10C21800A44BA54A1C7893B000F59C412031814677
:10C2280007911160002C00F09186A04A1268904294
:10C2380040F2DD809E4A029216689E499E4A01910C
:10C24800013C1C709D4B009206F480560493002E0E
:10C2580040F0DB809A4B1B78022B01F0D880042B2E
:10C2680001F04381012B01F0F780964B9945049B1F
:10C278009B7800F25685002B40F05785924B03932C
:10C2880017F078F9914B1B68DC00054640F1C78030
:10C29800039B1B7813F0010300F0CA80009AB2F9DF
:10C2A8000610019A528C914281F2C481002D40F00F
:10C2B800C680874C94F88C20002A40F0C0808549BD
:10C2C800854A086890F82D0000211160516091603E
:10C2D800824A002840F0B4801070002B40F0B580EE
:10C2E8007F4B1A78002A40F01981019900984E8BEB
:10C2F800B0F90070898BB0F90200B742CCBF802436
:10C30800002444F040038F42A8BF23469B0843F013
:10C318008004B042C8BF234643F040048842A8BF07
:10C328001C460098A408B0F90470B0F9060044F05F
:10C338008003B742C8BF1C4644F040038F42A8BFE1
:10C3480023469B0843F08007614CB042C8BF3B4678
:10C3580043F0400794F88E608842B8BF3B469E423F
:10C3680001F09A83A4F8902084F892205D4984F81B
:10C378008E300E78002E01F09B825F2B01F00E8329
:10C388006F2B01F04B83039B1B78D80700F1C68005
:10C3980094F89220002A40F0C180B4F99030322BF2
:10C3A80040F3BC8094F88E300120572B84F892001B
:10C3B80000F0A68002990968490741F1AF815A2B1C
:10C3C80041F0AC8194F89430002B41F0F48694F855
:10C3D800963083F0010384F89630002B41F0938760
:10C3E8000C201CF03BFD404B404D059399E0304B31
:10C3F80002931E68304B2F4A009306F480562F4B49
:10C4080001920493002E3FF425AF00212F48F6F740
:10C4180035FC00287FF41EAF10F0DAFE1AE7029B05
:10C428001B6858023FF534AF039B1B7803F00103E8
:10C43800274C002284F88C20002D3FF440AF274A77
:10C4480001211170002B3FF44BAF029B1B68D906EA
:10C458007FF546AF264A1278D2063FF541AFDF0492
:10C468003FF53EAF17F072F800287FF439AF1D4B47
:10C478001B78002B01F0B4861E4B9B78002D41F0F1
:10C4880036873BB11C4A1D4B12681B689B1A002B50
:10C49800C1F21A8710200E4C1CF0E0FC012384F82E
:10C4A8008D301DE7245D0020F05B0020205D00201A
:10C4B800686B0020247100203C3C0020F43B0020E5
:10C4C800E6350020404B4C00186F00201C710020FE
:10C4D800602000200849002018300020FC1E0020A1
:10C4E800E33F00207C1B00200C4900200449002069
:10C4F8008830002008300020BC7100204C46002005
:10C50800144B154A19684FF47A73B3FBF1F3C3EB74
:10C51800431103EB8103DB00A2F8A8300F4B104D49
:10C528000593029B1B685F0700F141860D4E069537
:10C538000DF1400A0022CAF8042006F150091092B1
:10C54800344640F6330B4FF0190840F28337009D0C
:10C558000DE000BF586B0020CC6800200C4900207B
:10C5680004490020705D002004344C4520D0A17897
:10C57800E378994218FB0170F6D26178043118FB10
:10C58800037335F911105945A8BF5946B1F5617FB4
:10C59800B8BF4FF461718142E6DD9942E4DC21784D
:10C5A8002729E1D850460434F6F758FB4C45DED12C
:10C5B800CC4A069D1378CC4A9AE8030082E8030027
:10C5C800002B40F04585C94B1A78002A00F06E858B
:10C5D8000121C548F6F752FB002840F09282049BDF
:10C5E800DB78002B40F08D82C14B06932B881FB25D
:10C5F80027F001071FFA87F84345A5F8008000F0E7
:10C608008287BC4F4FF002090E204FF0140A4FF0FA
:10C61800FF0B87F8009087F801A087F802B01CF09C
:10C628001DFC4946B048B5F80080F6F727FB0028FE
:10C6380041F0838128F002039BB243452B800BD045
:10C64800AC4B02201421FF2218700E2059709A70EA
:10C658001CF004FCB5F8008018F003011ABF012192
:10C668000846012019F08AF824219F48F6F706FBAE
:10C6780030B9039A13785F0744BF23F0040313709B
:10C68800069B1B6813F00A0F11D006219648F6F78F
:10C69800F5FA002800F0A5872B88580641F1158186
:10C6A80007219148F6F7EAFA002840F042870C2162
:10C6B8008D48F6F7E3FA2A88002800F0418242F410
:10C6C80080739A422B8009D08A4B02271421FF22BB
:10C6D8000E201F7059709A701CF0C0FB864B1B7897
:10C6E800082B00F039820E2B00F03682029BD3F81B
:10C6F800008018F4806F12D0804B1B79002B00F05B
:10C70800E28114217848F6F7B9FA002840F0E08170
:10C7180012F034F91CF0E4FA029BD3F80080039B72
:10C7280093F80090764B19F0010900F0428201223B
:10C738001A70059B00991B68B1F906105A8971484F
:10C7480001279142077080F21A826F4B4FF07E5298
:10C758001A60019B6D4FB3F818A0009B97F904204D
:10C76800B3F90030387897F801C0002AA3EB0A071C
:10C7780014BF01224FF0FF32002FB8BF7F42B7F538
:10C78800FA7FA8BF4FF4FA77B84280F2BA823F1A0C
:10C7980007EE907AF8EEE77A5D4F9A45C7ED007A92
:10C7A80003DDF1EE677AC7ED007A009BB3F902E08A
:10C7B800AEEB0A03002BB8BF5B42B3F5FA7FA8BF04
:10C7C8004FF4FA73984280F299821B1A07EE903A56
:10C7D800F8EEE77AF245C7ED017A03DDF1EE677A04
:10C7E800C7ED017A009BB3F90400A0EB0A03002B04
:10C7F800B8BF5B42B3F5FA7FA8BF4FF4FA7363453D
:10C80800CCBFA3EB0C03002302FB03F307EE903A23
:10C81800F8EEE77A5045C7ED027ABCBFF1EE677AC9
:10C82800C7ED027A18F4805200F04182B1F5FA6F30
:10C83800384BA8BF4FF4FA61B1F57A7F1878B8BFC2
:10C848004FF47A71A1F57A71002841F06680DFF81B
:10C85800DCE031488EFB013CCB17C3EB6C1303F1D2
:10C86800010C6FF0630830F91CC030F9130008FBA5
:10C878000313ACEB000103FB01F38EFB031EDB1774
:10C88800C3EB6E1303441BB207EE903AB8EEE78A87
:10C8980087ED038A002A40F09B832B885A0640F1D3
:10C8A80007811E491E4A91ED010AD2ED018A92EDD7
:10C8B800026A91ED034AD2ED033A91ED028A92EDB4
:10C8C800007AD1ED005AD7ED011A97ED002A154AE2
:10C8D800154930EE445A78EEC66A75EEC84A65EED8
:10C8E800266A27E0F04B00201C710020E840002059
:10C8F800B04800201C3A00207C300020C062002094
:10C90800196F0020581F0020B01E0020E02F0020C3
:10C91800D0620020A824002040610020B406002036
:10C92800700A0020A80A0020602000201F85EB5113
:10C938000000000077EE237A37EE639A75EE889A46
:10C9480024EEA71AB0EE663AA9EE893A13F003036B
:10C95800B0EE415A70EE044A78EE867AA9EE895A0A
:10C96800F0EE660AA4EEA73AD4EEA70AA4EEE75AB8
:10C9780033EE013AF0EE607AF0EE674AF6EE000A1E
:10C9880035EE80AAE9EEC94A20EEC33A35EE665A7A
:10C9980077EE286A77EEC17AAAEE263A25EE205A73
:10C9A80076EE636A34EE48AA74EE814AE9EE897A33
:10C9B800AAEE265A37EE687A34EE084A64EEA04AA0
:10C9C80063EE036AE4EE074A75EEC05A36EE236A50
:10C9D80067EEA07AB0EE667A95EE057AE5EE056A1E
:10C9E800E5EE867AB1EE648AF0EE665AF0EE476AB2
:10C9F800B1EE674AE8EE246A63EE270A67EEA43AC6
:10CA0800E4EE275AB1EE450AB0EE609AB0EE631A2A
:10CA1800A4EE277A23EE244AE7EEA76AA5EE249A25
:10CA2800A0EE031AE8EE245AB0EE448A31EEA16A69
:10CA3800E0EE240AA5EE278A66EEA16A72EE028A63
:10CA4800E5EE033A61EE211A26EE096AA4EEA47A0D
:10CA5800A0EE274A0CBFD7ED022A5FED4B2A82EDE4
:10CA6800005AA2EE256AE0EEA86AE2EE081A73EE12
:10CA7800A33A27EE227A34EE044AF0EE005AE3EEA7
:10CA8800A26AA4EE226AA1EEA57AC7ED016AC1EDF9
:10CA9800366A81ED356A87ED006A81ED377A82ED75
:10CAA800013AC2ED027AC2ED034A0BB987ED027A68
:10CAB800B9F1000F40F0288121F020F913B0BDEC46
:10CAC800068BBDE8F08F039B1B78D9077FF520AE56
:10CAD8004FF40F7013F08CFA00283FF41DAE1BF0D2
:10CAE800C1FE4FF40F7013F025FA00283FF414AE7E
:10CAF8001BF0B8FE4FF40F7013F01CFA0028EED1AB
:10CB08000AE69C4B06931B689B077FF56FADB5F84B
:10CB1800008018F0010F7FF48DAD48F001039845AF
:10CB28002B803FF487AD944B022214211A700E20FB
:10CB3800FF2259709A701CF091F9B5F8008079E5D8
:10CB480022F480739BB29A422B807FF4BDAD8B4B4D
:10CB58001B78082B7FF4C7AD2A8822F040039BB2CC
:10CB68009A422B803FF4C2AD834B02271421FF2247
:10CB78000E201F7059709A701CF070F9B6E5B1F567
:10CB8800FA6F80F23D84187A8B1A03FB00F3C2F522
:10CB9800FA6293FBF2F3C3F1640307EE903AF8EEFE
:10CBA800E77A9FED777A774B67EE877AC3ED007A5D
:10CBB800CFE51B780293002B7FF4BBAD724A126855
:10CBC800002A3FF4B6AD714A039212F8030CDFF85D
:10CBD80000B21146D71E16F08FFC9BF800A0039AEE
:10CBE800002800F04285029BBAF1000F53D107F1EB
:10CBF8000801787916F080FC002841F0D882644951
:10CC0800B87A16F079FC002800F04285BAF1020FD4
:10CC180041F0C9825F49F87B16F06EFC002841F0AC
:10CC2800BE825D49387D16F067FC002800F0428519
:10CC3800BAF1040F41F0AF825849787E16F05CFCD7
:10CC4800002841F0A2825649B87F16F055FC00280A
:10CC580000F04285BAF1060F41F09382514997F8E6
:10CC6800230016F049FC002841F087824E4997F8C6
:10CC7800280016F041FC002800F04285BAF1080FA0
:10CC880041F07782494997F82D0016F035FC0028C5
:10CC98003FF44FAD09231A4602EB82021744444A77
:10CCA8007878B9788BF800301070517041E5019BA5
:10CCB800588B8142C0F2A283B1F5FA6FD4BFC0EBA2
:10CCC8000101C0F5FA614FF47A7303FB01F1DFF853
:10CCD80004E19EF800C0C0F5FA63B1FBF3F1BCF1C2
:10CCE800000F3FF4B4AD9EF80130324801FB03F366
:10CCF80080FB0301DB17C3EB6111A8E5DFED2E7A9A
:10CD080068E5DFED2D7A47E52C4A2D4B1178186838
:10CD180001F0010118F028FD13B0BDEC068BBDE849
:10CD2800F08F13B9049A01239370264B049A1D7847
:10CD380092F8214003931B2016F016FC012C05F0F5
:10CD48000108814600F0438605F00205049A1E4E4C
:10CD580092F82030DFF880A01C4F05959346052BEC
:10CD680000F2B286DFE813F0C100B7003A00E30032
:10CD7800E500D800B04800201C3A00207C30002094
:10CD88000AD7233CB01E00201C6F0020D639002093
:10CD9800E0390020E5390020EA390020EF39002089
:10CDA800F4390020F9390020FE390020033A002028
:10CDB800206F00201F85EB510000000084710020C7
:10CDC80088710020186F0020386100200049002079
:10CDD80008000020A82400207C1B0020012C04BF90
:10CDE80005238BF82030B8F1000F12D0019B308852
:10CDF800B3F918100022134661F30F0260F31F42C3
:10CE080061F30F03009861F31F430360032342603B
:10CE180005939B4DDBF814102A68914280F0388501
:10CE280047F230510322CBF81C108BF82020022047
:10CE380020F086FE10F0CCF92968DBF81C200A44A3
:10CE48000421CBF818208BF82010012C40F0948690
:10CE58002A68DBF81810914280F036869AF80000AC
:10CE680020B916F081FB002840F02E863A6822F09F
:10CE780002023A602A687388642101FB03234FF495
:10CE880080600022CBF810308BF820208BF803202C
:10CE980004F09EF99BF8203061E716F06BFB01283F
:10CEA80007D1774D72882B68642101FB0233CBF8D8
:10CEB8001030B9F1000F01D0B3797BBB012C00F021
:10CEC80003866F4DDBF810102A689142C0F0618626
:10CED80001238BF82030012C1ED0F379012B2AD0A6
:10CEE80016F0C8FA9BF8203039E7B8F1000FD4D112
:10CEF800059D4FF48060B9F1000F00F0178304F02E
:10CF08007FF9049A00231361002D3FF4B9A928463C
:10CF18001BF0A4FFFFF7B4B9594DABE716F0AAFA16
:10CF280003224FF47A738BF82020CBF81C30544D31
:10CF38007DE7534D89E716F09DFA032240F6B83392
:10CF48008BF82020CBF81C304D4D70E74D4F3B78C7
:10CF5800002B01F085804C4BDFF84481DFF844B1A9
:10CF6800DFF844A1019345465E46009099460EE0DD
:10CF780019F804109847032C28DC88B93B782AF85C
:10CF8800020F01349C4205F1040580F23581072C1B
:10CF9800E1B23046DBF80430EADD984700B2EDE74D
:10CFA80038F824206B88801A4FF47A719B1A01FB99
:10CFB80000F040F6CA0290FBF3F00844904240F2B9
:10CFC800EE23A8BF10469842B8BF184600B2D5E76E
:10CFD8001D212E48F5F752FE28B100F037BD043662
:10CFE800A6423FF45AAC31782629F8D1B278F378C2
:10CFF8009A42F4D2049BDB78002B7FF44EAC234892
:10D00800F5F73CFEDFED227A002801F06E8038EE5D
:10D01800678A20482049FDEEC87ACAF57A73CDEDB3
:10D02800007ABDF90020120380FB0240D2171BB220
:10D03800C2EBA01203FB02F343F30F33534407EE92
:10D04800903AF8EEE77A0123C7ED037A0B7024E4EF
:10D05800124B03E004339C423FF4B5AA1978232904
:10D06800F8D19878DA789042F4D20848F5F706FEB5
:10D0780000283FF4A8AA14201BF0F0FEFFF7A3BA7B
:10D08800BC710020345E0020247100201C71002037
:10D0980000007A44D34D6210281F0020705D0020E4
:10D0A8004C5E0020DC5B00205E200020DFF8F09260
:10D0B800DFF8F0A2AB4F069209F15A084FF0010BC6
:10D0C800494619F8010C16F017FA00B399F804004C
:10D0D80099F8023099F803E000EB400107EB810171
:10D0E800013BD1F8A02003EB4303534493420ED0F5
:10D0F80097F8CC20C1F8A0300BFA00F022EA000023
:10D10800069B81F89CE0C1F8A43087F8CC0009F1AF
:10D118000609C845D4D1944B944A1B780693059BBD
:10D12800DFF884A212681B680793AAF19C094FF0E4
:10D13800000B9046DAF8043083B31F7877B3DAF837
:10D148000820A8EB0202002A0CDB99F8CC20012168
:10D1580001FA0BF122EA010208F5FA7189F8CC20EC
:10D16800CAF80810069ACAB19AF800205978043209
:10D17800D2B2002940F0648201990098098B30F9F5
:10D18800122001F1C800824240F3C88499F8CC10FB
:10D198009A7841FA0BF3D80740F126850BF1010B79
:10D1A800BBF1040F0AF10C0AC4D1FFF711BA6D4C98
:10D1B80094F896305BB1039B1B78DE0707D5009B7C
:10D1C800B3F90620019B5B8B9A4200F3FC84112182
:10D1D8006748F5F753FD002800F01A8294F89A3052
:10D1E8002BB994F8943013B93223A4F8983001235A
:10D1F80084F89A30FFF79AB9DDF800905D4A0292F8
:10D208005D49126842F2010AA1FB091B12EA0A0AE7
:10D218004FEA9B1B00F0F981584D5948524C594927
:10D228002E780078267008701EB156490E7886F060
:10D2380001064C4C0F2184F82410002B00F04D837C
:10D24800019D514BB5F826C0B5F824E0019D0C931B
:10D2580018462D8B00784D4B0E9594F82550059562
:10D268004B4D0095A3FB00535B0803EB4303C31A24
:10D27800DBB20B90CDF824C002F48052089304F17D
:10D2880028000BF59673CDF8349097F80080DDF8F8
:10D298001490DFF818C105943D4C0A910F920021B3
:10D2A80006930496CDF80CE0049B002B00F09282C4
:10D2B800059B039D33F911201FFA82FEAE454FEA04
:10D2C800410303D3099DAE4540F2C9825CF8212091
:10D2D800934580F08982E25EBAF1000F40F09E82A9
:10D2E80001314145E25200F10600DDDB0A9A059C56
:10D2F800284B84F824200F2A49460CBF012200221B
:10D30800DDF8349084F825101A7000F0ED82224B75
:10D318001B491C4ADFF854B004931C46042001231F
:10D328000B70137020F00CFCDBF80030A168626809
:10D33800E3605B1A934284BF002384F82130029B88
:10D348003C781E68002C00F0BD86019A134DB2F897
:10D3580024E0178B0E4916F48056284640F00083C7
:10D36800324636E060200020E53B0020BC710020FA
:10D378001C710020686B0020D34D6210B85B002040
:10D388006D0A00206E0A0020255D0020ABAAAAAA1B
:10D398003C3C002089300020F43B0020805E0020C7
:10D3A800ED380020A4050308FC200020285D00209B
:10D3B8006F12833F437803EB830303EB830303F28A
:10D3C800EE239BB20132A24221F8023B00F1020097
:10D3D8000ED015F81230002B00F04582022BE9D050
:10D3E80001320B8821F8023BA24200F10200F0D181
:10D3F8000C9A137801331370FEF729BF114666E4BF
:10D408001B7AC3F1640307EE903AFFF7C8BB019A91
:10D418000099537DD27D013B31F913301AB1C3F520
:10D428003B6308331BB2A3F57A7307EE903A1FEDFE
:10D43800207ACD4AF8EEE77A40F2FF3167EE877A34
:10D44800FCEEE77ACDED037ABDF80C308B4228BFAD
:10D458000B461380FEF709BFC44CD4F88830A9EBFB
:10D468000303002BFEF601AFC14AC24B527C01995F
:10D4780033F812308A7DDFEDC06A9FEDC06AC97D3E
:10D488009BB207EE102A07EE903AB8EEC77AF8EE8C
:10D49800E77A27EE267A67EE867A079AC4F8882014
:10D4A800C7EE876A40F2FF32FCEEE67ACDED037AEA
:10D4B800BDF80C30934228BF134609B1D31A9BB26A
:10D4C800AF48B04D0178B04C35F81160226825F8A6
:10D4D8001130921B13440131A34D236001F00F0258
:10D4E8001B0902702B80FEF7C0BEFEF7C3F9A74BDD
:10D4F800A74A1B68C31A93427EF7B7AE9A4B00221D
:10D508001A80FEF7B2BE0221A248F5F7B7FB002841
:10D518003FF490A82F8018F0020F7FF49DA80220F6
:10D5280003F06EFEB5F80080FFF796B803F050FEE2
:10D53800E7E4994AB2F90030002BB8BF5B42B3F573
:10D54800E17FBFF6B4A8B2F90230002BB8BF5B4246
:10D55800B3F5E17FBFF6ABA8904B93ED057AD3ED19
:10D56800077AD3ED096A93ED030A77EEA67A30EECF
:10D57800070AF7EE000AB0EE007AE7EEC70A30EEC7
:10D58800000AF5F73FF9B6EE008A20EE488A9FEDCB
:10D59800840A38EE000AFDEEC07A17EE903A20337E
:10D5A800402B40F21E839FED7F0A7F4FDFED7D7A8F
:10D5B80087ED000ABDEEC87AC7ED017A17EE103A7A
:10D5C8002033402BC7ED027A00F22285B0EE480ADC
:10D5D800F5F79EF80A2087ED030A1BF03FFCFFF7DA
:10D5E80066B82A8822F040039BB29A422B803FF407
:10D5F80057A86E4B02271421FF220E201F70597066
:10D608009A701BF02BFCFFF74BB869490E780BE6B4
:10D6180094F89430002B3EF489AF039B1B7813F0E9
:10D6280001037EF483AF012284F8943084F89520B6
:10D63800FEF77CBF4D4C012284F88C20FEF7FFBE1C
:10D64800012900F09A8499F8CC20012303FA0BF3FE
:10D658000BF1010B1343BBF1040F89F8CC300AF12D
:10D668000C0A7FF467ADFEF7B3BF511D787915F04A
:10D6780043FF00283FF4C3AABAF1010F40F0978591
:10D6880007F10D01B87A15F037FF002840F08B85B7
:10D698004849F87B15F030FF00283FF4C2AABAF1D8
:10D6A800030F40F07C854449387D15F025FF00289C
:10D6B80040F071854149787E15F01EFF00283FF43F
:10D6C800C2AABAF1050F40F060853D49B87F15F050
:10D6D80013FF002840F055853A4997F8230015F0C4
:10D6E8000BFF00283FF4C2AABAF1070F40F04585A6
:10D6F800354997F8280015F0FFFE002840F03985D5
:10D70800324997F82D0015F0F7FE00283FF411A8CC
:10D71800BAF1090F3FF40DA8FFF7BCBA5D2B00F072
:10D728007B845B2B00F065825E2B00F00985562B0D
:10D7380000F00885972B00F01185A72B00F0F684E0
:10D74800234D2A88920740F08F84A3F1B702072A55
:10D7580000F27882DFE812F06F0276027602760233
:10D76800680276025C025502EC3B00206020002033
:10D77800C86D0020E86D00200000C8420000804409
:10D78800E7350020EC350020E8350020D81F0020C0
:10D7980060E316001C710020B4480020800A0020B5
:10D7A800DB0FC93F00000000B40600201C3A00202F
:10D7B800E53B0020E5390020EA390020EF39002058
:10D7C800F4390020F9390020FE390020033A0020FE
:10D7D80004490020039B002B3FD05CF8212093458F
:10D7E8004FEA4103FFF477ADBA4ABA4DD25C05EB74
:10D7F800030E002A00F09480022A47D19EF80120E7
:10D8080002EB820202EB820202F2EE2292B20329BA
:10D8180033DD12B2BAF1000F3FF462AD089D20F873
:10D828001520B9F1000F03D10B9D022D7FF658ADDD
:10D83800B0F802900288B0F804E04A449644A64A38
:10D848000FFA8EFE82FB0E52A44DA2EBEE7225F863
:10D8580003E012B24FF0010942E51A464B00069D5B
:10D868004CF8215038E5D3B2022B04D9032B7FF4AE
:10D87800B7AD7346A6E53B46A4E5012505FA01FECA
:10D888000A9D25EA0E0512B20A9525E5E25ABEE779
:10D89800934A1278002A7FF4C3AAB8F1000F3FF424
:10D8A800BFAA012C40F010819BF82030FFF757BA2F
:10D8B80031468C48F5F7E2F9002800F08B8084F8AF
:10D8C800936010F083F8FEF75EBD43F04002934288
:10D8D8002A807FF48EAEFEF7E3BE834B834A0C9218
:10D8E80001221A70824B00931B217E48F5F7C6F976
:10D8F80000287FF40CAD7F4BDFF81CB20493194667
:10D90800DBF80030CA688B609B1AC82B00F2DE83F4
:10D91800029B1E6806F480566AE55B78FFF7E5B956
:10D92800CAB2022A40F22783032AAFD10E9A0F9D6A
:10D93800039E002D08BF324669E728F0010292B223
:10D9480042452A803FF4E7AD0E2087F8009087F81B
:10D9580001A087F802B01BF081FAB5F80080DAE57B
:10D9680000220FE0437803EB830303EB830303F206
:10D97800EE239BB20132A24221F8023B00F10200E1
:10D988003FF436AD15F812301BB1022BEAD00B88E4
:10D99800F0E7D3B2032BFAD83B46EBE7B2F5FA7FB0
:10D9A800FEF6BCAD94F89230002B7EF4B7AD039B25
:10D9B8001B78012213EA020584F8922000F01983EB
:10D9C8000FF006FC4C4B4D4D0593FEF7AABD002504
:10D9D800FFF7BCB9039B4A4A1B781060DE077EF547
:10D9E800D7AC484B1B78002B3EF498AD049BDB78F2
:10D9F800002B7EF493AD94F893300133DBB2032B04
:10DA080084F893307EF68AAD3F4B5B7813B9002DCE
:10DA18007EF484AD0FF0DCFBFEF7B5BCB2F5FA7FFF
:10DA2800FEF67CAD94F89230002B7EF477AD039A25
:10DA38001278012184F89210D40700F10A830FF0BC
:10DA4800C5FF2D4B2D4D0593FEF76BBD049BDB7871
:10DA5800002B7FF4C8AADFED2D7A2D4938EE678AAE
:10DA6800CAF5FA63FDEEC87A1BB2CDED007ABDF9AE
:10DA78000020120381FB0201D217C2EBA11203FBA3
:10DA880002F343F30F33534407EE903AB8EEE78AB4
:10DA980087ED038AFFF7A7BA1E4A1D491068B4F933
:10DAA8009020C66981FB06018911F617701A00F5E6
:10DAB800FF407F3082423EF759AC891B0A4412B2BC
:10DAC800A4F89020FEF752BC059D002D3EF4D8AB7B
:10DAD800FFF71DBA805E002056555555D02000200E
:10DAE800EC1E00201C71002089300020255D0020DC
:10DAF8003C3C0020F43B00200C4900200449002055
:10DB080050460020E53B00200830002000007A4401
:10DB1800D34D6210BC4A0020BC710020C8398A422B
:10DB280042DA99F8CC109A7841FA0BF3D9073FF505
:10DB380035AB5242012008921BF062FA7B1E089A0C
:10DB4800162B00F2E980DFE813F0410154012901A6
:10DB58000202DC01ED01C701A60191017C01670108
:10DB6800E7000202D900ED01C701A601C500B10016
:10DB78009F001401FE00EA00AB460499DBF8002080
:10DB8800CB69059D13448B61002D3EF479ABFFF7FB
:10DB9800BEB915F06FFC032140F6B8328BF820109F
:10DBA800CBF81C20FFF743B999F8CC30012202FAD0
:10DBB8000BF223EA020308F5FA7289F8CC30CAF8A6
:10DBC8000820FFF7EBBA0021BD48F5F757F8002801
:10DBD8007FF4FDAA322384F89600A4F89830FFF762
:10DBE800F6BAF4F795FDE0E4002A0CBF0120022004
:10DBF800A1E70120FCF7BEFCB24BB34D0593FEF73D
:10DC080090BC022003F0A8FFAE4B0593FEF789BC39
:10DC1800AC4AAE4B05921146AD4A0A6002225A70D0
:10DC280015F006FDFEF77DBC002003F095FFA54B1F
:10DC38000593FEF776BC012003F08EFFA14B0593F8
:10DC4800FEF76FBC9E2B00F020839D2B00F01683FF
:10DC5800AE2B00F00C83AD2B00F00283EF2B00F00D
:10DC6800FC82FD2B00F0F682FB2B00F0E382FE2BFA
:10DC780000F01283F72B00F024837B2B00F0AA829C
:10DC8800904B0593FEF74DBCD9F8D000914B8178A5
:10DC98001144C829A8BFC82121EAE17181709B7885
:10DCA800002B40F01E8314F06BFDCCE4D9F8D000B3
:10DCB800884B41781144C829A8BFC82121EAE171DD
:10DCC80041709B78002BEED0132015F097FCD9F803
:10DCD800D000E8E7D9F8D0007E4B01781144C82974
:10DCE800A8BFC82121EAE17101709B78002BDAD026
:10DCF800122015F083FCD9F8D000D4E7754B0798AB
:10DD08009B78417911446429A8BF642121EAE17113
:10DD18004171002B40F0DF82D9F8D000C3E7D9F871
:10DD2800D0006C4B90F836109B7811446429A8BF3A
:10DD3800642121EAE17180F83610002BB3D0172056
:10DD480015F05CFCE8E7D9F8D000624B90F8371082
:10DD58009B781144FE29A8BFFE2121EAE17180F8D1
:10DD68003710002B9FD0162015F048FCD9F8D000AA
:10DD780099E70798574B41781144B1F5967FA8BFAA
:10DD88004FF4967121EAE17141709B78002BC3D062
:10DD9800152015F033FCD9F8D00084E707994D4BCE
:10DDA8000F7908931744642FA8BF642727EAE777F9
:10DDB8000F7115F03DFC089B9B78002BACD003201D
:10DDC800394615F01BFCD9F8D0006CE70798414B91
:10DDD80001781144FA29A8BFFA2121EAE1710170FA
:10DDE8009B78002B98D0012015F008FCD9F8D000BA
:10DDF80059E70798374B817811446429A8BF6421F3
:10DE080021EAE17181709B78002B85D0022015F002
:10DE1800F5FBD9F8D00046E7D9F8D0002D4B017AA8
:10DE28009B781144C829A8BFC82121EAE171017271
:10DE3800002B3FF438AF0B2015F0E0FBD9F8D000E9
:10DE480031E7D9F8D000234BC1799B781144C82910
:10DE5800A8BFC82121EAE171C171002B3FF423AFAB
:10DE68000A2015F0CBFBD9F8D0001CE7D9F8D00070
:10DE7800184B81799B781144C829A8BFC82121EA89
:10DE8800E1718171002B3FF40EAF092015F0B6FB4C
:10DE9800D9F8D00007E7D9F8D0000E4B417993F8AC
:10DEA80002E01144C829A8BFC82121EAE1714171E3
:10DEB800BEF1000F40F0F381112F7FF4E8AEF2E6D7
:10DEC8001C7100200C4900200449002060630020D8
:10DED8009E640020BE640020D9F8D000C84B0179A8
:10DEE80093F802E01144C829A8BFC82121EAE171CA
:10DEF8000171BEF1000F40F00E82102F7FF4D9AEF1
:10DF0800D1E60798BE4BC1799B78114481F308018B
:10DF1800C171002B3FF400AF052015F06FFBD9F855
:10DF2800D000C0E6D9F8D000B54BC17893F802E02C
:10DF38001144C829A8BFC82121EAE171C170BEF106
:10DF4800000F40F0F2810F2F7FF4C7AEABE60798C1
:10DF5800AB4B817993F802E011446429A8BF64218E
:10DF680021EAE1718171BEF1000F40F0A2810D2F0D
:10DF78007FF4C5AED0E60E9A49E400999B7831F952
:10DF88001220B2F5617F4FF4966191FBF3F345DB04
:10DF980040F633019142A8BF11460C2FA1F56171DB
:10DFA80091FBF3F100F0F580182F7FF44CABC9B268
:10DFB800C8290B46A8BFC823D9F8D020D77DD8B226
:10DFC800B8423FF440ABDF1B8D4BD07548BF0737D5
:10DFD800FF109B780137FFB23BB9002F3FF433ABFA
:10DFE80038461BF00DF8FFF72EBB182015F006FB7E
:10DFF800F3E70F201AF032FFB4F8903084F892500B
:10E00800FA3BA4F890307F4B7F4D0593FEF789BA11
:10E01800B0EE670AFFF7DEBA0020EBE50C2F40F000
:10E02800978000273946794B09915B78BB423FF4CA
:10E038000AAB734B0893384603F08EFD089B099989
:10E048009B781BB1C9B20C2015F0D8FA0137FFB282
:10E05800C3E76F4A6C4D13606A4B0593FEF761BACC
:10E068006C4A0192FFF7CAB80022BB2B10927ED0EF
:10E07800B72B00F0AC80BE2B00F0A680BD2B7FF440
:10E08800E1AD13464FF6FE7263495E488E890590EE
:10E09800C889324403448A81CB8112F0A1FDF3F789
:10E0A80065FE12F085FDFCF729FB01201AF0A8FF98
:10E0B800B4F890300022FA3BA4F8903084F892200B
:10E0C800FEF72FBA06F48056FFF792B9534A029B1F
:10E0D8001E68136823F004031360049A012306F4EE
:10E0E800805682F82130FFF783B938EE678A4C4BA7
:10E0F8004C491870FDEEC87ACAF5FA63CDED007A7E
:10E10800BDF90020120381FB0201D217C2EBA11254
:10E118001BB203FB02F343F30F33534407EE903A69
:10E12800F8EEE77AC7ED037AFEF7B7BB3E4A364DFD
:10E13800137843F004031370324B0593FEF7F1B9DB
:10E14800022057E5FCF776FC94F88E30FFF7F2BA18
:10E15800182F7FF478AA00210B462DE7334B2A4D60
:10E168004FF4C8721A80274B0593FEF7DAB90223D9
:10E178008AE708231A46FEF78FBD07231A46FEF7DB
:10E188008BBD06231A46FEF787BD05231A46FEF700
:10E1980083BDCFB247E704231A46FEF77DBD0323AC
:10E1A8001A46FEF779BD02231A46FEF775BD01230C
:10E1B8001A46FEF771BD134B84F8942084F8950035
:10E1C800114D0593FEF7F4BF134602225CE74FF6A4
:10E1D800FE7359E74FF4FA61022003F0E3FB4FE5C1
:10E1E800002D3EF457A9124C94F88D30002B3EF4C4
:10E1F80077A81AF01BFE002384F88D30FEF770B85C
:10E20800BE6400200C4900200449002060630020FF
:10E218005046002024710020E82F002000490020EB
:10E22800281F0020D34D6210883000202E72002055
:10E23800602000200021022003F0B4FBB4F89030E5
:10E248003F4A0592963B0022A4F8903084F8922029
:10E25800FEF767B900210120EEE700210846EBE749
:10E26800FF2100201DF08EFE94F88E30F6E4012187
:10E2780000201DF087FE94F88E30ECE40021FF208A
:10E288001DF080FE94F88E30E2E4002101201DF09C
:10E2980079FE94F88E30D8E400210320CCE71120D1
:10E2A8000993089215F0AAF9D9F8D000099B089AA1
:10E2B80002E60D200993089215F0A0F9099B089A27
:10E2C80055E600210420B7E71E4C0EF081FF84F8C4
:10E2D8008D50FEF705B80E2015F090F9D9F8D0004A
:10E2E800E1E4142015F08AF9D9F8D000DBE4002B1A
:10E2F8003FF479AF1449154A09684FF47A7000FB66
:10E30800031313606FE70B201AF0A8FD0C4B104D98
:10E318000593FEF706B910200993089215F06EF9D7
:10E32800D9F8D000099B089AE7E50F2009930892CD
:10E3380015F064F9D9F8D000099B089A03E600BFE4
:10E348000C49002060200020BC7100204C460020B1
:10E35800044900202DE9F04F2DED028B93B00546BE
:10E3680010F00CFBB34B1E7826B113B0BDEC028B3A
:10E37800BDE8F08FB04B1B685805F6D5DFF81C8355
:10E38800D8F80020002A00F01C81AC4CD4F82831C1
:10E3980003F5F43348339D42C0F01381A84994F83B
:10E3A8002C310968C4F828510133DBB2890784F895
:10E3B8002C3101F1108113F0070701F05D80282B43
:10E3C800A04B029301F090815E2090479E4B1B78F2
:10E3D800002B6BD0994C9D4AD4F83031EB1A9342FC
:10E3E80000F2CE87DFF8B8A29AF80080B8F1000FE3
:10E3F80033D1DFF86892D9F8000016F027FEC0B2D2
:10E4080001280ED90228924F41F06E823B78002BEA
:10E4180041F09C83D4F83831EB1AB3F57A6F81F068
:10E4280048848C480768002F40D09AF80030BBB960
:10E43800894BD9F800001B689B781E3B012B4FF0D5
:10E44800020141F28E83043010F0C8F90122002342
:10E458008AF8002084F8443126E07E4807682FB304
:10E46800D4F8403140F6B732EB1A93421ED994F8EB
:10E478003C31002B01F02F82013BDBB284F83C31A8
:10E48800002B01F0168117F8011B94F8442107604E
:10E4980094F8453171480A440133006884F84421EE
:10E4A80084F8453116F0D6FDC4F840516C4A029BF9
:10E4B80012781B68012A03F101030A9300F0B18660
:10E4C800684B1B786BB1684F3B6853B1029B5B4C40
:10E4D800D3F800B0D4F85831ABEB0303632B00F248
:10E4E8004086DFF8C08198F800A0BAF1020F01F069
:10E4F800BC80574F97F87430032B00F087875B4B2D
:10E508001B7873B15A4E33685BB14C4CFDF7B2F9C6
:10E51800D4F8643144F61F62C31A9342834600F26A
:10E52800D580544B1B78002B4ED1534B1B7843B1ED
:10E53800424CD4F8B43203F50043E8339D4280F0EE
:10E54800E6864E4B1B78002B3FF40FAF3B4E4C4CEE
:10E558004C4D06F2BD27206816F078FD00283FF4E0
:10E5680004AF206816F06AFD2B7880465A1E33B136
:10E5780020682A7016F06AFD0028F2D1F5E6032219
:10E588003946781E21F0C3FD96F8BC3296F8BD22B4
:10E5980086F8BF8283F47F4383F0FF039B1A1FFA38
:10E5A80088F89BB2B8EB132FD5D196F8BE22DBB210
:10E5B8009A42D0D1781E16F0C7F92B7818442870E3
:10E5C800C9E7204B029301E72F4C2278002A40F03C
:10E5D8001F86DFF8D49099F80040002C66D12B4EA6
:10E5E8003078002841F03D82144C294ED4F8AC22F2
:10E5F8003178284B93FBF1F313449D4295D3264A77
:10E6080094F8B032C4F8AC52D75CF90701F16F83C3
:10E61800BA0701F1B8837B0701F1FF8294F8B032A1
:10E628003178013393FBF1F201FB123384F8B032F5
:10E638007BE700BFE8400020686B002040210020F5
:10E64800B0480020BC710020B64900203F0D0300EF
:10E658000C0000201C490020184900201449002003
:10E66800B7490020C4490020A44F0020CC4900200D
:10E67800D0490020104A0020214A0020D649002015
:10E68800DC490020E0490020A8490020184A002061
:10E69800204A0020A08601001C4A002024490020AE
:10E6A80020490020E65C0020194A0020054E376EFC
:10E6B800002F41F05480044B89F80070C3F8AC5225
:10E6C80033E700BF284A00204021002094F86A312F
:10E6D800002B40F0FB87E04B1B6803F00802002A80
:10E6E80048F603414AF60B404BF60F4249F60747F6
:10E6F80004BF02460F4613F0040F4FF0190118BF6C
:10E7080017469A0684F86A1103D547F4804747F0FC
:10E71800200703F035FAC7F30909002841F05184AE
:10E72800CE4B9B79002B41F0BA84984664204FF079
:10E73800FF3A4FF0000C0A970B97ADF834C0CDF8AC
:10E748003AC0CDF83EC0CDF842C0CDF83090ADF813
:10E758003680ADF838A08DF846000AAF0FCFDFF845
:10E768000CE384F805C0AEE80F0097E80F00AEE8A8
:10E7780007002EF8023B71464FF0010C1B0CFE27D8
:10E788001F20C82201F81E39A770A27184F807C09B
:10E79800E07094F87A01207180F0F10383EA0313A2
:10E7A800DAB2130983F0E70343EA022383EAC203D8
:10E7B8001BB283EA0312D2B2C3F3072383EA12130C
:10E7C80043EA022383EAC2031BB283F0C80282EA47
:10E7D8000212D2B2C3F3072383EA121343EA0223D5
:10E7E80083EAC2031BB283EA0C0787EA0717FFB262
:10E7F800C3F3072282EA171242EA072200EB0C034E
:10E8080082EAC7070EEB0C0084F87A31278011F8EA
:10E81800013B7B4083EA0313DBB21A0982EA172221
:10E8280042EA032282EAC3031BB29FB281422780D5
:10E83800EDD183F07C0383EA0313DBB24FEA131EA6
:10E848008EEA172E8EEA032E8EEAC30E0FFA8EFE7C
:10E858001FFA8EF9DFF818C2A4F800905FFA8EFE4E
:10E868004FEA192984F8289084F827E00CF5D17824
:10E8780004F1220ADCF80000DCF80410DCF80820B7
:10E88800DCF80C3047460FC70CF1100CD445B846DD
:10E89800F0D1DCF800003860714F9CF8043088F83B
:10E8A800043007F1270884F8C9E184F8CA9117F8F9
:10E8B800011F306816F0CEFBB845F8D194F86B21EB
:10E8C800002A40F0FE866749029B08781B680A21E7
:10E8D80084F86B11002801F0B380DFF898E1012873
:10E8E800BEF80010059141F2C0830228BEF80280EC
:10E8F80001F07E83BEF804100491032801F0BD8363
:10E908000428BEF806A001F0C583BEF808100391DC
:10E91800052801F0BB830628BEF80AC001F0C683AB
:10E928000728BEF80C1001D0BEF80E2094F87A0122
:10E938000A93074687F0300383EA0313DBB24FEAF2
:10E94800131E494806978EF07A0E4EEA032E008869
:10E9580027718EEAC303DFF820E1C0EB00208EFBAD
:10E96800007E8644C017C0EB6E270797059F4FF0BF
:10E97800000967F30F09049F68F31F494FF0000867
:10E9880067F30F08039FCDF82C901BB24FF0000ED1
:10E9980083EA031067F30F0E0027C0B261F30F0775
:10E9A800C3F307236CF31F4E62F31F474FF0000CAD
:10E9B8009DF81C20CDF834E083EA10136AF31F4851
:10E9C800CDF830800E978DF83CC08DF83D2043EA95
:10E9D80000230DF1280883EAC007B8E80F003FB20A
:10E9E80087F0C80989EA0919DFF880E084F805C0CA
:10E9F8005FFA89F9C7F30727AEE80F0087EA191706
:10EA080047EA092398E8030083EAC9031BB283F0A5
:10EA180023074EF8040B87EA0717FFB2C3F3072250
:10EA280082EA1712069B704642EA072203F10108A0
:10EA380082EAC70720F814194FF0230CFE2116228A
:10EA4800C82384F87A8127800EF1020E84F807C063
:10EA5800A170E270A37111E0B0480020A048002026
:10EA6800E3220020DC5B0020EC3B00204821002052
:10EA7800422100203C3C00200308208010F8013B84
:10EA88007B4083EA0313DBB21A0982EA172242EABF
:10EA9800032282EAC3031BB29FB270452780EDD1DF
:10EAA80083F0F40383EA0313DBB21A0982EA17221C
:10EAB80082EA032282EAC3031BB21FFA83FEE74FEE
:10EAC800A4F800E05FFA83FC4FEA1E2984F81EC010
:10EAD80084F81F907968BA683868FB6807F5D17EB2
:10EAE800AEE80F0038697969BA6904F2C118AEE86E
:10EAF800070004F2A31784F8C19184F8C0C117F87D
:10EB0800011F306816F0A6FAB845F8D194F872716A
:10EB1800002F40F0E485D24B94F87AC1B3F9001085
:10EB2800B3F90220B3F904309FEDCE6A677107EE9E
:10EB3800103A029B1B680A938CF06A0383EA03135A
:10EB480006EE901AD9B20B0983F0D50343EA0123E4
:10EB580083EAC1031BB283EA03115242C9B207EE2A
:10EB6800902AC3F3072383EA111343EA0123F8EE3B
:10EB7800E77AF8EEE66AB8EEC77A83EAC1031BB211
:10EB880067EE867A66EE866A27EE067A002083F0BC
:10EB9800C80ECDED0C7ACDED0B6A8DED0D7A0E9089
:10EBA8000F9010908EEA0E180DF128095FFA88F878
:10EBB800C3F3072EB9E80F008EEA181E4EEA082E96
:10EBC8008EEAC80EDFF8B0820FFA8EFEA8E80F00B2
:10EBD8008EF01E0799E8070087EA071A5FFA8AFA93
:10EBE800CEF3072787EA1A1747EA0A2788E80700B3
:10EBF80087EACA071C214FF0050A4FF01E094FF09B
:10EC0800FE0EC8220CF10103E17084F872A184F8A9
:10EC1800079084F802E0A8F11001A27108F10C0035
:10EC280084F804C0278084F87A3111F8013B7B40CE
:10EC380083EA0313DBB21A0982EA172242EA0322A3
:10EC480082EAC3031BB29FB281422780EDD183F0D1
:10EC5800270383EA0313DBB21A0982EA172282EA3E
:10EC6800032282EAC3031BB21FFA83FCDFF8EC819C
:10EC7800A4F800C05FFA83FE4FEA1C2C84F825C074
:10EC880084F824E008F5D17904F1220AD8F80000C4
:10EC9800D8F80410D8F80820D8F80C304F460FC719
:10ECA80008F11008D045B946F0D16F4FB8F80030D8
:10ECB800A9F8003007F1240884F8C6E184F8C7C130
:10ECC80017F8011F306816F0C5F9B845F8D194F85F
:10ECD80073310293002B40F0FE8494F87AA1604BC4
:10ECE800624AB3F90410B2F90620614F6148DFF8AF
:10ECF80088E184F804A08AF0220383EA03135FFA08
:10ED080083FC4FEA1C1383F0590343EA0C2383EA7C
:10ED1800CC031BB2B2F5FA6F83EA031C5FFA8CFCD2
:10ED2800A8BF4FF4FA62C3F30723B2F57A7F83EAE8
:10ED38001C1343EA0C23B8BF4FF47A7283EACC035E
:10ED4800A2F57A724FF0640C0CFB02F287FB027C8E
:10ED580080FB0170D217C9174FF000091FB2C2EB30
:10ED6800AC12C1EBA0030DF12808CDF82890CDF81E
:10ED78002C90CDF83090CDF8349087F0C80CADF8D1
:10ED88003A20ADF83830C146B9E80F008CEA0C1CBF
:10ED98005FFA8CFCC7F3072787EA1C1747EA0C279A
:10EDA80087EACC07AEE80F003FB287F04A0383EA50
:10EDB8000311C9B2C7F3072383EA111343EA0123F6
:10EDC800724683EAC103D9F800C09DF80810617142
:10EDD8000AF1010705204A214FF0FE0984F87A71EB
:10EDE80042F810C914274FF0C80C84F87301238027
:10EDF8000EF1040EE17184F80290E77084F806C001
:10EE0800184612F8011B414081EA0111C9B20B09E9
:10EE180083EA102343EA012383EAC10109B288B2D5
:10EE280072452080EDD181F0140181EA0111C9B247
:10EE38004FEA111E8EEA102E8EEA012E8EEAC10EBE
:10EE48000FFA8EFE1FFA8EF94FEA192C034B03486E
:10EE580084F81DC05FFA8EFE10E000BF422100203A
:10EE6800B448002088C3E43AE32200203C3C002058
:10EE7800D34D6210676666664821002084F81CE05E
:10EE8800D94F59689A680068DB68A4F8009007F5BC
:10EE9800D179A9E80F0038697969B7F818A0A9E805
:10EEA800030004F2A317A9F800A0BA4684F8BFC16A
:10EEB80084F8BEE104F2BF191AF8011F306816F091
:10EEC800C9F8D145F8D1C94BC94A1B781278013B1A
:10EED80012F00100DBB214BFC0214021172B03D868
:10EEE800C44A13441B7B0293C34B1A8893071ABF67
:10EEF800002341F01001012312F4027F18BF0223FE
:10EF080012F0100F18BF062312F0200F18BF10239D
:10EF1800002840F0BF864FF0030994F87AC10A939D
:10EF28008CF0460383EA0313DAB2130983F09203E1
:10EF380043EA022383EAC2031BB283EA0310C0B286
:10EF4800C3F3072282EA101242EA002282EAC002D0
:10EF580012B282F0C80E8EEA0E1E00235FFA8EFEF1
:10EF68009DF808A08DF82CA00320C2F307228DF885
:10EF78002F9082EA1E128DF82D308DF82E108DF804
:10EF8800300042EA0E2998E8070089EACE0E0FFA07
:10EF98008EF8DFF86CE2E37188EA0819AEE803003E
:10EFA8005FFA89F9C8F3072888EA191848EA092195
:10EFB80081EAC90994F808808EF800200FFA89F9C7
:10EFC80088EA090282EA02185FFA88F8C9F3072278
:10EFD80082EA181242EA0822607AA17A94F80B9021
:10EFE800637182EAC80212B2504080EA0010C0B2CF
:10EFF800C2F3072282EA101242EA002282EAC00221
:10F0080012B2514081EA0111C9B2C2F3072282EA61
:10F01800111242EA012282EAC10212B289EA020905
:10F0280089EA09195FFA89F9C2F3072282EA1912F3
:10F0380042EA092294F80C80607BA17B84F804C022
:10F0480082EAC90212B288EA020888EA08185FFA56
:10F0580088F8C2F3072282EA181242EA082282EAF2
:10F06800C80212B2504080EA0010C0B2C2F30722B0
:10F0780082EA101242EA002282EAC00212B2514029
:10F0880081EA0111C9B2C2F3072282EA111242EAE7
:10F09800012282EAC102E17B94F8109013B281EA5E
:10F0A800030282EA0212D2B2C3F3072383EA1213DD
:10F0B80043EA022383EAC2031BB289EA030282EA13
:10F0C8000212D2B2C3F3072383EA121343EA0223DC
:10F0D80083EAC2031BB283F0320282EA0212D2B27E
:10F0E800C3F3072383EA121343EA022383EAC20322
:10F0F8001BB29AB24FF0FE08DBB222800920C82169
:10F108000CF1010C84F802804FEA1228AEF10E02CD
:10F11800E070A17184F87AC184F812800293637454
:10F1280051685EF80E0C92683EF8023C0EF5CA7CF7
:10F13800ACE80700ACF800309DF808308CF8029075
:10F148000EF5D27A84F8B48184F8B33117F8011F28
:10F15800306815F07FFFBA45F8D1C4F864B1FFF7FD
:10F16800E0B9DFF8A0A0DFF8A080DFF8A090412088
:10F178000FF088F8BAF9023088FB0320DB17C3EBDD
:10F18800A00080B20FF064F8BAF9003088FB0320C1
:10F19800DB17C3EBA00080B20FF05AF8BAF90430BD
:10F1A80088FB0320DB17C3EBA00080B20FF050F8F8
:10F1B80099F80010386815F04DFF94F85C3113F099
:10F1C800010800F097830D4AC4F858B10133DBB247
:10F1D800A2FB0312D20802EB8202A3EB420384F8DB
:10F1E8005C31FFF77EB900BF422100207C3000204F
:10F1F800186F0020EC05030804490020CDCCCCCCC6
:10F2080048210020B448002067666666B15B00208C
:10F21800894B8A49186815F0E9FE00232370FFF727
:10F22800D8B9874F386800283FF44AA94FF0000A38
:10F23800DFF83C82834CAB46554615F007FFF8B122
:10F24800F5B94FF00109AA46386815F0F7FE83B200
:10F258007E2B00F01F8298F80120002A49D194F8EB
:10F268004811B1B11B2B84F8482100F0ED810D2B1A
:10F2780045D0386888F8019015F0E8FE0028E3D1F9
:10F28800AA4650460AAA70495D460FF013F8FFF7E0
:10F2980017B97D2B00F0CB8394F84C2122B180F074
:10F2A8002003DBB284F84C1194F84721062A10D8C1
:10F2B800B4F84A1138681944A4F84A11A11801325F
:10F2C80081F8503184F8472115F0C0FE0028BBD1E1
:10F2D800D6E7B4F84A2188F8019013449BB21A0A79
:10F2E80052FA83F3FF2BA4F84A31386802D1574DFC
:10F2F800A3E7386815F0AAFE0028A5D1C0E738684A
:10F30800A4F84A2115F0A2FE00289DD1B8E794F888
:10F31800B832C4F8B452012B40F2E18294F8B92211
:10F328004B49981801EB8001013202F001024E6A44
:10F3380084F8B922BEB1474F0B970DF14808123F28
:10F34800A52348F8207D802284F81031152329460A
:10F35800404684F8112184F81231B047002840F063
:10F36800438294F8B8323C4A013382FB0312A2EB81
:10F37800E37202EB42029B1A84F8B832FFF7E1B855
:10F38800364A374B92F80BE0029A1B881068D4F87B
:10F3980034213449801A4FF47A72DFB202FB0EF23C
:10F3A8001B0A8F770F7590424FF00007CB774B758C
:10F3B8008F700F7180F080822B4B2C481A689B68E5
:10F3C800C4F8305180FB02E7D21780FB03E0C2EBA0
:10F3D800A702DB17C3EBA00310124FEA232C4FF050
:10F3E800F40E0A770127487781F8203030207522FB
:10F3F800782381F821C081F81AE0CF7681F82200BD
:10F4080081F8232081F82430FEF7ECBFDFF8649000
:10F41800D9F8000015F00EFE00283FF470A8D9F8BE
:10F428000000012115F002FE0222002387F8742053
:10F4380088F80030FFF763B8144A002068490020B4
:10F448001049002040210020862200209022002020
:10F45800EC0503086522002056555555C06200206A
:10F46800B8620020E4490020E4460020676666662A
:10F478000C0000200C5E00205E209047D8F8003079
:10F4880002209847FF2015F0E5F90378FF2B00F0DC
:10F49800668390F90130DF17FFB2D8B20FF0F2F9A6
:10F4A80038460FF0EFF9D8F800305E209847D8F8C2
:10F4B800003003209847FF2015F0CCF90378FF2B84
:10F4C80000F04A83B0F90830D8B2C3F307270FF029
:10F4D800D9F938460FF0D6F9B34B1B78042B74D002
:10F4E800DFF8F0A2B4F82E219AF80010DFF8E892BD
:10F4F80092FBF1F301FB13239BB2B9F80020A4F8A7
:10F508002E311F01BFB2642303FB02134900B3FB72
:10F51800F1F347EA0327C3F303225E20D8F800304B
:10F52800BFB217439847D8F8003006209847F8B27A
:10F538000FF0A8F9380A0FF0A5F99C4AB4F82E3153
:10F54800517AB9F8009001330129A4F82E3100F05E
:10F558006985537B09EB89091FFA89F9002B40F06B
:10F56800A383D8F80030924F5E209847D8F800302F
:10F578003A209847A7FB09377F091FFA87FA5FFAED
:10F588008AF00FF07FF94FEA1A200FF07BF9D8F8CC
:10F5980000305E209847D8F800303B209847642315
:10F5A80003FB17939BB28348053380FB0320DB17CB
:10F5B800C3EBA000C0B20FF065F900200FF062F9AC
:10F5C8007D4FBB79002B40F0F58294F82C31D8F8A8
:10F5D8000020FEF7F4BEDFF804929FED788AA9F1C7
:10F5E800300A4FF0240B5E2090475846D8F8003078
:10F5F8009847BAF81430F9EC016A07EE103AF8EEB9
:10F60800E66AB8EEC77A0BF1010BC6EE877A5FFAA5
:10F618008BFB67EE887AFDEEE77ACDED027ABDF9CD
:10F628000870F8B20FF02EF9C7F307200FF02AF987
:10F63800BBF1270F02D0D8F80020D4E794F82C317A
:10F64800D8F80020FEF7B7BE386815F0FFFC002890
:10F658007FF40FAE386884F8469188F8019015F069
:10F66800F5FC00287FF4F0AD0AE6FCF703F9544BEB
:10F678001B68A0EB030B40F6B8339B4500F2CC8126
:10F68800504B1A793A2A00F0E183002388F80030B9
:10F69800FEF735BF386884F846A184F847A184F896
:10F6A800489188F801A015F0D1FC00287FF4CCAD72
:10F6B800E6E594F8441194F8453143484A1CFEF7AE
:10F6C800EBBE013A84F86B21FFF720BA013B84F8BE
:10F6D8006A31FFF7F3B8013B84F873313DE5013F28
:10F6E80084F87271FFF7F3BA4FF0000A5E201F68C2
:10F6F80084F82CA19047D8F80030DFF8E490172060
:10F70800984750460FF0BEF8304BA3FB07239B0BDE
:10F71800A9FB03125209C2EB0212A3EB8203D8B26F
:10F728000FF0B0F8D8F800305E209847D8F80030CD
:10F7380018209847264BA3FB07239B09A9FB031214
:10F748005209C2EB0212A3EB8203D8B20FF09AF867
:10F7580050460FF097F8D8F80020FEF735BE002481
:10F76800DFF8808027464FF0500A02E0DBB283F3CF
:10F77800118816F804B0601C594630440EF070FC2D
:10F78800002840F067810BF101031C44EFF311835B
:10F798008AF31288326E9442E8DB0022DBB23266CA
:10F7A80083F31188FEF787BFEF3B0020C06200207B
:10F7B8001F85EB5167666666A048002000007A4402
:10F7C800EC5C0020D45C00201449002073B2E745AB
:10F7D800D34D6210CE620020B8620020EC480020B1
:10F7E8008988888805E901080A9EBE4240F2328469
:10F7F8003D46002141F2210015F8013B81EA03232F
:10F80800590013F4004F80EA010289B292B208BF8E
:10F818000A46530012F4004F80EA03019BB289B2F2
:10F8280008BF19464B0011F4004F80EA03029BB24F
:10F8380092B208BF1A46530012F4004F80EA03013F
:10F848009BB289B208BF19464B0011F4004F80EAF9
:10F8580003029BB292B208BF1A46530012F4004F3B
:10F8680080EA03019BB289B208BF19464B0011F424
:10F87800004F80EA03029BB292B208BF1A465100B9
:10F8880080EA010312F4004F9BB289B218BF1946EF
:10F89800B542B1D14046F2F72DFEB4490A9DB448AD
:10F8A8006D1A152DA8BF15252A461FF04DFBB14A24
:10F8B80094F8B832157056E5AF4B029A1B78126867
:10F8C800C4F83421013B012B3FF676AD1022022308
:10F8D8008A700B7170E50EF0B7FFFEF7E5BDA74A19
:10F8E80002EB8302566A25E50EF09EFF01233B706A
:10F8F800FEF797BDA24B1B88D90515D4DA0600F18F
:10F908007E83980600F1A083590600F1A5831A07A3
:10F9180000F1A583D80700F1A58313F0020F0CBFEF
:10F928004FF004084FF00C08964B974A1B78D27892
:10F9380003F001030AB143F00203532003930EF0CE
:10F94800A1FC924A128802EB820202EB820290002A
:10F9580080B20EF07DFC00200EF07AFC8C4A8D49B6
:10F9680012883868C2EBC212520081FB023111447E
:10F978004FEAE27ACAEB612A5FFA8AFA514615F031
:10F9880069FB99F80020039B386848EA03088AEA6B
:10F99800020A002189F800A015F05CFB414638688E
:10F9A80015F058FB99F80030386888EA0303DBB291
:10F9B800194689F8003015F04DFB94F85C31002B9E
:10F9C8007FF401AC4F200EF05DFC10F06BFB10F0E3
:10F9D80069FB10F067FB0121386815F03BFB6E4AA4
:10F9E80099F8003092F80080386808F0010841461C
:10F9F80083F0010389F8003015F02CFB99F80030EA
:10FA0800386888EA0308414689F8008015F022FB27
:10FA180094F85C31FFF7D7BB604AB2F85E31002139
:10FA28000133A2F85E3188F80010FEF768BD386827
:10FA380084F84C9115F00AFB00287FF405AC1FE40C
:10FA4800014684460390824604908046059002460B
:10FA5800FEF76CBF41463A2015F000F80743FFB2A5
:10FA680091E64F494F4B0093A1F13F074E4B4F4A48
:10FA7800099101F8404C0AA84D490897F2F712FE7F
:10FA8800089F7B1C08933C70089B2922591C0891ED
:10FA98001A70089BEA22591C08911A70089BC82200
:10FAA800591C08910AA81A701EF0E0FA00F1010822
:10FAB8000AA9424608981FF047FA089A02EB080379
:10FAC8000133089302F80840089B5A1C08921C70DE
:10FAD800089B5A1C08921C70089B5A1C08921C70A0
:10FAE800089B5A1C08921C70089B5A1C08921C7090
:10FAF800089B5A1C08921C70089B5A1C08921C7080
:10FB0800089B5A1C08921C70089B5A1C08921C706F
:10FB1800089B5A1C08921C70089B5A1C08921C705F
:10FB2800089B5A1C08921C70089B0122991812A85D
:10FB380008911A7050F8283DDB1B3B700EF0C4FE8C
:10FB4800164B3470C3F8AC52FEF7EFBCC4F838510A
:10FB580087F80080FEF765BC00273846B7E43846CA
:10FB68009CE415F063FAFEF771BC00BF5022002038
:10FB7800BC340020D1340020EF3B0020EC05030802
:10FB880004490020186F0020F43B0020B8620020D0
:10FB9800EC3B002003082080883000204021002012
:10FBA8006849002066630020C8290308D029030893
:10FBB800DC290308D8F80030DFF888A2DFF8809243
:10FBC8005E209847D8F8003028209847DAF80030A7
:10FBD80089FB0329DB17C3EBA9095FFA89F00EF04B
:10FBE80051FEC9F307200EF04DFED8F800305E2014
:10FBF8009847D8F80030042098473B89002B40F0FC
:10FC08000182DAF8087087F31007F8B20EF03AFEAE
:10FC1800C7F307200EF036FED7E47D4B0B93A3F114
:10FC2800400800222121A3F13D0903F8402C88F85F
:10FC3800021088F80120CDF8289013F087FC754B46
:10FC4800754A1B88754900280ABF114603270427EF
:10FC5800580500F1E481DA0700F1F98103F00203A5
:10FC68006F4A002B1CBF032711463A466D481FF008
:10FC78006BF909EB070312A86B4A013340F8203DE2
:10FC88009B1A002209F8072088F801300EF01CFEA4
:10FC9800FEF7C4BC654AD278002A0CBF4FF00409AD
:10FCA8004FF00509FFF739B99AF8003099FBF3F9D5
:10FCB80057E40123D9F800003B7015F0BFF9074657
:10FCC800D9F8000015F0BAF97F067EF4AAAB8E28A1
:10FCD8007EF4A7AB9AF80030002B7EF4BEAB544BF1
:10FCE800544A1A602D2384F83C31FEF7A1BBDFF893
:10FCF80058919FED518AB9F90230454A0B9207EEA7
:10FD0800903AF8EEE77A0DF1480867EE887AA2F1A2
:10FD18004003FDEEE77AA2F13D0148F8201D02F804
:10FD2800400C0822CDED027A5A701E229A70BDF856
:10FD380008104046F2F7B8FBB9F9003007EE903AE0
:10FD4800F8EEE77A404667EE887AFDEEE77ACDED81
:10FD5800027ABDF80810F2F7A7FBB9F9043007EEEC
:10FD6800903AF8EEE77A404667EE887AFDEEE77A51
:10FD7800CDED027ABDF80810F2F796FB40460EF07A
:10FD8800A3FDFEF745BC224A2C4B0B920DF1480807
:10FD9800A2F13D0048F8200D1988DFF8A890A2F1DB
:10FDA800400300204FF00A0E02F8400C082283F8A6
:10FDB80001E040469A70F2F777FBD9F80030204905
:10FDC800DA1781FB0313C2EBA30399B24046F2F79B
:10FDD8006BFB01F0E3FED9F808900A9B4FEA194241
:10FDE800591C0A911A700A9B4FEA1922591C0A9148
:10FDF8001A700A9B5A1C0A9283F800900A9B5A1C94
:10FE08000A92187040460EF05FFDFEF704BC00BF72
:10FE18006849002004490020AC290308B4290308D4
:10FE2800C42903082B49002029490020F43B00205D
:10FE38001C490020E449002058A08B41B8620020EA
:10FE480067666666E4460020B44800209978039304
:10FE5800184611F0C7FB00287FF417AC9549964F58
:10FE6800964A974C0988DFF86C929368F961116893
:10FE7800B4F85E21F863C7F86CB0FB64F962D9F88E
:10FE88000000FA6514F01AFF834600287EF432ABAE
:10FE98005146D9F8000015F0C9F8039B94F8602181
:10FEA800DB780493642A4FF0040387F8743040F039
:10FEB800178194F86131DFF820A2072B08BF84F876
:10FEC80061B194F86121069207EB021BDBF804107C
:10FED800059108461EF0CAF8DBF8083003935FFA6C
:10FEE80080FB18461EF0C2F8C3B20BEB0300069A5B
:10FEF8000599059308308AF8070022F00F008AF860
:10FF08000A0002F00F0203EBCB008AF80D208AF8F2
:10FF18000E005A460AF10F001FF016F8059B0399C8
:10FF28000BF109001A460AF1060318441FF00CF8F1
:10FF38009AF8073003F1010BD3B1013B5FFA83FC58
:10FF48000CF1080CDFF894E1D4440AF1070000230F
:10FF580010F8011B59408B00CA0883EA410302F0DC
:10FF680018024B404EFA02F253408445DBB2EFD1FF
:10FF7800544A04980BF802301EF032FF94F86131AD
:10FF88000022013384F8613184F860219AF8023044
:10FF98005BB11AF80610D9F8000015F05BF80136C5
:10FFA8009AF80230F6B2B342F3D894F860310322DB
:10FFB800013384F8603187F8742088F80020FFF74F
:10FFC80027BA3C4B404A1B88927903EB830303EB27
:10FFD80083034FEA83081FFA88F8002A53D0374B67
:10FFE8001B680FFA83FA01F0D9FD40B2FEF7A1BBF6
:08FFF800114694460392924663
:020000040801F1
:100000000492FEF797BC4FF0340891E401F0CAFD6A
:100010000EF03CFC00200EF039FC94F82C31D8F89E
:100020000020FEF7D0B903272A4922E6D8F800308D
:100030005E209847D8F80030392098475FFA89F059
:100040000EF024FC4FEA19200EF020FCFFF7BCBA9A
:100050004FF024086CE4204904270AE600211DE43F
:100060004FF0100864E44FF0200861E44FF00808F6
:100070005EE4114694460392924604929046FEF73F
:1000800059BC1146944603929246FEF753BC4FF07A
:10009000FF33AAE711469446FEF74CBC114694463E
:1000A0000392FEF747BC074B8046B3F900A06420DB
:1000B000FEF743BB1146FEF73DBC00BFB86200200F
:1000C0000C000020E446002040210020824F002048
:1000D000A0480020B8290308BC2903080C5E0020B2
:1000E0007C4F00200007090E97F87530DFF81CA13F
:1000F0000596190704BF0133DBB2072B28BF012384
:100100004FEA031B07EB0B023D49107C00228AF8E3
:100110000A2011F800C05FFA8BF203920AF10D0277
:10012000039E07EB0B013043BCF1010F1070C9684F
:1001300002F101000ED9ACF10206F6B206F1020E90
:100140009644024602F8011B72454FEA1121F9D18B
:1001500001363044BB4421F0600201339BF811109A
:10016000DBB20A43082B027000F1010244D04FEACF
:10017000031B07EB0B00224E007C224916F800C03F
:10018000039E511A06F1100E01EB0C0606965FFA5B
:100190008EF60396069E132EC2DD059EDFF870E0F4
:1001A000C9B28A1DD2B242F040008AF8070002F1BB
:1001B000010BCAB14A1DD2B20832524403920EF169
:1001C000010C00221CF8010B5040820082EA400220
:1001D000C10842400C4801F0180140FA01F14A40C0
:1001E00003996145D2B2EDD104980BF80E2087F83F
:1001F00075301EF0F9FDCDE60249059E511ACDE796
:10020000EC050308894F00200007090E7C4F0020F1
:10021000824F002008B512F09BFC024B024ADA60C4
:10022000FEE700BF00ED00E00400FA05024A034BC0
:10023000127819780BF062BEC01F0020C11F002089
:100240002DE9F04F2DED028BA0F10A0389B00C4689
:10025000ED2B00F26086DFE813F022015E065E06F9
:100260005E065E065E065E065E065E065E065E066E
:100270005E065E065E065E065E065E065E065E065E
:100280005E065E065E065E065E062F025E065E0681
:100290005E062C065E065E065E0699015E06560147
:1002A0005E063E015E0633015E0628025E0603021C
:1002B0005E06EF015E065E065E06EA01E4015E068A
:1002C000D2015E065E06CC015E06A5015E065E06F4
:1002D0005E068A045E065E065E065E066C045E06C8
:1002E00002015E063B0629055E065E065E065E06A8
:1002F0005E065E065E06FD045E06CF045E069C0496
:100300005E0665055E064A065E065E065E065E06DB
:100310000503F105EA05B905EE005E065E06280351
:10032000A6025E066F02E9025E065E065E065E06D5
:10033000DE025E065E06BD025E065E065E06AF0279
:10034000F303BB037A035E065E065E066C035E067D
:100350005E064C035E065E065E065E065E065E0692
:100360005E065E065E065E065E065E065E065E066D
:100370005E0605035E065E065E065E065E065E06B9
:100380005E065E065E065E065E065E065E065E064D
:100390005E065E065E065E065E065E065E065E063D
:1003A0005E065E065E065E065E065E065E065E062D
:1003B0005E065E065E065E065E065E063E035E0640
:1003C0005E065E065E065E065E065E065E065E060D
:1003D0005E065E065E065E065E065E065E065E06FD
:1003E0005E065E065E065E065E065E065E065E06ED
:1003F0005E065E065E065E065E065E065E065E06DD
:100400005E065E065E065E065E065E065E065E06CC
:100410005E065E065E065E065E065E065E065E06BC
:100420005E065E065E06620438045E065E065E06D2
:100430005E065E060904AF4E337853B1AE4F002519
:1004400037F8021F2046F2F759F833780135AB42EE
:10045000F6DC012009B0BDEC028BBDE8F08FA54EA3
:100460003378002BF5D0A54F0025B846236817F840
:100470001520591C21601A7098F8011001EB8101B8
:1004800001EB810101F2EE2189B22046F2F736F844
:1004900033780135AB4208F10208E7DCD9E7984D23
:1004A00028461DF0E7FD0028D3DD2B4605442268D1
:1004B00013F8011B501C9D4220601170F7D1C8E752
:1004C000904D05F1800655F8041F2046F1F7FEFF18
:1004D000AE42F8D1BDE78C4D05F14006B5F880106D
:1004E0002046F2F70BF8236895F88220591C21600A
:1004F0001A70236895F883200435591CAE42216098
:100500001A70EBD1A5E7814D0B682A7A591C21603E
:100510001A70A98B2046F1F7F1FF298B2046F1F7DD
:10052000EDFF698B2046F1F7E9FF2368EA7C591C4F
:1005300021601A70A98C2046F1F7E0FFE98C204673
:10054000F1F7DCFF2368AA7F591C21601A70236829
:1005500095F82020591C21601A70698C2046F1F70B
:10056000CDFF2368EA7A591C21601A70E968204699
:10057000F1F7ACFF23682A7C591C21601A702368AC
:1005800095F82120591C21601A7062E70B68604AB7
:10059000581C11782060197023685278591C21600A
:1005A0001A7056E70B685A4A5A4D11785A4A581C25
:1005B0002060197011682046F1F788FF2368534ABC
:1005C000591C127A21601A7029882046F1F796FF8B
:1005D000A9882046F1F792FF29892046F1F78EFF7E
:1005E00020460021F1F78AFF20460021F1F786FF1F
:1005F0002FE7084608224549F1F750FF29E70B6825
:10060000464A474990785D1C2560187023685278E7
:10061000581C20601A7023680A79591C21601A70CE
:1006200017E70B680122991821601A7011E7084634
:100630000021F1F74BFF0CE73A4D3B4E05F1300737
:1006400095F90210394B93F906208A4203F1080309
:1006500000F064849E42F6D10835BD42F0D1F8E640
:10066000334B03F15A0522685979501C20601170F0
:1006700022681978501C2060117022685978501C2B
:100680002060117022689978501C206011702268D7
:10069000D978501C20601170226819790633501CDB
:1006A0009D4220601170DED1D3E60B68174A591CB9
:1006B000527D21601A70CCE61E4D05F15006287857
:1006C00018F0A4FD2368027A591C21601A7023686F
:1006D0006A78591C21601A702368AA78591C216015
:1006E0001A702368EA780435591CAE4221601A70EA
:1006F000E5D1AEE6DC5B00203A3C0020805E0020C5
:10070000C42F0020643A0020683A002024710020A1
:100710007C300020882C0020E0640020083000207D
:10072000C41F0020507100204C4F00201C4F00209F
:10073000EC380020705D0020AF4D0B682A68591C12
:10074000127821601A702B6822689978531C2360F4
:10075000002311702A6821681A4401335279481C19
:10076000032B20600A70F5D123682A68591C127A7D
:1007700021601A7023682A68591CD27821601A7087
:1007800023682A68591C127921601A702B68204648
:100790005989F1F7B3FE2A682368527A591C2160FF
:1007A0001A702A68F8E620460021F1F78FFE2046ED
:1007B0000021F1F7A3FE4CE6904D08462988F1F799
:1007C0009DFE69882046F1F799FEA9882046F1F739
:1007D00095FE3EE68A4D05F16006A9882046F1F7B0
:1007E0008DFEE9882046F1F789FE29892046F1F738
:1007F00085FE2368AA7A591C21601A702368EA7A58
:10080000591C21601A7055F80C1B2046F1F75EFE4A
:10081000B542E2D11DE67B4952232268501C20607C
:10082000137011F8013F002BF7D112E67648002330
:100830002268056803EB4301561C6D5C2660157049
:10084000026825680A446E1C527826602A70026885
:1008500025680A4401339278691C0A2B21602A70AA
:10086000E6D1F6E500258146DFF8C881DFF8C8B19A
:10087000049503950595069501214FF6FF7A05E04D
:1008800001350B2D00F0688318F9011F4F1C4AFA3F
:1008900005F3F5D0DE07F3D5BBF800302B41D807C0
:1008A000EED505A8F2F7DEF9EAE7584D08462988A3
:1008B000F1F724FE69882046F1F720FEB5F90430EF
:1008C000534AD91782FB0323C1EBA301204689B207
:1008D000F1F714FEBDE50B684E4A591C12782160F1
:1008E00005A81A70F1F7FAFC23685A1C22601870E8
:1008F000AFE50B68484F591C3A7821601A703B7875
:10090000002B3FF4A6AD0025EEB2304613F0A6FF53
:1009100023684278591C216030461A7013F09EFFFC
:1009200001892046F1F7EAFD3B780135AB42EBDC6B
:100930008FE53A4D0846298AF1F7E0FD698A20469D
:10094000F1F7DCFDA98A2046F1F7D8FD81E5DFF853
:10095000ECE00027FEB2714600232268501C2060A4
:1009600016702268501C20601370226811F8010F65
:100970000133551C062B25601070EED10137062F70
:100980000EF1060EE6D1264900232268501C206095
:1009900017702268501C20601370226811F8010F34
:1009A0000133551C0B2B25601070EED123681D4AB6
:1009B000581C07212060197023680021581C2060F2
:1009C0001970236892F8F020591C21601A7040E5D4
:1009D0000B68154A15491078154A5D1C256018707A
:1009E00023688978581C2060197023689278591CF4
:1009F00021601A702DE500BF0C4900202061002005
:100A0000343700202006030808490020B44800209D
:100A100067666666E6350020AD610020CC4B00209D
:100A20004B3B0020683A0020446B0020E82F002058
:100A3000F82F00205006030804490020273B00201F
:100A40000A68AC4BAC491878551C256010702268B8
:100A50005878551C2560107022689B78501C2060C7
:100A600013702046C988F1F749FDF2E405A8F1F7B3
:100A700035FC00283FF4EDACBDF814102046F1F72A
:100A80003DFD23689DF81620591C21601A702368CB
:100A90009DF81720591C21601A7023689DF81820B2
:100AA000591C21601A7023689DF81920591C216077
:100AB0001A7023689DF81A20591C21601A7020466C
:100AC000BDF81C10F1F71AFDC3E48C4B03F170055F
:100AD00022681978501C2060117022685978501CC7
:100AE0002060117022689978501C20601170226873
:100AF000D978501C2060117022681979501C206030
:100B0000117022685979501C2060117022689979FF
:100B10000733501C9D4220601170D9D199E4784D63
:100B20000846E989F1F7EAFCA9892046F1F7E6FCD5
:100B30008FE40B68734D591C2A7921601A70236861
:100B40006A79591C21601A7029882046F1F7D6FC71
:100B50002368AA79591C21601A7069882046F1F728
:100B6000CDFC2368EA79591C21601A7071E40B6886
:100B700000255A1C0A60204629461D70F1F7A6FC84
:100B800029462046F1F7A2FC29462046F1F79EFCB3
:100B90005FE45D4E0B6872795C4D591C21601A70E0
:100BA0002B682046198CF1F7A9FC2B682046D98BBD
:100BB000F1F7A4FC71892046F1F7A0FCB189204629
:100BC000F1F79CFC2B682046598CF1F797FC2B68B9
:100BD0002046998CF1F792FCF1892046F1F78EFCC2
:100BE000318A2046F1F78AFC2A68236892F8262089
:100BF000591C21601A702CE4434EF378002B00F04E
:100C00007E820B680822591C21601A702368012219
:100C1000991821601A7023683D4D591C2A7921606A
:100C20001A702368AA78591C21601A7029882046F6
:100C3000F1F764FCE9892046F1F760FC2368F2795A
:100C4000591C21601A702368EA78591C21601A70B7
:100C5000FFF7FFBB0BF046F9FF28054600F06B825B
:100C600008A8002300F80C3D0BF00EF92268294B70
:100C7000511C2160157022681978501C2060117079
:100C800022685978501C2060117022689978501C95
:100C90002060117022689DF81410501C20601170A3
:100CA00020469988F1F72AFCFFF7D3BB0B681A4D51
:100CB000591C012221601A702368AA78591C2160EE
:100CC0001A701BF025FC2368144A15495E1C266027
:100CD0001870B1F90010B2F90000F1F789FD23682E
:100CE0005A1C2260187029882046F1F707FCFFF78C
:100CF000B0BB00BFE02F002020610020F4370020AF
:100D0000E82F002038610020446B002008490020B3
:100D1000CC4B0020206F0020BE640020A86F002074
:100D2000AA6F002020460021F1F7E8FB20460021B1
:100D3000F1F7E4FB20460021F1F7E0FB2368A64D24
:100D400000265A1C22601E7023682A68591C92F8DB
:100D50002C2021601A7023682A68591C92F83620CA
:100D600021601A7023682A68591C92F83720216084
:100D70001A7023685A1C22601E7023685A1C226055
:100D80001E7023685A1C22601E702B682046598FE3
:100D9000F1F7B4FB2B682046198FF1F7AFFB2368FE
:100DA0002A68591C92F82E2021601A7023685A1C58
:100DB00022601E702B682046598EF1F79FFB2B682E
:100DC0002046998EF1F79AFBFFF743BB834D844E83
:100DD0009FED848ADFF84C82DFED838A05F12007DE
:100DE0000EE0FCEEE77ACDED017ABDF80410204666
:100DF0000435F1F783FBAF4206F118063FF429AB47
:100E0000717C0029F3D0794BD5ED007A1B78012B4A
:100E1000E7D1774B1B68DB0440F16781F5EE407A40
:100E2000F1EE10FA40F08F8140F2DC51DFE7084626
:100E300010227049F1F732FBFFF70BBB6E4B9B8A18
:100E4000B3F5006F00F25981B3F5806F00F279813C
:100E5000B3F5007F34BF01270227684D05F10C066A
:100E600055F8041B91FBF7F1204689B2F1F746FBD8
:100E7000AE42F5D1624D634F05F10C06B5EC010AA7
:100E8000D7ED077A80EE270A1EF0A2F981B220463C
:100E9000F1F734FBB542F1D15B4D05F10C0655F885
:100EA000041B204689B2F1F729FBB542F7D1FFF7C1
:100EB000D0BA564D08462988F1F720FBA98820466C
:100EC000F1F71CFB29892046F1F718FBFFF7C1BA9F
:100ED0000B6800255A1C0A601D700B685A1C0A60BA
:100EE0001D700B685A1C0A6029461D7049E60B6884
:100EF000474A4849D078484A5D1C256018702368E5
:100F00004979581C206019702368D278591C2160D7
:100F10001A70FFF79EBA0020FFF79CBA23685A1C8C
:100F20002260197029882046F1F7E8FA2368EA78E8
:100F3000591C21601A7023682A79591C21601A7083
:100F40002368AA79591C21601A7023686A79591C90
:100F500021601A70FFF780BBDFF8CCA000254FF0AE
:100F6000A8080135C5F1200208FA02F2A5F1200314
:100F70002AFA05F6164328FA03F31E43282D06F035
:100F800001024FF000030BD01343EAD0E8B212F095
:100F9000EFFA0028E5D0294605A8F1F763FEE0E75F
:100FA0001E4B1B78DA0700F1B68000251C4E2F4639
:100FB00002E00135282D39D029463046F1F762FE8E
:100FC0000028F6D0294605A8F1F75CFE002840F07D
:100FD00087800137EDE700BF08490020403000203E
:100FE0000C4B00200000404200E08244F04B002007
:100FF000686B002030300020BC480020EC48002006
:101000005C6B0020CC68002068610020882C0020E8
:10101000E82F00209C4A0020F82F0020186F0020A5
:10102000E46C0020DB9B914190E33FF4644B654D01
:10103000B3F850102046F1F761FA00212046F1F78D
:101040005DFA614B19684B0103F02002C1F34003C4
:101050001343C1F3800243EA4203C1F3C00243EAEF
:101060008203C1F3401243EAC20301F010011943A5
:101070002046F1F743FA03A904222046F1F70EFABD
:1010800023682978514A581C2060197011886429F6
:10109000A8BF64212046F1F731FAB9F1960F3FD08D
:1010A00000212046F1F72AFA2168B7F1190348BF59
:1010B000A7F11203A3F3C4034A1C226020461A4678
:1010C0000B7004A9F1F7EAF92368414A581C112171
:1010D0002060197020461168F1F7F8F9FFF7B9B9E7
:1010E000394603A8F1F7BEFD73E7F4EEC87AF1EED6
:1010F00010FA44DA4FF47A7179E60827ADE60B6806
:10110000B178344A581C2060197023681278591C31
:1011100021601A707FE5059B43F00103059344E7C6
:1011200023680322591C21601A7023686A78591CAD
:1011300021601A70B8E723685A1C22601870FFF704
:1011400088B9042789E6F4EEC87AF1EE10FA3FF583
:101150006BAEF4EEE87AFDEEE77AF1EE10FA17EEF8
:10116000901A1ED86FF4F973303903FB01F140F285
:10117000E73391FBF3F101F2DB5189B237E6FDEE83
:10118000E77A40F2E73217EE903A303B02FB03F386
:1011900088FB0312D917C1EB622101F2E93189B250
:1011A00025E640F2F313A1F5836103FB01F140F260
:1011B000E73391FBF3F101F2DD5189B217E600BF8D
:1011C000C406002060630020B0480020EE2C002000
:1011D00000490020DC2F002038B5094D2B8823EA78
:1011E0000000834228800AD0064B1421FF220E20E3
:1011F00002241C7059709A7017F034FE288838BD8C
:10120000044900201C3A002038B5094D2B881843AA
:10121000834228800AD0074B1421FF220E2002248B
:101220001C7059709A7017F01DFE288838BD00BFD9
:10123000044900201C3A0020704700BF30B4034628
:1012400000F12405064C07CC0C3343F80C0C43F892
:10125000081C43F8042CAB42F4D130BC704700BFEB
:101260005C060308034B33F80C2F02809B788370D5
:10127000704700BF5C0603086E4B1B78002B39D00B
:101280002DE9F0416C4B6D4D9B792C682860013B3A
:1012900082B0041B032B00F29B80DFE803F04902BD
:1012A000302812F06BF9002800F09A80644B6549F1
:1012B0001B786A8FD1ED037A6A64DB0700F1A9809D
:1012C00002FB04F007EE900ADFED5F6A5F4BB8EEB9
:1012D000E77AD5ED107A5A60E7EE267A1A60BDEE0D
:1012E000E77AC5ED107A85ED0F7A83ED027A02B0C8
:1012F000BDE8F081554A1360536093607047544BCA
:101300001B681801F3D5FF2013F0A8FA03780A2B05
:1013100088BF00214D4B9CBFB0F90420B0F90610E6
:10132000A96488BF0A46EA645A601A609960DEE7D9
:10133000484A494BD279DFF8308133F81220B8F9A6
:1013400002304648B8F9001092B207EE902A40F6F3
:10135000E44707FB02F6C3EB1633B8EE670A4FF417
:101360007A7606FB03F393FBF1F32B61EEF7E8FFCC
:10137000D5F810E0D5ED027ADFED336AB8F9022036
:10138000324BB8F900C0C3F804E00EFB04F007EEDE
:10139000100AB8EEC77ABCEEC06AE7EE267A8DED89
:1013A000016ABDF80410C5ED027ABDEEE77A07FBCD
:1013B00001F7C2EB173706FB07F683ED027A96FBBF
:1013C000FCF685ED017AEE601E6002B0BDE8F081AA
:1013D0001E4B00221A605A609A6002B0BDE8F0818C
:1013E0001B4B1B68DE067FF561AF154B6A8F1B78C0
:1013F0006A64D9077FF564AFB5F93810184B00FB64
:1014000001F083FB0013C017C0EBA31002446A6411
:1014100056E7FDEEE77A134E17EE900AA0F57A71C3
:1014200001FB01F386FB0306D817C0EB2610084426
:10143000E2E700BFCE620020A04800200024002088
:10144000186F0020D06200202FE33E31E4460020D8
:10145000686B0020C86D0020E86D00201424002077
:10146000D34D62101F85EB51D82F0020F0B53E4BB5
:101470005B79012B83B03DD0022B0FD03B4B002278
:101480001A805A803A4B1B78022B05D1374A394BC8
:101490005188128819805A8003B0F0BD364B1B6802
:1014A0001B01EFD5FF2013F0D9F903780A2B56D88A
:1014B000B0F902203149D31781FB0212C3EBA2031A
:1014C0009BB207EE903AB8EE670A2D4C04F1540037
:1014D000A4F85230EEF734FFFCEEC07A234AB4F899
:1014E0005230CDED017A5380BDF80430A4F850306D
:1014F0001380C7E7234A244B9278214D33F81240DA
:10150000A4B207EE904A05F17C00B8EE670AEEF748
:1015100017FF1E4A1549107896785378FCEEC07A6A
:1015200000EB4010CDED017ABDF8042044F6FB77C6
:10153000C3EB033300FB027200FB0474B2FBF3F253
:10154000B4FBF3F3B2FBF6F2B3FBF6F392B29BB249
:10155000A5F87820A5F87A300A804B8092E79FEDB5
:101560000C0A0023B1E700BFA0480020B8620020A9
:10157000CC610020D0610020686B00206766666641
:1015800000240020C86D0020E86D00205B6300206F
:1015900000000000F8B52D4D2D4968792D4C2E4BDB
:1015A0002E4E042264270A7001284FF0000184F8AF
:1015B000A02084F8A970A4F8A210A4F8A41084F8BC
:1015C000A810C4F8AC1031701980598021D00228BD
:1015D00010D0A979224A00230129136084F8B03081
:1015E0005360936023D0022912D11E4AE3635360F3
:1015F0009360F8BD282204F150001EF0A6FD4CF2C5
:1016000050319FED190A04F15400F1F7E7F9E0E7D2
:10161000F8BD282204F178001EF097FD4CF25031FD
:101620009FED110A04F17C00F1F7D8F9D1E70F4AD8
:10163000636053609360D3609FED0D0A02F1100068
:101640004CF25031BDE8F840F1F7C8B9A04800208D
:10165000EF3B002000240020B8620020CE62002072
:10166000E44600203C240020CDCCCC3D04240020C6
:10167000CDCCCC3E2DE9F04F0C68B94F2588B94E42
:10168000B6FBF2F285B0013B013ABC429BB2ADB26F
:1016900092B2BDF838609DF83CE063D007F5006772
:1016A000BC425FD0B4F1804F5CD0A7F59837BC4204
:1016B00058D007F58067BC4254D0AB4FBC4257D0DE
:1016C00007F58067BC4253D025F4407507F58C3789
:1016D000ADB2BC422580E36222850ED0A34B9C4272
:1016E0000BD003F540639C4207D003F580639C4216
:1016F00003D003F580639C4201D10023238601239C
:1017000063614B79CA79BEF1000F01D082F001020A
:1017100012F0020130D012F0010F4FF040054FF0EF
:1017200000020CBF90464FF0080894460392914681
:101730009646174601924FF4806102954FF0040AD5
:101740000C2B00F2E080DFE813F0AE00DE00DE00DC
:10175000DE008A00DE00DE00DE006500DE00DE0066
:10176000DE002E00804F25F07005BC42ADB2A7D13F
:101770002580E3622285C2E74FF4806512F0010FF5
:1017800003954FF001050CBF0027022702918A46FE
:1017900088464FF480424FF4805C4FF010094FF4BC
:1017A000807E0195CCE7216ADFF8B4E121F4805115
:1017B0002162216A6568D4F81C8021F4005141EA55
:1017C0000C0C744528F4E6414CEA073741F4C0415B
:1017D00000F0E7800EF5006E744500F0E280656071
:1017E000E16126642762E26942F40062E261626CB0
:1017F00042F4004262642288214692B242F0010221
:1018000021F8342B0022CD1844600560CA5005B081
:10181000BDE8F08F226ADFF8489122F480722262DC
:10182000226A6568D4F81CA022F4007242EA0E0E07
:101830002AF0730A4C454EEA07274AF0600200F08E
:10184000A480DFF828E1744500F09F806560E261C4
:10185000E6632762E26942F00802E261C7E7226AB2
:101860003F4D22F010022262226A6168D4F818C04B
:1018700022F0200E2CF080724EEA090922F4E64292
:10188000AC4249EA071742F4C04271D005F5006541
:10189000AC426DD06160A261A6632762A26942F486
:1018A0000062A261A3E7226ADFF8B4C0019D22F0C2
:1018B00001022262D4F820906168A26922F4803289
:1018C0003D4322F0730229F00207644545EA07050B
:1018D00042F0600238D0254FBC4235D007F5406752
:1018E000BC4231D007F58067BC422DD007F5806738
:1018F000BC4229D06160A26166632562A26942F0A0
:101900000802A26173E70C2B3FF671AF01A252F8F7
:1019100023F000BFFD180108EF170108EF170108B9
:10192000EF1701089D180108EF170108EF170108CC
:10193000EF17010855180108EF170108EF17010804
:10194000EF170108E717010825F00C0545EA08051F
:1019500021F4407145EA0A0541EA0E01CAE700BFD9
:10196000002C014000A24A04001000400034014055
:1019700027F08007029D47EA081727F040072F430A
:10198000039D21F44061294384E727F4006747EA77
:10199000082727F4806725F440550F434CEA0505D6
:1019A00054E725F48045154319E700BFF8B5494CC5
:1019B00094F8B4305BB3042829D8474AB4F8CA3045
:1019C0009FED467ADFED466A94F8C85002EB80003E
:1019D00007EE903A0269B4F8CE300E46F8EEE77A98
:1019E000642106EE102A01FB032367EE877AB8EE26
:1019F000C66A07EE103A67EE867AB8EEC77A87EEC7
:101A0000870A20EE260A002D4FD0012D00D0F8BD08
:101A1000D4F8C47007EE907AF8EE677A27EE800A61
:101A20001DF0D6FB70B9D4F8B80013F095FEB4F8E9
:101A3000CC003044F9F7C8FFD4F8B800BDE8F8404E
:101A400013F090BE2749284A48620023CF625362B0
:101A5000D762EFF31183502080F312880D80DBB240
:101A6000158083F31188214BCD60D5601A68B4F8D6
:101A7000CC10114431441A689142FCD819491A4AD1
:101A80000B88D4F8B80023F001031B041B0C0B8057
:101A9000138823F001031B0400241B0C1380CC606B
:101AA000D460BDE8F84013F05DBED4ED317AD4F8CF
:101AB000BC50F8EE677A27EE800A1DF089FB0B4BCD
:101AC00028601B68B4F8CC1019443144C4F8D41011
:101AD000F8BD00BF002400205C0603080AD7233CA1
:101AE000CA269B3E0010004000140040BC7100203C
:101AF00008B5044BD3F8B80013F02EFE024B0022B9
:101B00001A6108BD002400200014004008B5044BF1
:101B1000D3F8B80013F026FE024B00221A6108BD6C
:101B20000024002000100040012800D9704701293E
:101B3000FCD88842FAD030B4084B01EB410103EBEA
:101B4000810100EB400080000D684C688968C55039
:101B5000C2185460916030BCE8E700BF8664002082
:101B600002280649064B074A28BF0220487000EBAE
:101B7000400003EB8000106011F05EBD6063002048
:101B8000866400200C490020044B587920B1044B96
:101B90001878003018BF0120704700BFA04800200F
:101BA000CE6200201F4B1878002839D01E4A1389B6
:101BB000FBB11E4A9FED1E6AD2ED026A07EE903A13
:101BC000F8EEE66AF8EE677A07EE103A77EEE66A24
:101BD000B8EEC77A66EE866AC6EE877AFDEEE77AD9
:101BE00017EE900A6428A8BF642020EAE070C0B213
:101BF000704710B40F4B54781B88117804FB1032D7
